:020000040000FA
:1000000000400020B1670100ED670100EF670100CB
:1000100000000000000000000000000000000000E0
:10002000000000000000000000000000F167010077
:100030000000000000000000F3670100F567010008
:10004000F76701004D960000156C0100F76701008D
:10005000F76701000000000001E90000F7670100F8
:100060004D030000F7670100C5E80000F7670100D5
:10007000F7670100F7670100F7670100F767010004
:10008000F76701006D710100F7670100F767010074
:10009000F767010019A00100F59F01008904000025
:1000A00099040000F7670100000000000000000054
:1000B0000000000000000000000000000000000040
:1000C00010B5064C2378002B07D1054B002B02D02E
:1000D000044800E000BF0123237010BD98020020F7
:1000E000000000001CBE0300084B10B5002B03D01D
:1000F0000749084800E000BF07480368002B00D10B
:1001000010BD064B002BFBD09847F9E7000000001C
:100110009C0200201CBE030098020020000000008A
:10012000164B002B00D1144B9D46402292029A1A86
:10013000924600218B460F461348144A121A2BF0A0
:10014000EBF90F4B002B00D098470E4B002B00D043
:1001500098470020002104000D000D48002802D01F
:100160000C4800E000BF21F063F92000290029F0CD
:1001700029F820F035FEC0460000080000400020AD
:10018000000000000000000098020020280B002062
:100190000000000000000000C46005614661876146
:1001A0004146C161494601625146416259468162F8
:1001B0006946C16271468160124B1A68026018601C
:1001C000002070470F4B1A6812681A6070470D4B79
:1001D0001A68002A01D124F02BFA506010681860C8
:1001E000D468156956699769D1698846116A894644
:1001F000516A8A46916A8B46D16A8D4691688E46CD
:1002000001207047B409002070B506000D000028D9
:1002100014DD002907DD15481AF05CF80124864238
:1002200009DC002407E00100C02000061AF052F8A3
:1002300001248542F5DAE4B2200070BD002907DD13
:10024000C02000061AF046F801248642F3DBE8E7F6
:100250000024A042F0D0010004481AF03BF801232A
:10026000854200DB231CDCB2E6E7C046FFFFFF3F10
:100270008022044B52001A600123034A1360034A90
:100280001360704700E100E00C8C004000800040EB
:100290008022054B5200DA67044BFF3A5A60002275
:1002A000034B1A607047C04604E100E00080004044
:1002B0000C8C004070B501251D4B1E4C18601E4B68
:1002C000E550C046FFF7E4FF1C4A1D4BE560E250D5
:1002D000002303211B4AFF20A3500432A1504919D7
:1002E0000832A1508021C12209039200A150053A91
:1002F000FF3AA350C224144BA4001959C13A8143B8
:10030000FF3A0A4380211A510C341A590906120285
:10031000120A0A431A51C0220434195981430A436C
:100320001A51802212041A60802252041A6070BD91
:10033000C402002000800040FC0F00007017000085
:100340004C0500000405000000E100E070B51F4C02
:100350001F4D636C002B0AD0002363641D4B1B6888
:100360009847A823DB00EA5800018018E850A36CE6
:10037000002B09D00023A364164B5B689847164BEB
:100380000001EA588018E850E36C002B0AD00023E3
:10039000E364104B9B689847A923DB00EA580001EF
:1003A0008018E850236D002B0ED000230B4A2365E4
:1003B000AB580B495B18AB500A4A136806331360FD
:1003C0008022094B12045A6070BDC046FC80004078
:1003D0000080004004000020440500004C0500009F
:1003E00070170000C0080020FCE100E0F7B50191A3
:1003F000032823D8134B8000C758C223124D9B00FB
:10040000EF50012344192364A8230F210F4EDB0072
:100410009C46E358AE59921BD218D3170B409A183A
:1004200001990B4B1211C150C1239B00EF50634641
:100430000020013212019619E650FEBD0120404213
:10044000FBE7C04650C00200008000404C050000A1
:100450000400002003280BD8074B8000C158C2239A
:10046000064A9B00D150064A064BC25000207047F6
:1004700001204042FBE7C04650C00200008000401F
:10048000172E02000400002010B5024B1B6898478D
:1004900010BDC046C402002010B50024054AA35870
:1004A000002B02D00021A15098470434102CF5D124
:1004B00010BDC046B4020020074A89008B58002BAB
:1004C00006D1885080211800044A490451607047C1
:1004D00001204042FBE7C046B4020020FCE100E0FE
:1004E000F8B5224E3568686801281DD9AA68431EF0
:1004F000D15C0A2918D1002B03DD591E545C0A2C4B
:1005000013D11C00844202D2115D20290FD0002B90
:100510000FDC1218023AE31A14789B083A3C614245
:1005200061415C18002C11D1F8BD0B00E3E70134E8
:10053000E8E7611C8842ECD1591E0029E9D0013955
:10054000575C0A2FF0D0202FF7D0E2E7084F0422A3
:100550003900280027F045FC0421380012F090F8FB
:100560003369013C04333361DCE7C046C802002034
:10057000769B030010B52022002102482AF0CCFF10
:1005800010BDC046F4090020084B10B54268186041
:100590000020986018750138D86008005A601A6108
:1005A000996127F0ACFAFFF79BFF10BDC80200204D
:1005B000F8B503780400002B1DD00F4EB06C002856
:1005C00004D021002BF004F9002814D020002BF0D7
:1005D00009F9471C380028F0A1FC051E0BD03A0091
:1005E00021002AF07EFF054B054A1968043B9960FB
:1005F0009A42FAD1B564F8BDAC0900200C0A00207B
:10060000F0090020F0B5B64C06002068A5684368E4
:1006100085B00193002D00D010E1731E042B0AD881
:1006200027F048FC6368984200D1A3E0012E00D176
:1006300040E1022E10D0032E00D19BE0042E13D1F6
:10064000206821694368994200D32AE1012227F0FA
:10065000C9FC0025012726E123696268934200D97D
:100660004EE10126764285E0052E00D10EE1062EF0
:100670000FD123685D682369AB42AD416D42002D07
:10068000EFDD2368290098682369C01811F0F8FF8E
:1006900020E00B2E22D1019B22692068991A27F0B5
:1006A00095FC2368019A5B689A4204D91300226979
:1006B000981A12F01DF82268236951689068C91AC7
:1006C000C01811F0DDFF236858682369C01A401B69
:1006D00011F0FCFF23695D192561C2E70E2E13D1CD
:1006E000E368002BBDDB2068013BE3606268436880
:1006F000991A27F06BFCE368002B17DB1233794A59
:100700009B00995820680FE0102E16D1E368062B45
:10071000A7DC5A1C734913339B0059580029A0D0F9
:1007200020686368E260436027F010FC6368226918
:10073000D61A22685568ED1A0BE0152E0DD12369E3
:10074000626861689A1A206827F04CFC2369626825
:100750009E1A0127002E30DCA3E70D2E0DD1624832
:1007600027F0CDF9206827F0D7FB63680026C01872
:10077000FFF71EFF300005B0F0BD01231B2E66D031
:10078000082E01D07F2E21D121696268914200D8C4
:1007900067E7002320688668B618F75C202F13D11E
:1007A00001339F188F42F8D30126032B00DD033657
:1007B000891B320027F016FC0127300011F086FF5C
:1007C00023699E1B26617FE00126F1E7092E29D1CE
:1007D00063682269D11A22689068444AC01803AB42
:1007E00003F08AF9061E00D13BE70027431C0BD11A
:1007F000A06927F084F963682269D11A2268906899
:10080000C01811F03DFF4CE723692068F918039BDD
:1008100001375A1C03921A7827F0C6FBBE42F3D167
:1008200035003EE73300203B5E2B00D919E732004C
:100830002169206827F0C1FB012532E7012D08D18D
:1008400004234F2E03D002235B2E00D00023A3608D
:1008500007E7022D21D13300303B092B03D80323B6
:100860002675A360FDE60023A360412E00D14DE76D
:10087000422E00D134E7432E00D1FAE6442E00D1B7
:10088000EAE6482E16D0462E00D0EAE60027236876
:100890003E005D682369ED1A11E0032D28D17E2EFC
:1008A00003D000252F002E0009E0237D312B01D03D
:1008B000372B0DD100252F00236962689E1A002373
:1008C000A3609E4200DD78E7002F00D1D7E6E8E67E
:1008D0001A00FB21343A0A42D8D0332BE1D1AFE6DB
:1008E000C8020020AC09002006B00300B4EA0200F0
:1008F0000023042DABD1462EC8D0482EDAD0A6E76F
:10090000002501262F0058E7A3230021024A5B009F
:100910000248D1527047C046AC0900204CCA0200C0
:10092000A3230121024A5B000248D1527047C0460E
:10093000AC0900204CCA0200A323044A5B00D35A2E
:100940000348002B00D103487047C046AC09002083
:10095000AC090300A409030010B503F0D5FA01485F
:1009600010BDC0464CCA020003000F2010B508405D
:1009700003280ED819F006FC0204090D180010BD5A
:100980000648002BFBD10648F9E7180026F0CAFA02
:10099000F5E7180026F0E1FAF1E7C046AC090300DC
:1009A000A4090300F0B50D00002785B011000390E5
:1009B0001E0028000F4B0222009702F059FFA81CCE
:1009C000800028F09EFA039B040003606B1E3D002C
:1009D0000393436033688360039B9D4202D32000EE
:1009E00005B0F0BD0135AF00F0590EF047FAE71938
:1009F000B860F1E7FFFF0000054B002805D0002399
:100A0000022802D1012349000B4318007047C04659
:100A1000A409030010B5024924F002FD10BDC04630
:100A2000B17B0300F0B50700443787B004003800FD
:100A30000E00002527F02CFA2069431C1CD00A2840
:100A400004D1200022F057FA0125F5E713F096FDB6
:100A5000002803D0200022F04EFAEDE72369232B73
:100A600008D1200022F047FA23695A1CE4D00A2B4F
:100A7000F7D1E1E75C2B0ED0E369226AA363E2635E
:100A8000002E17D1636A002B1DDA220007214032A5
:100A9000117001331EE0200022F02DFA23690A2B89
:100AA000D8D0E369A363236AE3630423403423704B
:100AB00007B0F0BD012BE5D1012AE3D006222300C7
:100AC00040331A7007E0002B1FD02200062140326D
:100AD0001170013B6362200040300378082BE7D19E
:100AE0000023E56CB24EA46C9A00915900228F1835
:100AF000944200D170E28F5CBC46AF5CBC4500D133
:100B000068E20133222BEFD1D2E7002D34D0A36A63
:100B1000002B31D12100052040310870551E636241
:100B2000226BA44B606BD3185B001B5A9D42BFD055
:100B300017D9E16A8A4207D30831490028F0F7F94A
:100B4000E36A60630833E362236B5A1C2263626BBF
:100B50005B009D52636A9CE7013B2363636A013B30
:100B60006362236B934A9A185200125A9542F3D348
:100B70009ED002230B70AEE72069431C1AD18D4A28
:100B8000236B616B9B185B005A5A23004033002A89
:100B900097D005221A7000236362864A236B9A1845
:100BA0005200525A002A00D182E7013B2363636A54
:100BB000013BF1E727281FD022281DD0752804D03B
:100BC000102302009A43622A04D16369272B0ED0B6
:100BD000222B0CD0722800D015E26369622B00D062
:100BE00017E2A369272B02D0222B00D011E275282F
:100BF00004D1200022F07FF900234DE0622842D189
:100C0000200022F078F9002302932369722B04D18B
:100C1000200022F070F90123029323000C224033BC
:100C20001A700123059323690393222B01D02723F4
:100C30000393200022F05FF90123039A04932369B0
:100C400093420BD113006269934207D1200022F036
:100C500052F9200022F04FF9032304930026236960
:100C60000193013300D1C9E0049B012B03D1019B07
:100C70000A2B00D1C2E0049BB34214D831003800E3
:100C800027F0A4F927E77228B6D1200022F033F923
:100C90002369622BBCD00123029323000B22403333
:100CA0001A700023BEE7019B039A934208D11100FA
:100CB0003800013612F0A6F9200022F01CF9CEE728
:100CC000019B5C2B00D096E0200022F014F9029BDF
:100CD0002569002B04D05C21380012F093F95AE00A
:100CE000622D00D1BEE130D84E2D78D01BD8222DF8
:100CF00053D0272D51D000260A2DDDD028003038C2
:100D00000728E8D8050003266369303B072B42D843
:100D1000013E002E3FD0200022F0EDF82369ED00C7
:100D2000303B5D19F0E75C2D37D0612D5AD0552D41
:100D3000E4D1059B002B27D05C21380012F062F92A
:100D4000E9B2380027F0F9F813E0742D13D008D871
:100D50006E2D00D188E1722D14D0662DCED10C25D8
:100D60000AE0762D0CD0E4D30226782D10D06B1C2F
:100D7000C4D10026A0E70925059B002BE0D112E095
:100D80000B25F9E70D25F7E70826752D00D1043E60
:100D90000025013E12D26B1CEBD0074B9D4225D89B
:100DA000059B002B20D12900380012F02BF9E0E739
:100DB0008CCA0200FFFFFF7FFFFF1000200022F01F
:100DC0009AF823691800019313F0FCFB002800D166
:100DD00013E1019827F04DFA2D012D18D9E7A54808
:100DE0000EF0F8FD0725DBE7FF2DA9D9230001222E
:100DF00040331A70BDE76B461979A2E7049BB342F2
:100E000000D83BE72300032240331A7036E713F083
:100E1000CDFB002807D02600216940362E291CD1A1
:100E20000A23337029E023692E2B04D1606913F063
:100E3000BDFB0028EFD121692E2954D000260222C3
:100E40008D4D2F78002F01D0B9426CD1200022F0B7
:100E500052F8002F76D1012231E609233370302970
:100E60000BD1626917331343623B162B03D8834DB2
:100E7000DD4001231D4001231D40380012F0C2F85F
:100E8000200022F038F814E0002D16D1652801D09A
:100E9000452812D10A2365213370380012F0B2F8C8
:100EA000200022F028F8216902220B002B3B9343FB
:100EB000E3D02069431CE7D10DE613F06BFB00285B
:100EC00008D021692E29ABD00B00202293434A2B56
:100ED000D3D1A5E7206913F069FB0028F1D123697C
:100EE0002E2BEED0F7E52600380012F08BF820000C
:100EF00022F001F8236940362E2B00D0B6E0656958
:100F00002E2D00D0B2E02900380012F07BF8290025
:100F1000380012F077F8200021F0EDFF200021F0DA
:100F2000EAFF0D23A3E03B00633B9343DBB2681C65
:100F3000002B03D105000136013582E7452FFAD198
:100F4000013EF7E7330001352A78652A09D16A782E
:100F500021690136914212D1200021F0CCFF3300EB
:100F600001352A78452A20D16B7822699A420AD124
:100F7000200021F0C0FF3300414AD25C04E01F0092
:100F800002353B00E0E70122230040331A702300C2
:100F900040331B78042219009143422901D0442B8D
:100FA00010D1A36A0133A36295E5632AE4D16A787C
:100FB0002169771C9142DFD1200021F09CFF02358E
:100FC0003E00DEE7432902D0452B00D083E5A36A2B
:100FD000013BE8E701328AE53A78002A00D090E543
:100FE000212B08D1274BA8331A680E23002A00D1E1
:100FF000023303705CE50E33FBE72300012240332C
:101000001A700500B8E6622803D16369722B00D11B
:10101000E7E513F0BFFA051E206904D15F2802D06E
:101020007F2800D8F3E62300082240331A70C1B2AB
:10103000380026F082FF200021F05DFF2069431C6C
:1010400000D148E513F0A6FA002809D120695F28ED
:1010500006D07F2804D813F0A9FA002800D13AE579
:10106000217CE5E7082587E60A2585E64A233370D3
:1010700031E5C04632300300F02F0300012040006C
:10108000B1300300AC090020F0B50E00002485B09B
:1010900011000700039322000C4B3000009402F073
:1010A000E7FBB01C800027F02CFF050007604660BE
:1010B000B44202D1280005B0F0BD039BA700D85967
:1010C0000DF0DCFEEF19B8600134F1E7FFFF00001E
:1010D00010B54379012B03D1C06A27F009F810BD80
:1010E0000B00C26A0249006B27F03EF8F7E7C046E2
:1010F000881F030010B54379012B03D1C06A27F084
:1011000017F810BD0B00C26A0249006B27F02CF8DB
:10111000F7E7C046981F030010B54379012B03D1B0
:10112000C06A27F005F810BD0B00C26A0249006BC7
:1011300027F01AF8F7E7C046781F030010B5024BF6
:101140003F2222F026F810BD833B020010B5024B6F
:10115000912222F01EF810BDB1220000F7B50F0059
:1011600011001A00C38AC579868A019300230400FE
:10117000C3718382C382104B22F00BF8A368002B4B
:1011800018D1E18A002908D0A38A002B05D1206B51
:1011900027F062FD206B27F0F2FBA38AE28A390078
:1011A000200021F0A6FF6B1E9D416B469B88E571D8
:1011B000A682E382F7BDC046C11E0000836870B5F9
:1011C00004000D00002B09D11100054823F020FB7D
:1011D000A060200029000C3022F042F870BDC0460B
:1011E00048DC0200F0B58DB06B4601921B7904001B
:1011F00043710123E16203610B780D00012B06D0DE
:101200000021954A2000FFF7D9FF0DB0F0BD019BEA
:10121000012B07D9836B0A001E680300019908336C
:10122000406BB047AB681800049323F018FD637956
:101230000490032B0FD109900C2109A823F028FD5D
:10124000A36B02009B680999606B9847A368688349
:10125000002B00D0BCE0049823F001FD049003783B
:10126000002B3AD00A3B0F2B32D809A921F015FFE9
:10127000099B772B2AD006D803220292312B08D063
:10128000764A0499BEE7812B1DD002220292992B47
:10129000F6D1049823F0E3FC5A21049004A823F02B
:1012A000F7FC049D0390039B9D4218D16379012BA9
:1012B00004D9A36B02995B68606B9847A368002B05
:1012C00000D085E0A1E701230293E2E70023FBE7DA
:1012D0000100634A2000FFF771FF0223F4E7049541
:1012E0002B78432B04D1280023F0B9FC0500DAE762
:1012F000392B01D05B4AC4E705A9280023F0B9FCCB
:1013000003780600912BF5D123F0A9FC059B9842A8
:10131000F0D105A9300023F0ACFC037807000A3BAC
:101320000F2BE7D823F09BFC059B06009842E1D0E9
:101330000378A02BDED123F092FC059B9842D9D1F3
:1013400006A9380021F0A9FE300023F08DFC9C2175
:10135000079007A823F09CFC0100079823F073FC7A
:10136000069B06002E2B1BD1012804D10798037879
:101370000A3B0F2B01D93C4A83E72669731C236182
:10138000019B012B21D909A921F087FEA36B099AA2
:10139000DB683100606B9847002816D1334A70E74C
:1013A0002F2B1BD1012803D107980378032B01D0E1
:1013B0002F4A66E7019B012B07D9A36B676B1E6958
:1013C00023F02DFC01003800B047A368002B8AD021
:1013D000200004990C3021F043FF16E7302B23D175
:1013E000012803D907980378032B01D0214A48E745
:1013F000019B012BE9D908A923F002FC01270790E2
:1014000007980378032B01D01B4A3AE709A923F078
:10141000F7FBA36B07905B69099A0899606B01372A
:101420009847BE42ECD1D0E7019B012BCDD90328D0
:1014300000D95FE7079B1800099323F010FC0A907E
:1014400023F00DFCA36B0B909F69320009AB06994A
:10145000606BB847B9E7C04610330300343303006C
:1014600041330300693303008C330300A8330300C6
:10147000B8330300D4330300F933030010B5024A34
:10148000FFF79CFE10BDC0461B3403007FB50B78F0
:1014900004000D004E1C002B0AD0032B0BD103A916
:1014A000280023F0ADFB03990600206B27F0FEF91E
:1014B000300004B070BD012B07D18E1C497805297E
:1014C000F6D0006B14F07EFDF2E7042B0BD14B78C5
:1014D0008978006B0902194327F030FA280023F0BD
:1014E000BEFB0600E4E7052B15D14379042B04D09D
:1014F0002A49006B27F02EFAF0E788784B78000233
:10150000184303A925F0ADF90399246B06F0FEFA00
:1015100001002000EEE71A000A3A0F2A09D803A9B1
:10152000280021F0BAFD039906002000FFF7D0FD46
:10153000BEE7082B0CD103A9280023F057FB039B1F
:10154000226A9B0006009958206B27F003FAAFE748
:1015500003AB02AA01A9280023F0B2FB02990500FF
:10156000206B14F0E5FC019B0D4A9B009B58002B5F
:1015700006D10C4A29002000FFF720FE039E97E7C2
:10158000039A290020009847A368002BF6D0E3684F
:10159000002BF3D1029BE360F0E7C0464CCA020087
:1015A00050CB020052320300F0B587B000920A001F
:1015B0000493531E9A410D00060004990098059269
:1015C00023F041FB2C1E019009D02B780024842BA2
:1015D00005D102002100306B27F0BCFB2C00019BE1
:1015E000009F013B0393059B0293049B9F421ED1E6
:1015F000002C39D1019A059B944663441900306B45
:1016000027F09CFB002D3CD1009B9F422AD0009BE1
:101610009C4239D1200023F027FB0022010030003A
:1016200000F038F8009823F01AFB0090ECE73B78C4
:10163000842B07D1002C10D1039A0299306B27F02C
:1016400089FB3C00380023F00AFB029B07000133B2
:101650000293039B013B0393C7E70D4A3900300017
:10166000FFF7ACFD07B0F0BD002DCDD0AC4208D1E6
:10167000200023F0F9FA00220100300000F00AF8FF
:10168000C2E700222900F8E700220099C7E7C04618
:1016900046310300F0B50B7817001A000A3A85B0FE
:1016A00004000D000F2A10D803A9280021F0F5FC32
:1016B00003992000002F01D0022F03D1FFF71AFD5C
:1016C00005B0F0BDFFF704FDFAE76A4A192B00D810
:1016D000CBE01A3B7C2B00D182E005DC252B08D027
:1016E000772B11D0644AC0E07E2B00D194E0912B7F
:1016F000F8D1002F00D0B7E003A9280023F0B9FAF1
:101700000200039B00219BE002A9280023F0B1FA0C
:101710000600022F03D001002000FFF7B7FE3000C3
:1017200023F09DFA0299060021F0AEFC0028D9D1E1
:101730003378922B13D1300003A923F09AFA0600D4
:10174000300023F08CFA039A0190904207D2022FC6
:1017500003D031002000FFF799FE019EF0E73378B7
:10176000A12B21D1022F06D1206B27F08DF9206B00
:1017700027F049F90EE0300023F076FA010020004E
:10178000FFF784FE206B012FF2D127F051F9206B77
:1017900027F021F9300023F062FA029921F074FC5D
:1017A000002800D08CE79DE7A22B9BD1300023F0CE
:1017B0005BFA03A921F071FC012F07D1206B27F000
:1017C0002DF90399206B27F0E4F8E3E7022F02D10B
:1017D000206B27F042F90399206B27F007F9D9E72E
:1017E00003A9280023F045FA0399060021F04CFCD8
:1017F000002800D076E7002F36D1350003A9280055
:1018000023F037FA060023F02AFA03789D2B1BD128
:1018100000231A00310013E0002F25D103A928006E
:1018200023F027FA0399050021F02EFC021E02D0B6
:101830003B003A0066E72B789A2BDFD003002900A3
:101840002000FFF7B1FE3BE79E2B05D103A923F053
:1018500010FA039B0200DDE7BE2B00D142E723F024
:10186000FEF9320003004DE7044A29002000FFF78B
:10187000A5FC25E7E7300300FF3003001A31030021
:10188000F0B50B788FB00A3B0400019103920F2B47
:1018900000D9E6E0080023F0E2F90378912B00D0AC
:1018A000DFE0019823F0DBF90BA923F0E2F90378DC
:1018B00042780A3B1B021343AD2B00D0D1E023F04A
:1018C000CEF903780500A02B00D0CAE023F00CFA73
:1018D000002800D0C5E0280023F0C1F90B9B9842F6
:1018E00000D0BEE0280023F0BFF99C210C900CA88A
:1018F00023F0CEF901230C9E070030000D9323F056
:10190000AEF905000C90874200D1A0E023F0A7F9C2
:101910000C9087420AD00378032B00D0A1E00DA9D8
:1019200023F06EF90C90874200D09AE03378483368
:10193000DBB2022B00D894E02B784833DBB2022BC9
:1019400000D88EE00B9B1800049323F088F9039ACB
:101950000290904201D1002302930D9B27690593C9
:10196000238B27830693638B0793E38B08937B1C5E
:101970000393BB1C09936B469B896383A38BE3830F
:101980003B1D23612B780393032B03D029002000F8
:10199000FFF77CFD31002000FFF778FDF91C206B7C
:1019A00027F087F8B91C206B26F04CFF206B27F03E
:1019B00035F8002201992000FFF76CFE0499200001
:1019C000FFF764FD791C206B26F03CFF0599206B26
:1019D00026F06CFF1221206B27F01CF9206BF91CFC
:1019E00026F030FF039B206B032B33D027F020F829
:1019F000206B27F032F8059B1921002B00DA1A2101
:101A0000206B27F007F9BA1C0121206B27F05DF845
:101A10006B461B8B23836B469B8B63836B461B8CB4
:101A2000E383029B002B03D019002000FFF72EFD5B
:101A30003900206B26F006FF206B27F003F8039B8C
:101A4000032B02D0206B26F0FDFF0FB0F0BD350058
:101A50002E4E6BE726F0E2FF29002000FFF716FD6F
:101A6000C9E7238B25690293638B6F1C0493E38B77
:101A700067830593AB1C0693A38B0198E383244BE8
:101A80002B432383EB1C236123F0E9F801002000A2
:101A9000FFF7FCFC0600206B27F068F83900206B8C
:101AA00026F0D0FEA91C206B27F06AF800220199CD
:101AB0002000FFF7EFFD31002000FFF7E7FC0600F4
:101AC000206B26F0B6FE002803D13900206B26F0EB
:101AD000F0FFA91C206B26F0B5FE206B27F05CF808
:101AE0006B461B8923836B461B8A63836B469B8AE9
:101AF000E383039BB34203D031002000FFF7C6FC11
:101B00002900206B26F09EFE9FE7C046A53A030001
:101B10000080FFFFF0B5170085B0040008000D003D
:101B200023F09DF83900060021F0AEFA019000285C
:101B30001ED02379002B16D0E36A1E78002E12D116
:101B400013212000FFF7C4FA29002000FFF79EFCB4
:101B5000330032000121206B27F03BF9206B26F087
:101B600071FF05B0F0BD29002000FFF78FFCF5E7FD
:101B700033783B2B1DD1290001222000FFF78AFD7D
:101B8000300023F071F84378811C4E3BDBB21826FD
:101B90000A2B01D8224AD65C2000FFF777FC3100DF
:101BA000206B27F037F8022229002000FFF772FD92
:101BB000D7E73C2B2ED1300003A923F05AF80600BA
:101BC0000700039B9F421FD101992000FFF75EFC95
:101BD000206B26F023FF002229002000FFF75AFD8A
:101BE000019BB342BDD0300023F039F8019B0500C2
:101BF000834202D0206B26F011FF3100002220002A
:101C0000FFF748FD2E00EBE7380023F028F8019796
:101C10000700D6E731002000FFF738FC019AC3E740
:101C2000DC300300F0B589B0040005910492009304
:101C3000029100292AD1A379002B2CD0E36A1D78C8
:101C4000012D28D105212000FFF742FAE16A029B0D
:101C5000088D834206DB0021554A2000FFF7AEFACB
:101C600009B0F0BDCE6ADA00B21856782E420BD019
:101C700052880121206B26F05AFD002302211A0010
:101C8000206B27F0A6F8EBE70133E2E79C2105A8DB
:101C900022F0FEFF029000273E00059D039701976A
:101CA000029BAB4216D1002E0AD0039B002B70D1B1
:101CB000206B26F064FE002F70D1206B26F05FFEB3
:101CC000049B002B6FD03300019A0099206B27F002
:101CD00089F8C5E72B78B82B10D1B73B1E4202D04C
:101CE000344A2900B9E7012328001E4322F0BCFF33
:101CF0000390280022F0B3FF0500D1E7B92B0BD1E8
:101D0000B73B1E4201D02C4AEBE7022328001E43BA
:101D100022F0AAFF0700ECE7BA2B2CD1280022F012
:101D2000A3FF050022F09BFF0378BE2B0BD1200000
:101D30000622290021F0D1FA009B280001330093EC
:101D400022F08DFFD6E72B780A3B0F2B01D91B4AD7
:101D5000C7E707A9280021F0A0F905000799206B23
:101D600026F0ECFD29002000FFF790FB019B050009
:101D70000133019394E7019B002B01D0104AB0E797
:101D800029002000FFF782FB009B05000133009330
:101D900086E703992000FFF779FB8CE739002000E4
:101DA000FFF774FB8CE73300019A009968E7C0469F
:101DB00038340300563403006D34030085340300C7
:101DC000A6340300F0B589B00400039103A80721ED
:101DD00022F05EFF0027E36A02905E7E0398029B7A
:101DE000834215D1180022F03FFF029B03901B781D
:101DF000010032002000242B4CD121F005FA05000F
:101E0000013F4AD229002000FFF774F909B0F0BD64
:101E100005A922F02EFF4021039003A822F038FFED
:101E200006A90500039821F038F9069B01902A2B9A
:101E30003CD1854207D8214A00212000FFF7BEF996
:101E4000059B0393CAE7019822F009FF8542F2D16E
:101E500007A9019821F021F9079B2B2B24D02D2BCA
:101E6000E9D10426ECE707A921F017F907990390B7
:101E7000206B26F08EFD03988542F4D10599280049
:101E800021F002F90028DBD1A07129002000FFF722
:101E9000FDFAD5E721F02FFCB1E7002301211A005C
:101EA000206B26F096FFABE70126C9E703992000D7
:101EB000FFF7ECFA01370390DDE7C046E731030096
:101EC000F7B50A780E0013000821293B8B43DBB2DB
:101ED0000400002B02D10133C371F7BD13002A3B6C
:101EE0008B43DBB2002BF8D013000A3B0F2B2FD90A
:101EF000282A11D101A9300022F0BBFE070022F0F0
:101F0000AEFE019B984205D022F0A9FE019B050080
:101F1000984208D1002506E0300022F0A5FE070017
:101F200022F09DFE050001A9380021F0B6F8E37902
:101F3000002D02D02A78002A0CD1002BCDD1E38AC3
:101F4000002BCAD0184A31002000FFF737F9C4E748
:101F50003700DFE7002B1ED0A38A01339BB2A38298
:101F6000012B09D1E18A206B002911D026F074FEE3
:101F70000021206B26F097FE29002000FFF786FA4B
:101F8000206B019926F0DAFC206B26F098FEA4E77E
:101F900026F0F5FCECE7E38A29000133E382200018
:101FA000FFF774FA99E7C04605320300F0B5040064
:101FB0000E00056987B002936B1C0393AB1C036191
:101FC0002900006B170026F0AEFD200021F06DF80F
:101FD00031002000FFF75AFA206B26F0E3FD691C60
:101FE000206B26F066FD2900206B26F02BFC206B71
:101FF00026F03CFF2669731C2361029B9F4218D187
:10200000A38B206B013BA38326F0A5FD206B26F05C
:1020100031FF0399206B26F015FC0C9B002B03D09D
:1020200019002000FFF732FA3100206B26F00AFC7D
:102030001BE0380022F018FE0023059323690500F9
:102040000193013323610378002B10D122F007FEA6
:1020500022F005FE029B834224D03F4A2900200043
:10206000FFF7ACF8A38B013BA38307B0F0BD0700DB
:102070006A2B07D122F0F8FD070022F0F0FD05A938
:1020800021F00BF8206B26F0C9FC39002000FFF787
:10209000FDF92121206B26F0BDFD019A0021206B66
:1020A00026F013FD280022F0DAFD0700206B26F051
:1020B000C9FC059900294BD1206B26F0C3FC0025F3
:1020C000206B26F0BFFC059BAB4209D02569206B35
:1020D0006B1C2361290026F032FD200020F0E5FF73
:1020E00039002000FFF7D2F9059B0700002B02D032
:1020F000206B26F057FD206B26F075FD059B002B0D
:1021000019D00F21206B13F05DFF2900206B26F002
:1021100099FB0F21206B13F055FF05992000FEF766
:10212000E9FF20000599FEF7F7FFA38B206B013B29
:10213000A38326F010FD3100206B26F0BAFC019934
:10214000206B26F07FFB0321206B26F077FB54E702
:102150002000FEF7CFFFB2E7C8340300F0B587B028
:10216000039143790400012B06D1C36A1B78002B2D
:1021700004D11E4AFFF722F807B0F0BD039B4321AC
:1021800003A8019322F084FD02900398029B8342EE
:10219000F2D005A90B2720F080FF02AB059DFF18A8
:1021A00003903A002900E06A24F0C4FC3B78060062
:1021B000002B03D103780E4A042B0AD12900E06AD0
:1021C00024F0E5FC002803D00378023B022B05D95C
:1021D000084A01992000FEF7F1FFD6E70423337087
:1021E0002900E06A24F0E6FCCFE7C0466A3203002B
:1021F0008F320300B0320300F0B587B00391447909
:102200000500012C09D1019103A8432122F040FDD2
:1022100002900398029B834201D107B0F0BD05A94B
:102220000B2720F03AFF02AB059EFF1803903A00FF
:102230003100E86A24F07EFC3B78002B08D103785B
:10224000012B05D0074A01992800FEF7B7FFE0E708
:1022500004703100E86A24F091FC0028D9D00470A1
:10226000D7E7C0463332030010B5438B0400002B80
:1022700002D1054AFEF7A2FFA28BE38B618BD21A33
:10228000206B13F0C5FE10BDCF31030010B5038BDA
:102290000400002B02D1054AFEF790FFA28BE38BCE
:1022A000218BD21A206B13F0B3FE10BDBA3103009C
:1022B000F7B50B7804001A000A3A0E000F2A08D866
:1022C00001A9300020F0E9FE01992000FEF724FF6B
:1022D000F7BD912B44D16946300022F0CAFC0100C1
:1022E0002000FFF7D3F803780500922B10D101A945
:1022F00022F0BFFC0500280022F0B1FC019B070082
:10230000984205D029002000FFF7C0F83D00F2E711
:102310002B78A12B16D1280022F0A6FC010020006A
:10232000FFF7B4F80500206B26F0B8FB00992800F1
:1023300020F0AAFE0028CBD1214A31002000FEF770
:102340003DFFC5E7A22BF7D1280022F08DFC01A9A3
:1023500020F0A3FE01990500206B26F088FBE5E73D
:10236000962BE9D1080022F0BFFC0028E4D1300010
:1023700022F07AFC060022F077FC05000100200024
:10238000FFF796FF280022F06AFC03789D2B9FD070
:102390009E2B0ED101A922F06CFC019B05009842F6
:1023A00096D020002900FFF783FF280022F057FC79
:1023B000F3E7BE2BC0D001002000FFF779FF87E7CD
:1023C00060310300F7B502260D00C16A0400097EE2
:1023D000314005D0344A29002000FEF7EFFEF7BD5A
:1023E0000191297808000A380F281DD8280001A972
:1023F00020F053FEE279E36A002A03D09A8B01327F
:102400009A8302E05A8B01325A83012601990029EE
:10241000E5D06B46DF1C3A00E06A24F08BFB3B788A
:10242000002B3CD1214AD6E71A32914204D1280030
:1024300022F01AFC01A9DBE71A33994223D1E37990
:10244000002BC7D101272800E77122F04DFC03269D
:102450000028DBD1280022F007FC0278E36A0A3A60
:102460000F2A09D828001A7E17431F7622F0FCFB9A
:1024700001A920F012FEC9E71A7E280017431F7633
:1024800022F0F2FBF2E7280022F0EEFB01A920F097
:1024900004FEE36A1A7E16431E760526B6E702237B
:1024A000467003709BE7C046E8320300F732030032
:1024B000C36A70B51B7804000D00012B04D00C4AD0
:1024C0000021FEF77BFE70BD1100280020F0DCFD2E
:1024D000002807D00F21206B13F074FD206B26F02D
:1024E0008BFCF0E729002000FEF7D0FFF6E7C0469E
:1024F000CE320300C36A70B51B780400013B0D00A7
:10250000012B04D9164A0021FEF758FE70BD1100B8
:10251000280020F0B9FD002807D00F21206B13F010
:1025200051FD206B26F083FCF0E72B78C22B11D1F4
:10253000280022F099FB01002000FEF7A7FF206B86
:1025400026F014FB206B0F2113F03CFD206B26F0CE
:102550007DFCDBE729002000FEF798FFE1E7C0469D
:10256000E7340300F0B50D0085B004001100280029
:1025700020F08AFD071E05D00021206B26F093FB7A
:1025800005B0F0BD2B78AF2B0BD1206B012126F0CD
:102590008AFB29002000FEF779FF206B26F08FFBD5
:1025A000EEE7AE2B61D1280022F05EFB050022F0A1
:1025B00056FB02900378B22B4DD103A922F059FBB0
:1025C000039B0290984203D0992102A822F060FB5D
:1025D0002B78AF2B20D103990298266B22F033FB86
:1025E000411C300026F05FFB29002000FEF74EFF63
:1025F000206B26F064FB0127029E039B9E4210D1B4
:10260000002FBDD131000298246B22F01CFB411C2D
:10261000200026F06CFBB3E729002000FEF736FF10
:10262000EAE73378310020000193FEF72FFF019B8A
:102630000600002F0BD0AF2B05D00F4A2900200039
:10264000FEF7BCFD9CE7206B26F039FBD5E7AF2BEE
:10265000D3D10A4AF2E72B780422AF2B00D005220F
:102660002900200020F039FE8AE729002000FEF72B
:102670000DFF0121206BCCE7783103009B31030073
:10268000F0B504000D00012362711100C562036101
:102690002A0087B0006B13F07FFB6279012A02D118
:1026A00000236B84AB84AE6833781E2B0AD13000D4
:1026B00022F0DAFA01002000FEF7E8FE206B26F097
:1026C0009BFB2AE02B78002B08D131002000FEF77D
:1026D000DDFE0F21206B13F075FCEFE7012B21D1FC
:1026E000300022F0BCFA63790500012B07D10023EA
:1026F0000100E3710C22524B200020F04AFD28001B
:1027000022F0ADFA22F0ABFA01002000FEF7BEFE87
:10271000206B26F08EF80028DBD0206B13F0CEFB68
:1027200007B0F0BD022B17D1012A07D100231332C5
:10273000E3713100434B200020F02BFD300022F0EC
:102740008EFA01002000FEF7A1FE2B7E5B07B5D5B7
:10275000206B26F077F9BCE7033B032B3BD8300016
:1027600022F07DFA05A922F084FA22F078FA67793E
:102770000390012F09D10B2202ABD2183900E06A75
:1027800024F0D8F9022303706F832B78032B14D124
:102790000021206B26F06DFA01212000FEF798FC45
:1027A0000023059A009303993300200021F099FA41
:1027B0002B78062B00D081E78BE7042B04D1002176
:1027C000206B26F070FAE7E7052BE5D10021206B9E
:1027D00026F08DFAE0E7012A06D105AA0521280096
:1027E00024F0A8F90223037005A9A86820F055FC7D
:1027F0000D212000FEF76CFC0C212000FEF77AFC76
:102800002969206B26F09AF811212000FEF772FC4E
:10281000A86822F024FA22F022FA01002000FEF734
:1028200035FE0521280024F075F90378022B00D12C
:102830004FE742880521206B25F079FF3EE7C0462F
:102840001139020005390200F0B51E000F009BB0DF
:102850000BAC00210690150020003C2228F05CFE05
:10286000069B0B975B6826712362069B186822F013
:10287000F6F922F0D4F96062800026F054FB0022C1
:10288000069BA06200951B681100200020F017FC39
:1028900025F0B9FF00230290206303930026330044
:1028A0001FE0FFF7EDFE15E0A268002A1DD1A16A26
:1028B000B2005558002D13D06A69002A10D125F0B6
:1028C000E1F86B7E6861012229002000042BE8D129
:1028D000FEF788FC2369039A9A4200D203930123EE
:1028E0000136626A07929642DED3002BD6D104935A
:1028F00001339C46079B049A934202D00D9A002A0A
:102900002DD000260399029825F082FF3500149BF4
:1029100004939E4200D2ECE00D9B0393002B00D069
:1029200011E1029825F07CFF002D02D0280025F04F
:1029300011FE0024069822F0E1F9159B1B685D69E1
:10294000149B02939C4200D20AE1159826F000FBEA
:102950000D99002900D10EE10800FDF738FC04991B
:10296000159B8900CB58002B38D06046197E014258
:102970001CD01C8D601EC000002C17D00226D96A06
:1029800009184D7835422DD0002A0FD00F005088FD
:102990001678059050685578089011CF11C26A4694
:1029A000928A0E704A80089A4D704A6000211A8DF2
:1029B00019840592059A91421CDB0021059A8A42EE
:1029C00036DC5E68002E09D00021328D09920A00A3
:1029D000099881423CDB0020002A65D1049B013329
:1029E000049387E7002A02D1012D00D10A00013C9F
:1029F0000838C1E7D86ACA0082181878072802D1B7
:102A00005468052C12D00138052804D81078002805
:102A100001D1604610701078022803D064465078C7
:102A2000204203D0188C441C1C8450800131C1E723
:102A3000D86ACA0082181078032807D164465078F3
:102A4000204203D1188C5080013018840131B5E741
:102A5000F06ACD004019089000780024033801285E
:102A600010D90131B4E7DF6AE00038180778042F85
:102A700007D1089D6F683D004768BD4201D1428083
:102A8000013201340598A042EDDCEAE7DC6AC100BE
:102A900061180C78042C03D165464C782C4202D086
:102AA0004C88A4184C80013005998142EEDC598B8A
:102AB00092B251185983198C52181A848EE7029BCE
:102AC000022221000BA81793FFF7DAFD0D9B049358
:102AD000002B04D1032221000BA8FFF7D1FD0D9B91
:102AE0000493002B2DD1042221000BA8FFF7C8FD71
:102AF00027E00D9B0493002B00D00DE7159B04935A
:102B0000049AB3009C58002C1BD0637E042BD6D1B2
:102B1000002D03D1039825F00CFD05000023179329
:102B2000184B032221000BA819931895FEF75AFBA6
:102B30000D9B0493002B04D1042221000BA8FEF767
:102B400051FB0136E3E6169B0EA8996820F088FB3E
:102B5000169B0E9A1B690B990D9802F0EFFDE0E6AB
:102B6000159B0293029AA3009858002801D023F0E5
:102B7000C8FF0134E4E60A00280024F08FFF1BB0F0
:102B8000F0BDC0468C1B030070B50E001049040058
:102B9000002522F045FC73689D420AD3012B03D126
:102BA0000C49200022F03CFC0B49200022F038FCAC
:102BB00070BD002D03D00949200022F031FCAB008C
:102BC000F3180122996820000BF052FA0135E2E770
:102BD0007D930300033503004A950300003503008D
:102BE00070B50D0001281ED0002803D0022807D0A0
:102BF000002004E04B680E48002B00D10D4870BD4A
:102C000000260D4C6B689E4203D3012064002043D4
:102C1000F5E7B300EB18996802200BF0CDFF4010E8
:102C200024180136EEE74B685B001843E7E7C0461F
:102C3000AC090300A4090300F8CD020010B504009C
:102C4000102026F05EF9044B84600360034B436060
:102C50000023C36010BDC04628010300B14102003B
:102C600070B506000D000C48002E0FD0B41CA40057
:102C7000200026F046F9094A030002604660002D54
:102C800004D00022083C944201D1180070BDA8581D
:102C9000991888600432F6E7F8CD020000CE0200F1
:102CA000F0B5040085B00D00160007284CD003D8FD
:102CB000052824D0002144E00300193B042BF9D857
:102CC00008000BF0BDF930000BF0BAF92C4B426A4A
:102CD0009A4205D030002B4921F098FB061E0CD0FB
:102CE0003300290072680831009208336A682000B6
:102CF00011F0ECFD2449002823D1244921E01000E3
:102D00000BF09EF91F4900F053FC011E19D06B68AF
:102D1000726800219818FFF7A3FF070029006B686D
:102D200008379A0008310400380028F0DAFB310037
:102D300068687368800038189A00083128F0D1FB61
:102D40002100080005B0F0BD03A910000BF09EFAA9
:102D500000218842F5D0039888420FDD6B68584304
:102D6000FFF77EFF0400230028000833009308309B
:102D7000039B6A68042125F083FAE1E70449E0E750
:102D80003D2C000000CE0200AC090300A4090300A2
:102D9000F8CD020030B5040085B0042A2DD10325FA
:102DA0000D4020D1164B0A689A421CD101AA4068F6
:102DB00011F052FD002802D112480CF00BFE019BCD
:102DC00002982900C01AFFF74BFF050021006B682D
:102DD00008319A00019B08309C00091928F081FBFA
:102DE000280005B030BD0A000023616820680BF0A0
:102DF000E7FA023080000059F3E70020F1E7C0460F
:102E0000EC00030005350300F0B50C0011000022B2
:102E100085B01E0000920123200000F029FD184D0E
:102E2000002C1DD03568AB0703D1164B2A689A4297
:102E300016D0102026F065F8040030680CF01EF85B
:102E400000250426039003980CF064F8071E0AD1AD
:102E500028002100FFF704FF0500200026F078F885
:102E6000280005B0F0BDAE4205D8F100200026F0E4
:102E70005EF804007600AB001F510135E3E7C04661
:102E8000F8CD020000CE0200F8B504000D00A368E2
:102E9000002B0AD0344AE968914206D0EB58002B47
:102EA00003D00422E3681A60F8BDA86B002822D082
:102EB00063680022D90006230430194308F044FE59
:102EC000021E18D0237C002B06D042680020E36845
:102ED00021680BF015FFE7E72368181E07D0224989
:102EE000EE688E4203D021498D4200D01869E36814
:102EF00052682900EDE72368002B12D16E6B002E7B
:102F0000D2D075680836002DCED000276B1E174A28
:102F10009F421AD3164BED18AD00AD599542B6D16C
:102F2000C2E7227C002AE9D10F4AE9689142E5D044
:102F30000E4A9542E2D01869E26861680BF022FF00
:102F4000E3681B68002BD9D0AEE7BB00F158914273
:102F500001D10137DAE72000FFF796FFE3681B682D
:102F6000002BF6D0A0E7C046213200000007030086
:102F7000FFFFFF3FF0B5146889B01700002C14D193
:102F800043685E6B002E10D0736803AD01938368B5
:102F9000083603936960AC60EA602C74019B9C4224
:102FA00005D108492800FFF76FFF09B0F0BDA30065
:102FB000F1582800FFF768FF3B68002BF5D101347A
:102FC000ECE7C0460007030010B54A68014922F04B
:102FD000F2FA10BD81360300F0B58BB004000E008C
:102FE000150000210822684628F096FA14220021D4
:102FF00005A828F091FA202307936B4605940893BF
:103000001C23002D02D0042D10D11A23216805A8FD
:103010000693FFF739FF0221009F042F0ED12A00EB
:10302000310020690BF07CFA0BB0F0BD1B23216846
:1030300005A80693FFF728FF0321EDE7381EF3D01C
:1030400002AB00220294039604950BF01DFE042DA2
:10305000EAD00148E8E7C0464CCA0200F0B51F4B71
:103060008BB08200D35803AF0C0008220021060069
:103070003800019328F050FA019B05AD6B601423D2
:10308000AB600023280021680594EF602B74FFF7E4
:10309000FBFE0398042805D1216930000BF08CFD5C
:1030A0000BB0F0BD00280AD0210023F039FE022E1B
:1030B000F6D10BF0D9F8440001202043F0E7022EAE
:1030C00001D00020ECE72623216828006B60FFF781
:1030D000DBFE3B68002BF4D16400EDE704D0020076
:1030E000F0B51600724272418BB01F320C00019293
:1030F00000210822070003A828F00EFA019B05AD65
:1031000006930823079303AB089300232168280044
:103110002B740594FFF7B8FE039B002B08D1002EFB
:1031200006D11F33216828006B60AE60FFF7ACFE4C
:10313000039804281AD120690AF082FF144BC26850
:103140009A4211D1002E07D02368586823F084FBDF
:103150000100380022F064F98022324321693800EE
:103160000AF086FF0BB0F0BD3200F7E7002805D06B
:10317000210023F0D5FD00220100F0E7200023F01C
:103180008CFD230002000349380022F014FAE9E71D
:10319000455500003635030070B504000D000B499D
:1031A00022F03EF96968002220000AF061FF084918
:1031B000200022F035F9A968002220000AF058FF0B
:1031C0000449200022F02CF970BDC0463F360300B0
:1031D000003503007AB00300F7B5002543680830D6
:1031E0000F0006002C000193019BAB4201D120008F
:1031F000FEBDAB00F358084A934205D0074AD96890
:10320000914203D03B6001340135EDE73900586B42
:10321000FFF7E2FF2418F7E7000703002132000060
:10322000F0B58FB005000F00406B05A90192029325
:10323000FFF7D2FF061DB600300025F062FE040045
:10324000002120C022F08BFB32002000103A103009
:10325000002128F061F9012F05D1029B1B6803931F
:10326000042B00D186E007AE08220021300028F0B0
:1032700053F90922002309A8426029000332826021
:10328000C66003740993FFF7FFFD079804282ED149
:103290000598029BC668019A3900B047206120005A
:1032A0000AF0CEFE854265D100230822290009A834
:1032B000089307930B9309940A92FFF7E5FD079B88
:1032C000002B57D00198384336D107AA010023F0CC
:1032D00038FD0500294B9D424CD0280023F0DDFC31
:1032E00027490200274802F0B9F9FCF770FF0028CF
:1032F000D5D0019A3A4306D106AB012106950BF0D1
:10330000C3FC0400CBE7019B5C00E4190134A4007A
:10331000200025F0F6FD221F0390029920C028F01E
:10332000E0F8791C039B019A30680BF0ADFC0400B7
:10333000039825F00DFEB2E7019B5D00ED19023503
:10334000AD00280025F0DDFD2A000600079B02994C
:1033500003600393089B083A4360083028F0C1F8E3
:1033600032000199380023F0ECFC0500300025F014
:10337000EFFDAFE720000FB0F0BDC0464CCA020021
:1033800087350300CCDC020010B5C468002C06D1E0
:1033900042680449044802F061F9FCF718FFA047AD
:1033A00010BDC04648360300CCDC0200F8B504006E
:1033B0000D0016001F0020F024FF002809D1200076
:1033C00023F06BFC0B4902000B4802F047F9FCF7B5
:1033D000FEFE042806D13B003200290020690BF0D4
:1033E00053FCF8BD210007F0E3FE3B00320029004A
:1033F000F5E7C0466B350300CCDC0200F0B5154B99
:1034000089B016008200D5580C000C22002107005C
:10341000684628F081F8182303A8456083600025DA
:103420006B462168C36003940574FFF72DFD009B74
:10343000042B06D13200216938000BF0ABFD09B036
:10344000F0BD181EFBD06A4629000120029623F029
:1034500078FCF4E774CE0200F0B50D0085B001A948
:1034600007001600280002AA20F0C2FE00230199DE
:1034700002988B4225D13C2025F055FD244B0400B9
:103480000360244B47608360234B4563C360234B39
:1034900086630361224B03A94361224B8361224B64
:1034A000C361224B0362224B4362224BC36228005A
:1034B000FFF792FE012812D91F49204821F0A8F9F0
:1034C00009E09A008258D468002C06D152681C4941
:1034D0001A4802F0C3F8FCF77AFE0133C9E7A36B80
:1034E0000022181D4E2108F02FFB051E0DD00322CF
:1034F00043681A4009D11B685B68F22B05D1031D94
:103500000121104820F0D7FE6860200005B0F0BD12
:10351000C8CF0200E130000021320000AD330000CE
:103520005D300000FD3300002D420200D92F000065
:10353000814302003743020011360300CCDC020055
:10354000E835030050CF020037B50D001C00002302
:103550001100009301220333280000F089F9012DA6
:1035600007D0032D09D00949094821F051F9FCF78A
:103570002EFE20680AF064FD3EBD206804F0D0FAFB
:10358000A2686168FFF768FFF6E7C046653603008A
:10359000CCDC020070B505000C200C0025F0B1FC5D
:1035A000024B45600360846070BDC0468CCF020052
:1035B000F8B50F00B8421FD0032505401ED1114BAE
:1035C00002689A421AD1406B002816D0446808302D
:1035D0000600002C14D0631E9D4204D30A4BE4184D
:1035E000A400A059E6E7AB003900F058FFF7E0FF70
:1035F000002802D10135EEE70120F8BD0020FCE7EC
:103600002000FAE7C8CF0200FFFFFF3FF0B585B00A
:103610000500019108008B0717D10B68154A9342EA
:103620000BD10123029301AB03930024029E039F5D
:10363000B44210D1104805B0F0BD104A934204D1F5
:1036400003AA02A920F0D4FDEFE70D490D4821F0AF
:10365000DFF8FCF7BCFDA300F9580B4B994206D0EC
:103660002800FFF7A5FF002801D10134E0E7074853
:10367000E1E7C046C8CF0200A409030000CE020063
:10368000AF350300CCDC020000070300AC090300E7
:1036900010B5830703D1064B02689A4205D005494D
:1036A000054821F0B5F8FCF792FDFFF7AFFF10BD1C
:1036B000C8CF020048350300CCDC020010B504007E
:1036C000080020F0C9FE0300002C03D0012C06D016
:1036D000002003E00348002B00DC034810BD40003D
:1036E0002043FBE7AC090300A409030070B545685B
:1036F000C6688468102025F004FC034B4560C66052
:103700000360846070BDC0465CD0020070B50D00DF
:103710004A688B680849040021F04DFFEA68012AD5
:1037200004D10649200021F07BFE70BD0449200031
:1037300021F041FFF9E7C0468E3603004A950300A9
:103740009B36030030B5040087B00D000020042A2A
:1037500020D1200020F080FEAB071DD1154B2A6838
:103760009A4219D103AA290011F076F8102025F009
:10377000C8FB114B039A0360E36861685A4352180F
:103780004260049A616801925A4352188260059A15
:103790005343C36007B030BD002301002A002068F6
:1037A0000AF00EFEE36858436368C31801205B000B
:1037B0001843EFE7EC00030020D00200F0B5214BE6
:1037C0008DB005AC0138009304310194072300F05B
:1037D00081F8A0681C4D0026A84202D00AF018FD0E
:1037E000C6B260691827A84202D024F0CEFE0700B6
:1037F000A0691922A84202D024F0C7FE0200206965
:10380000A8420DD003AA02210AF0C6FD039B186846
:1038100024F0BBFE039B0700586824F0B6FE0200AC
:10382000390003A813F080F9059903A813F0D8F91B
:1038300003A8E3683200616813F0E2F928000DB0D4
:10384000F0BDC0463CD102004CCA020010B50EF0DB
:10385000F3FE034B002800D1024B180010BDC046F8
:10386000AC090300A40903000048704744D20200D9
:1038700010B51C0002AB1B78002907D0002B05D126
:103880000F49104820F0C4FFFCF7A1FCA24207D169
:10389000824213D003000C490A4801F0DFFEF3E72F
:1038A000824205D9121A0949064801F0D7FEEBE712
:1038B000844203D2030022000549EDE710BDC04653
:1038C00015370300CCDC02003E37030077370300D6
:1038D000A9370300F0B50025170087B00C9C0D9E9A
:1038E00003900491059302950195059B9D4208D193
:1038F000019B039A934241D22449254820F088FF36
:1039000026E0039B9D4211D263689B05F4D4019B82
:10391000049A01330193AB00D058FF22636813402F
:10392000012B22D10AF0B2FD307015E0236800228D
:10393000D90006233800194308F006F900280FD1F2
:103940006368DB0506D522681249114801F086FE3E
:10395000FCF73DFCA368336001350C340436C4E742
:10396000029B406801330293D7E7022B03D10AF090
:103970004FFC3060F0E7032BEED1FAE73B68029A88
:10398000DB0805499A42B8D307B0F0BDEF37030012
:10399000CCDC0200D837030010380300F8B50378F8
:1039A0000400002B1BD0402B1CD101200023190048
:1039B0001D001E002278002A3CD10132002E0FDCAF
:1039C000002D0DDC00290BDC033B934208D9013CA0
:1039D00023785C2B04D0002801D00A2B00D10022D0
:1039E0001000F8BD3D4920F0E7FD0028DDD13C493D
:1039F000200020F0E1FD0028D7D13A49200020F036
:103A0000DBFD0028D1D13849200020F0D5FD002869
:103A1000CBD13649200020F0CFFD0028C5D1344954
:103A2000200020F0C9FD0028BFD13249200020F03D
:103A3000C3FDBBE7272A12D1002B01D0032B09D1EC
:103A40006278272A06D1A278272A03D10234243AA1
:103A5000D31A02E00122012BFAD90134AAE7222A63
:103A600012D11A000427BA430AD16278222A05D15A
:103A7000A278222A02D102343A00E9E7002B01D0D1
:103A8000022BEAD10222E3E75C2A09D16778272FCB
:103A900001D0222F04D11A00571EBA41A418DCE726
:103AA000002BDAD15B2A12D006D8282A0DD0293A69
:103AB00057425741F61BD0E77B2A0AD07D2A0AD00D
:103AC0005D3A57425741ED1BC7E70136C5E701355F
:103AD000C3E70131C1E70139BFE7C0466A300300DF
:103AE0009B3003008130030097300300477F0300C1
:103AF000F6BC030065350300F0B505008BB0461831
:103B0000049207930296029B5C1EA54201D902957E
:103B100010E0207810F03EFD002801D00294F2E77A
:103B2000207810F043FD0028F8D123785F2BF5D0E2
:103B30002E2BF3D0734B1D68029CB44245D3029BDD
:103B4000E31A0193B44223D20027AB689F421CD2F0
:103B5000FB000393EB68FA00985800283AD0042839
:103B600038D009A904F068FC019B099A010093422E
:103B700030D11A00029827F03CFE00282AD1EB68C9
:103B8000039A9B185868002826D100200BB0F0BD7E
:103B90000024260027000394AB689C4238D3039B83
:103BA000002BF2D0012B63D0019B9E4260D80023F2
:103BB00040260393039BAA68934260D3524904981A
:103BC00021F02EFC01204042E0E723782E2BB6D0D6
:103BD0000134B2E70137B8E7032318420DD1026878
:103BE0004A4B9A4205D123F04AFF0500631C029319
:103BF000A2E7474903008A4202D00AF021FA0300F3
:103C00009D6B002DC1D0434B2A689A42EED0BCE791
:103C1000EA68E3009858002826D0042824D009A98F
:103C200004F00AFC099B05900693069A019B9342B7
:103C30001AD801001A00029827F0DBFD002813D1E2
:103C4000019B002F08D1069E059F0AE0059AF95CAA
:103C5000D25C91420AD101339E4202D3069A93422A
:103C6000F4D9039B01330393013495E71E00F8E771
:103C7000019B079AFB181360019BF01A86E7039BD0
:103C8000EA68DB009858002838D0042836D009A903
:103C900004F0D2FB099B05900693069A019B934280
:103CA0002CD801001A00029827F0A3FD071E25D189
:103CB00033000F220F33DC171440E41824112401C1
:103CC000A41B012C00DC1034069A33199B18402BDE
:103CD0000BD9059A1049049821F06DFC099E0DE05E
:103CE0000E49049821F09CFB0137BC42F8DC059991
:103CF000049821F095FB099BF6183619039B0133B4
:103D0000039357E7AC09002007B00300201003001D
:103D1000C8CF020094D602002E380300799B03001E
:103D200010B588B001AA6946040001F03FFD009B70
:103D3000022B2AD902AA322104A80FF057F9019BBD
:103D400013495A6802A821F036FC20000AF078F9DD
:103D5000104BC2689A4210D123680F495A6802A8D2
:103D600021F029FCE368002B07D05A68002A04D010
:103D70000022996802A80AF07BF904A824F0CCF884
:103D80000EF0CCFC04A824F078F808B010BDC046B2
:103D90005F380300455500006838030070B5050022
:103DA00090B0002804D11F481EF088F810B070BDF4
:103DB00004A8FCF7F1F9041E19D12E68290001A806
:103DC000012202F035F923002200310001A8FEF79C
:103DD0003BFD040003200EF01FFC200022F099FFA1
:103DE000012040420EF018FCFCF7ECF9DEE7012060
:103DF00040420EF011FC05990B480AF05DF9059858
:103E00000AF01EF909490400FFF7D2FB0028CDD1C2
:103E100007492000FFF7CCFB0028C7D10598FFF722
:103E20007FFFC3E732380300B4EA020090DC0200EF
:103E300014DA020037B52A4B01AA1A6007F0C6F956
:103E4000E120C00007F0CCF92649274806F00CF81D
:103E50000AF006FE0EF0BEFBFCF78CFB0EF0B6FC83
:103E60000023224C224D63672B78012B0BD1F823C2
:103E70009B021A784D2A1BD15A78502A18D159889A
:103E80001C4820F0B6FB2B78002B25D108F08EFAC9
:103E90000028F8D0184823F032FE082200211748E5
:103EA00027F03AFB00239034236022F02EFF37BD29
:103EB000002307211A00124806F044FC002802D013
:103EC00020F0A1FBDFE7482001220E49FF300BF074
:103ED000B7FC22F051FFD6E708F0C6FAD8E7C04693
:103EE000E80200200038002028130020AC09002040
:103EF0004402002004E0030074380300180A002084
:103F00006C380300F8CD020007B506F03FF8054B0A
:103F100001A81968091A890805F0F0FF06F04AF8A7
:103F200007BDC046E802002010B50AF0D5F919F027
:103F3000B9F80022084B18F0A9FA084A084B17F004
:103F400071FE19F001F90323020002209A43054B88
:103F50001043C01810BDC04600806640182D445460
:103F6000FB2109400000808010B50AF0B5F919F076
:103F700099F8094A094B18F089FA0022084B17F002
:103F800051FE19F0E1F80323020002209A43054B89
:103F90001043C01810BDC046182D4454FB210940E1
:103FA000008066400000808010B50AF095F9011C81
:103FB00017F05AFA024B002800D1024B180010BD2E
:103FC000AC090300A409030010B50AF085F9440008
:103FD00064080849201C17F047FA002805D1054954
:103FE000201C16F0C7FA002801D0034810BD034872
:103FF000FCE7C046FFFF7F7FA4090300AC09030074
:1040000010B50AF069F9034B034002201843024B34
:10401000C01810BDFCFFFF7F0000808010B50AF0C3
:104020005BF9440064080849201C17F01DFA0028B9
:1040300007D10549201C16F093FA002801D1034846
:1040400010BD0348FCE7C046FFFF7F7FAC090300BB
:10405000A40903001FB5002301930AF03DF901A94B
:1040600019F06CFB0322030002209343064903432B
:104070005B180293019B934303435B1802A90393CC
:10408000FEF7EEFD05B000BD0000808070B50D00AC
:104090000AF022F9041C28000AF01EF917F0FCF9B6
:1040A0000100201C19F026FB0323020002209A4382
:1040B000014B1043C01870BD000080801FB5002365
:1040C00001930AF009F901A919F0EAFA032302247D
:1040D0009843074B2043C0180290019822F022FF1A
:1040E00002A903902000FEF7BBFD04B010BDC0463E
:1040F0000000808070B50D000AF0EEF8041C280066
:104100000AF0EAF8011C201C19F0A6FD03230200A6
:1041100002209A43014B1043C01870BD00008080FC
:1041200070B50D000AF0D8F8041C28000AF0D4F885
:10413000C00FC307600040081843032302249843BC
:10414000014B2043C01870BD0000808070B50D0089
:104150000AF0C2F8041C28000AF0BEF8011C201C5A
:1041600019F002FD0323020002209A43014B104381
:10417000C01870BD0000808010B50AF0ADF819F0CD
:1041800097F80323020002209A43024B1043C01801
:1041900010BDC0460000808010B50AF09DF819F0EF
:1041A0008FFC0323020002209A43024B1043C018E5
:1041B00010BDC0460000808010B50AF08DF819F0DF
:1041C0002BFC0323020002209A43024B1043C01829
:1041D00010BDC0460000808010B50AF07DF819F0CF
:1041E00091FB0323020002209A43024B1043C018A4
:1041F00010BDC0460000808010B50AF06DF819F0BF
:1042000043FB0323020002209A43024B1043C018D1
:1042100010BDC0460000808010B50AF05DF819F0AE
:10422000AFF90323020002209A43024B1043C01847
:1042300010BDC0460000808010B50349034801F05E
:104240000DFAFBF7C4FFC0468238030044DD0200CC
:1042500070B5060008680D000AF03EF80021041C45
:1042600016F07EF9002801D0FFF7E6FF201C19F0B8
:104270005BFD041C012E06D1032302209C43204336
:104280000C4BC01870BD68680AF026F80021051CA8
:1042900016F066F90028E7D1281C19F045FD011C2D
:1042A000201C16F035FC0323020002209A43104321
:1042B000E6E7C0460000808010B50AF00DF819F05E
:1042C00057FC0323020002209A43024B1043C018FC
:1042D00010BDC0460000808070B50D0009F0FCFFE5
:1042E000041C280009F0F8FF011C201C19F098FD9F
:1042F0000323020002209A43014B1043C01870BDF3
:104300000000808010B509F0E7FF0021041C16F0C2
:104310001DF9002801D0FFF78FFF201C19F014FFB2
:104320000323020002209A43014B1043C01810BD22
:1043300000008080F0B5836999B05A1E06339B0057
:104340000492C218079102920F210122C31804336C
:1043500003930369019006A81A4009180A70032202
:1043600093430A930CA8FBF717FF031E01D000F03C
:104370003FFD019A5568D468079A002A00D184E26B
:104380002A785E2A00D180E2079807930BF03AFA68
:1043900004000AE0D24B63600434D24B1A6B002A4B
:1043A00000D171E200221C6B1A63FBF70BFF0D9426
:1043B00000F01EFDCC4BEEE7CC4BECE77F216B7899
:1043C0005B06DB173A78DB01100052B2084003436A
:1043D0000137002AF6DB01225B001343DBE70023F1
:1043E0007F213A78DB01100052B20840C318013730
:1043F000002AF6DBDB000622EFE7032203379743B0
:1044000008CFC8E70023C6E700237F213A78DB0105
:10441000100052B20840C3180137002AF6DB9B0097
:104420005B42029A9858002800D0EEE2B049B148A9
:1044300020F0EEF9ACE700237F213A78DB01100091
:1044400052B20840C3180137002AF6DB029A9B00DB
:104450005B42985824F09FF8E5E700207F223B78E4
:10446000C00119005BB2114008180137002BF6DBC0
:10447000251D0AF045FB60605EE000207F223B784E
:10448000C00119005BB2114008180137002BF6DBA0
:10449000251D0AF003FBEEE700217F223B78C901CE
:1044A00018005BB2104041180137002BF6DB206882
:1044B00022F056FC206070E700217F223B78C90182
:1044C00018005BB2104041180137002BF6DB2200C8
:1044D00001CC0AF087FC60E7251D0AF029FBCAE73A
:1044E000251F0422216828680AF01AF8286023E0B2
:1044F00000237F213A78DB01100052B20840C31834
:104500000137002AF6DB9B005B42029A2168995032
:10451000E3E000237F213A78DB01100052B208402B
:10452000C3180137002AF6DB9B00029A5B42216820
:104530009858251F24F031F82C002EE700207F2208
:104540003B78C00119005BB2114008180137002BFD
:10455000F6DB2168251F0AF0FFFAEDE700207F2235
:104560003B78C00119005BB2114008180137002BDD
:10457000F6DB2168251F0AF007FBDDE700217F221B
:104580003B78C90118005BB2104041180137002B7D
:10459000F6DB231F1A6820680AF04CFC083CFCE696
:1045A0002200231F083A12682168186809F0B8FF32
:1045B0000C3CF2E600237F213A78DB01100052B276
:1045C0000840C3180137002AF6DB029A9B00D31A71
:1045D0001A68002A00D129E700221A60DDE60025CA
:1045E0007F223B78ED0119005BB211404D19013774
:1045F000002BF6DB029BAD005D1B286823F0CBFF90
:10460000002800D112E70021286823F0C6FFC4E685
:1046100000207F223B78C00119005BB211400818CE
:104620000137002BF6DB0AF0A3FAB6E600207F2262
:104630003B78C00119005BB2114008180137002B0C
:10464000F6DB0AF0ADFAA8E62368A4E62368A360C7
:10465000231F1B68636008349FE6231F19682268C4
:104660002160BAE7221F1368216823602300083BFA
:1046700018681060196090E67B783A781B02134343
:104680001D4A9B18EF1888E67E783B782068360232
:104690001E4309F0FBFEEF1C251F2C00002800D153
:1046A0007BE6164BF618BF1977E67E783B782068D4
:1046B00036021E4309F0EAFEEF1C251F2C000028DD
:1046C00000D06AE6EDE77E783B78360220681E432C
:1046D000EF1C09F0DBFE0028E3D1043C5DE6C04698
:1046E000A4090300AC0900204CCA0200AC09030075
:1046F00094380300D4DA02000380FFFF0080FFFF3C
:104700007E783B78360220681E43EF1C09F0BEFE1F
:104710000028C6D0E1E726002768220038001721CC
:1047200008360AF05FFB3800320016210AF05AFB07
:1047300000213200080022F004FBAB786A781B02EB
:1047400013430A9A0F210C320A920A9AEF1CFB18A3
:104750001360022206ABC9180A9D0B781A43231D69
:1047600013436B6000230A9A0B709360A0603400BF
:1047700013E625002668AC4B083D9E4208D16660D2
:10478000A6602A000021032022F0DBFA2E60D3E687
:10479000012131402CD07610231F012E11D126008B
:1047A0001A680C3E0592A04A00211A60032022607C
:1047B0006260320022F0C5FA059B336003232B6050
:1047C000ECE626002A68103E05921A68002106923F
:1047D000954A03202A601A602260320022F0B1FA62
:1047E000059B069A336023000C3B1A600523E6E71D
:1047F0002B682E602600103E23603200032022F03A
:10480000A0FA09F043FE00280DD00122864B06A92C
:1048100033600A9B5B6813400E32521813700A9B78
:104820000C3B0A93A3E7236833602300043C22680F
:104830000C3B1A6080E67B783A781B0213437B4A74
:104840009B18EB186360EB78083423600F267F21F8
:104850000220012506AA2368B6180B4205D1221FA3
:104860001768002B00D0A3E698E60A9A013B52682D
:10487000024270D0220008C20523636014000A9B24
:104880001F680A9B0C3B0A933D00019B6F1C5D60F7
:104890002B78180010385A2800D907E315F07CFC53
:1048A0007AFD8AFD8CFD06038EFD06039FFDADFD9E
:1048B000B2FD0603B4FDCBFDDDFDEDFDFCFD0CFE00
:1048C0001CFE20FE28FE39FE4EFE5EFE6EFE80FEC1
:1048D0008AFE9FFEB8FEC6FE060306030603060315
:1048E000D4FED6FE1DFFDDFEE2FEECFEF4FE05FF6B
:1048F00013FF30FF0603060306033BFF69FF630057
:1049000063008000A300A700B700B700CBFF060339
:10491000060306030603060306030603060306034F
:10492000C800DA00EC00FE000D0116012B013D016C
:104930004F016C0182013002570282026F020603AE
:104940009701A201AD01BA01C601E201FC01190201
:10495000DA02EF0200030A9A52682A4032700A9A79
:104960000C3A0A9279E77B783A781B0213430A9A49
:10497000EF1C0C320A920A9AFB1813602B780A9AE1
:10498000403B584258410F21430006A809180878B7
:1049900003432343536000230A9A0B709360FCE4A3
:1049A000206800F0A3FE251F002804D0FBF70AFCB6
:1049B0002B680D931CE223681B4A2C00934200D104
:1049C000EBE45B10DBB2012B00D03FE702220A9B35
:1049D0000399994200D8A3E1FBF7F4FB0020019B67
:1049E000DC6019B0F0BD20680AF048FA62E57E7814
:1049F0003B7836021E43019BEF1CDC6020680AF006
:104A000063FA002801D1043C4DE66060C4E4012251
:104A10000A9B06A95B6813400E32521813700A9B5A
:104A20000C3B0A93B9E4C0464CCA02000380FFFF66
:104A300000207F223B78C00119005BB211400818AA
:104A40000137002BF6DB8300E41A04342100FEF763
:104A500007F92FE500207F223B78C00119005BB2E7
:104A6000114008180137002BF6DB8300E41A0434E8
:104A7000210020F024FF1DE500237F213A78DB018F
:104A8000100052B20840C3180137002AF6DB9B0021
:104A90005B422168185906F0F5FB1EE600207F22D4
:104AA0003B78C00119005BB2114008180137002B98
:104AB000F6DB251D1FF04CFEDDE42500231F083D1D
:104AC0001A68216828681FF07BFE35E500237F21E6
:104AD0003A78DB01100052B20840C3180137002AAF
:104AE000F6DB01339B00221F5B42126821681859D4
:104AF0001FF066FE52E500207F223B78C0011900BE
:104B00005BB2114008180137002BF6DB8300E41A72
:104B1000043421000EF022F8CCE400237F213A78FF
:104B2000DB01100052B20840C3180137002AF6DB3F
:104B30009B005B422168185923F093F8CDE50023D0
:104B40007F213A78DB01100052B20840C3180137C8
:104B5000002AF6DB251F022B05D1DC4A21682868D4
:104B600008F0C0FCC2E42600083E226829683068CC
:104B700008F0B8FC3060FAE500257F213B78ED01B4
:104B80001A005BB20A4055190137002BF6DB2200F0
:104B9000290020680AF0E8FCCD4B5D19AD006419CE
:104BA000FFF7FBFB00257F213B78ED011A005BB28C
:104BB0000A4055190137002BF6DB22002900206836
:104BC0000AF026FDFF222B0A13401540E5E70322D9
:104BD000FB1C93430022186811001F1D251D22F0A5
:104BE0005DFF48E40322FB1C9343251F22682968CC
:104BF00018681F1D22F052FF78E40322FB1C934328
:104C000019795F1D8A00A41A04342200186822F062
:104C100060FF4FE40322FB1C934318798021C243B9
:104C2000490092005F1DA4180143EEE700207F2198
:104C30003B78C0011A005BB20A4010180137002B04
:104C4000F6DBFF25FF220100C3096D0011402B4058
:104C50005B189B00E41A000A0240231D20680AF03A
:104C600013F827E400217F223B78C90118005BB2CA
:104C7000104041180137002BF6DBFF22CB09520010
:104C80001340CAB29B189B00E41A083C2200002083
:104C90000AF03AFBFFF70EFC00237F203A78DB0195
:104CA000110052B20140CB180137002AF6DBFF2178
:104CB0001800FF250840DA096D002A40451C5219EA
:104CC0009200A41A1B0A1940220022F03AF8FFF7BA
:104CD000F1FB00217F223B78C90118005BB2104034
:104CE00041180137002BF6DBFF22CB09520013409D
:104CF000CAB29B189B00E41A0C3C22000120C7E7B3
:104D00000F2206ABD2181378002B00D15EE60121EA
:104D10000A9B5B680B4013700A9B0C3B0A9355E699
:104D20000A9B5B6813420ED003220A9B21685B68D2
:104D300093431C0059609A600A9B08341F680A9BC1
:104D40000C3B0A93A0E50A9B0C3B0A933FE66B7869
:104D5000022B03D1043C2068FFF718FB002BFAD18B
:104D60000A9B039A934203D25A495B48FFF760FBC0
:104D70009868002801D0FFF709FB0C3BF1E7079E7C
:104D8000231F0593002E1CD0079E0021320007919F
:104D90000BAB201F00680AF0C9FC012815D12F00B9
:104DA0000B9B2360FBF70EFA019B06AA5F60DC6099
:104DB0000F239B181A780A9B01201343019A136151
:104DC0000FE60BAB32002168E3E700282FD10B9BE5
:104DD000043C002B00D13D4B2360002E4CD03F49BA
:104DE00030001FF01FFD002846D0FBF7EBF90D96B1
:104DF0000D9B3B491868FEF7DBFB002800D1AEE0B5
:104E0000019B5A68002A00D1A9E01378432B00D0F7
:104E100092E0937850781B02D11C0343019ACB187F
:104E20005360D3680593043BD360FFF79BFA0228D5
:104E30000FD12B490B981FF0F5FC002805D00B98DB
:104E400000F0ECFB043C2060C7E7FBF7BBF90B9BD1
:104E5000AFE5059C00207F223B78C00119005BB2C2
:104E6000114008180137002BF6DB251F2A6821683E
:104E70000AF0E6FCFFF73AFB059CFFF78EFA0021EB
:104E80007F223B78C90118005BB2104041180137FE
:104E9000002BF6DB250001CD0AF0E4FCFFF7EBFA6E
:104EA0002068251F21F068FFFFF746FBAF2B05D8D0
:104EB0000120803B5B000343FFF76DFABF2B11D845
:104EC000B022D31A9B00FFF7ACFAC0464CCA0200CE
:104ED000FFFFFF3FDA380300C4DB0200E8D802001E
:104EE0000CDC0200CF2B04D8C022D31A9B00FFF7A2
:104EF0000CFBD62B06D8D03B1800216809F05CFECD
:104F0000FFF7D8FAFA2B08D8251FD73B18002268DC
:104F100029680AF03FF8FFF7E9FA4C494C481FF0BE
:104F200077FC0400FBF74EF9049B019A06339B00C3
:104F3000D3185C60022054E55E2B10D1019B019ACE
:104F4000DC680D98231DD36000F068FB019B606056
:104F50005B68019A059301335360FFF703FA0D9BD9
:104F60003C4A934231D03C4A93422ED0019B0BA83D
:104F70001B6805930B9323F069F804000BA823F03A
:104F800065F805000BA823F061F8019B01005B6840
:104F90000593019B1B680693069A059B9E1A1F2387
:104FA00001229C46361B0B9C2378002B09D058B25B
:104FB00000282EDB6046013418405B090B948642C2
:104FC00031D22B000D9800F0B9FB0F23012106AA66
:104FD0009B181A78002A29D10A9A039991422DD850
:104FE00001221A700A9B0D991B680593059A019B73
:104FF00005915A6003220A9B5B6893430A9A916069
:10500000164A5A600D9A9A6012680C331A60019A17
:105010000AE70F20E0271840FF001B011F406378BC
:1050200002343B43CAE7361AD218BCE70A9A5268E0
:105030000A401A700A9A0C3A0A92CAE7049B019A2B
:1050400006339B00D3180D9A5A6073E7C0380300EB
:1050500010DB02003CD702004CD702004CCA020011
:1050600010B504000C2023F04CFF034B4460036098
:105070000223037210BDC0464CD6020010B50400D6
:10508000102023F03EFF044B0360237A0371636812
:1050900083600023C36010BD10D6020010B5040069
:1050A000102023F02EFF044B84600360034B436009
:1050B0000023C36010BDC04628010300E94602007A
:1050C00010B5043020F06AFC004810BD4CCA020044
:1050D000002803D0012808D0002005E007224B68F3
:1050E0000448934300D1044870474B68DB085B00D9
:1050F0001843F9E7AC090300A409030010B50349FC
:1051000003481FF085FBFBF762F8C0461E39030019
:10511000D8D9020070B515001A001C0006F014FD65
:10512000002802D04368002B0BD12B1E04D1074B63
:10513000022C01D1FFF7E2FF012C00D143601800DF
:1051400070BD022CFBD100224260F8E74CCA02007D
:10515000F8B504000D000B7A124A9B00995820F014
:105160005FF91149200020F05BF92800FFF786FF66
:105170000126070038001FF0C1FA051E04D10B49B3
:10518000200020F04DF9F8BD002E03D10849200081
:1051900020F046F901222900200008F069FF0026CE
:1051A000E8E7C04688D602005639030059390300A3
:1051B0000035030030B5002585B001A90400019534
:1051C0001FF07DFAA84205D10A490B481FF020FBC9
:1051D000FAF7FDFF636802A9083B63600368029366
:1051E00043680393042328C00220FDF739FD05B06E
:1051F00030BDC046F9380300D8D90200F0B51368B5
:105200001400012287B00F680D000092D908022314
:105210000600FEF72DFB022E12D10323686803401F
:105220001DD101682B4AC968914218D12A68904261
:1052300006D0059305A968681FF041FA061E06D13D
:10524000002563689D4233D3234807B0F0BD381D65
:105250000122316806F078FC73684360EAE709F0E0
:105260000DFE0390039809F055FE0028E8D009F0E0
:1052700005FE050009F04EFE0290280009F04AFEE6
:105280000600280009F046FE029B002B03D0002EEA
:1052900001D0002805D0114911481FF0B9FAFAF7DA
:1052A00096FF381D0122029906F04EFC4660D9E7B0
:1052B000A368EE009959002909D0042907D0381DA8
:1052C000012206F041FCA3689E1973684360013512
:1052D000B7E7C046C55400004CCA02002639030097
:1052E00044DD020073B50C0015001B280DD000230F
:1052F0001F2808D1081D0022290006F025FC1A4BA2
:10530000002800D1194B180076BD0323194208D19B
:10531000174922688A4204D12B4002D12968914260
:10532000F1D0AB07EED1134B2A689A42EAD16A68F2
:105330006368534007229343E4D1019301A92000FD
:105340001FF0BDF9061E01D1074BDCE7281D002226
:10535000316806F0F9FB0028D4D04168706808F085
:1053600005FF0028EAD1CDE7AC090300A40903003A
:10537000D0D6020094D60200F7B50B681C4A040090
:105380000D00934203D05A681A4920F014F91A49C3
:10539000200020F045F800230127019301A92800EF
:1053A0001FF08DF9061E0CD11449200020F038F8AA
:1053B0002B680F4A934203D01149200020F030F8A7
:1053C000F7BD002F03D10F49200020F029F801225A
:1053D0003168200008F04CFE0B49200020F020F836
:1053E00001227168200008F043FE0027D6E7C0467E
:1053F00094D60200183903001C39030073B8030067
:105400004A950300003503004536030010B504003B
:105410000C2023F076FD034B4460036000230372ED
:1054200010BDC0464CD6020010B504000C2023F07D
:1054300068FD034B446003600123037210BDC04646
:105440004CD6020010B50430002206F07DFB002887
:1054500005D1044904481FF0DBF9FAF7B8FE4068AB
:1054600010BDC0461E390300D8D9020010B5024B4A
:1054700008C020F074FA10BD94D60200F8B50700F9
:1054800048680E0009F0FAFC040008F0DBFF0C4D40
:10549000022F00D9B568002809D11FF059F906007C
:1054A000200009F037FD011E03D13000F8BD401087
:1054B000F3E7331D0122180006F046FB4560EFE7D5
:1054C0004CCA0200F0B5070089B000201E000D0094
:1054D00001921FF03DF90E4B040007609F4203D17B
:1054E0000423027913430371019B2B430DD03368CE
:1054F000AA00B218019905A80394049320F041FA78
:10550000681C05AA03A9FFF779FE200009B0F0BDC9
:10551000D0D6020010B5002A03D11FF05BF908486D
:105520000AE0042A09D10430002206F00DFB00280D
:1055300001D1FFF7E3FD406810BD1FF041F9EEE730
:105540004CCA0200F7B50D001100002206000092BF
:1055500028001F000B4BFEF78BF9102023F0DEFC18
:10556000041E08D1084A094B094CDA610023266061
:105570002000A360FEBD39002800FDF771FBE0604C
:10558000F4E7C046FFFF0000F8CD0200AC090020A0
:10559000BC09002010B5013810C9FDF761FBE060BF
:1055A000004810BD4CCA0200F8B57F2553B2040074
:1055B0000E0017001540002B0ADB6B1E012B07D8CD
:1055C0000B68586821F048F9010020001FF028FFFF
:1055D000022D0ED10F4920001FF022FFF368002B8F
:1055E00002D05A68002A0CD10B4920001FF018FF86
:1055F000F8BD002DF2D03A00F1682000FDF7C4FAA2
:10560000F6E7012AF7D100229968200008F030FD62
:10561000EEE7C04645360300C7760300C36803487B
:105620005A68002A00D098687047C0464CCA0200E9
:10563000136810B51400002B03D17D2902D1C36873
:10564000136010BD044B02689A42FAD1BA29F8D10E
:10565000FFF7E4FF2060F4E70CDC02000EB470B545
:10566000050087B0102023F059FC041E0BD11B4B02
:105670001B4A1C4C1D619861DA61200007B070BCA8
:1056800008BC03B018470021056081600120FDF7C8
:10569000E7FA0B9B0500E060002BEED025211800F7
:1056A00026F088F8061E09D10B9826F09BF83200E8
:1056B00001000B9802F012FAA860DEE702A81021A0
:1056C00022F0B0FB0CAA0B9902A801920DF0EEFC9F
:1056D00002A90548E56802F0CBF9EDE7AC09002026
:1056E000F8CD0200BC090020DC14030010B5030053
:1056F000820708D1064A0168914204D1054AD96857
:105700000120914203D004491800FDF751FF10BD5C
:10571000C8CF0200455500001CD8020010B5040097
:1057200008F08EFC044AC1682300914200D023692E
:1057300000229A6010BDC04645550000F7B505002F
:10574000160001930F0008F07BFC174BC2682C0079
:105750009A4200D02C69A568002D13D10C2023F0AB
:10576000DDFBA06000280CD00323E580A380E28845
:10577000A16893000332E280019ACB181F605E603B
:105780009A60F7BDE388A18802338B42EFDB0331D7
:1057900089000122280023F0D7FB0028F1D0A3883C
:1057A000A0600333A380E2E74555000070B5060012
:1057B0000D00140008F044FC074BC1683200994208
:1057C00000D032699368002B02D12B60236070BD3A
:1057D000D2882A60FAE7C046455500000023FA2126
:1057E000084A89001360084A1370084A1360084A7F
:1057F0001160084A1370084AD36613670122074BE9
:105800001A707047F002002016090020EC020020F8
:105810001400002017090020AC09002018090020FE
:1058200010B5084B084A1978002907D1116B0029D7
:1058300002D0FFF7D3FF10BD30BFF4E700221A708B
:10584000F9E7C04618090020AC090020837F024810
:10585000002B00D101487047AC090300A4090300E4
:10586000A02010B50F49C0054B7F5A1C002B09D151
:105870004C8C0D4BA3430D4C03510D4B4A775200FA
:10588000D05A0DE010335B00CB185C88A123DB00FD
:10589000C450092AF1D10120FAF7DCFD0120404271
:1058A00010BDC04618000020F01F00000C050000CD
:1058B000F82A03000023E021A02210B583770C4BC7
:1058C0000902D205D1500B480DF0BAFF0A480DF07D
:1058D000B7FF0A480DF0B4FF09480DF0B1FF0948C1
:1058E0000DF0AEFF08480DF0ABFF084810BDC046F4
:1058F0000C050000741E03007C1E03008C1E0300B8
:10590000941E0300A41E03001C1E03004CCA0200C8
:1059100073B5041E09D1194D2B78002B2BD01849D3
:1059200018481EF08FFF2C7073BD174EF56E08F0EF
:1059300087FB164B2100984214D0154B2340062BB1
:1059400005D0A30712D1134B22689A420ED101A9A8
:10595000200002F071FD019B012B0CD1007821F099
:10596000D6FE010028001EF06DFFDDE70A490B4856
:105970001EF04EFF3063FFF731FFD5E71709002017
:10598000000D030018000020AC090020800D03006A
:10599000070080FFDC140300B3390300CCDC0200F5
:1059A000034B1878013843425841C0B27047C04693
:1059B00016090020F7B5A123A024224AE405DB0044
:1059C000E250C37F012219000D318A4001331E4984
:1059D000DBB262500191032B31D0C3770200030088
:1059E000002122333632198002339A42FBD1C47F20
:1059F000164A63000133D318052204259446012179
:105A000067465A1E12781E787A43114F0633BA1829
:105A10000F00AF4092191279013552008218568C4E
:105A20003E4356840D2DEBD10D34A023A122A1407D
:105A3000DB05D2009950828E01995A50F7BD0023A0
:105A4000CBE7C046F01F00000C0500007D390300C5
:105A50001800002070B5304D8CB0AB7F002B1FD0EC
:105A60002800FFF7A7FF2D4A2D4913680968063360
:105A700013608B4207D300242A4B14601B78012B40
:105A800010D0022B43D000232A8C6B77FF33FF33D7
:105A90001A4205D0E1222449D2000120FAF7A6FCDF
:105AA0000CB070BD214EF36E002B02D0336F002B73
:105AB00002D1FFF793FEE6E704F002FA6846FAF730
:105AC0006BFB00280CD11A4B186809F0FDF9040093
:105AD000FAF778FB04F0FEF92000FFF719FFD2E790
:105AE00004F0F8F9019B13491868FDF761FD0028DF
:105AF000F2D1019808F0A4FA0F4B984203D10F4954
:105B00000F481FF058FD019B00243363E4E70D4963
:105B100028001EF097FECCE718000020EC020020C1
:105B2000140000201609002061580000AC09002074
:105B3000F00200200CDC020098DA0200F0390300C9
:105B4000B4EA0200000D0300F7B50024009308AB8F
:105B5000124D1B780600080017000193EC662C67B5
:105B600009F08CF96A460E4B127818600D4BEE6600
:105B70001F600D4B28671A700C4B1C7009F0A4F9BC
:105B8000FFF7C6FE01220A4B1C600A4B1A70019BEC
:105B9000A34201D0FFF744FEF7BDC046AC09002088
:105BA000F00200201400002017090020180900202E
:105BB000EC02002016090020F0B500242B4B8DB01C
:105BC000DC661C672A4B07AC40C90138009301947E
:105BD0000523FDF77FFE0798636805900293237BFA
:105BE000257A0393234B277C0340062B05D083079C
:105BF0002ED1214B02689A422AD106A902F01CFC40
:105C0000069B002B21D0012B0CD1002D0AD1002F97
:105C100008D1007821F07BFD0590059930001EF039
:105C200011FE12E005980BF08BFA0590237C002BF7
:105C300003D005980CF096FD0590039B029A009303
:105C400005992B003000FFF77FFF0C480DB0F0BD29
:105C500008F0F6F90A4B9842E8D1002D01D1002F47
:105C6000DBD005A90120FCF7FBFFDEE7AC09002033
:105C700054DE0200070080FFDC1403004CCA02005F
:105C8000800D030030B5104B89B003AC20C901383A
:105C9000009301940523FDF71DFE02A9039802F06D
:105CA000CBFB227C237B02990092039A0BF032FA01
:105CB000237A01000093280000236268FFF744FF65
:105CC000024809B030BDC04690DE02004CCA020056
:105CD0000022074B10B51A70064B02321A70064BA1
:105CE000064A1B68063B1360FFF79AFD10BDC046CD
:105CF000180900201609002014000020EC020020E2
:105D000010B5FFF7E5FF014810BDC0464CCA0200C0
:105D100010B5042901D8042A05D90A490A481EF0F9
:105D200077FDFAF754FA092B01D90849F6E705245B
:105D3000614341188A18137101229A40038C13435E
:105D4000038410BDC139030044DD0200D6390300CD
:105D5000F8B548680C000D6808F05AFA0600A0680B
:105D600008F056FA0700E06808F052FA3A0003001B
:105D700031002800FFF7CCFF0048F8BD4CCA0200F4
:105D800010B5042901D8042A05D9064906481EF091
:105D90003FFDFAF71CFA0523594340188018007993
:105DA00010BDC046C139030044DD0200F7B51B4FEA
:105DB000019038000DF036FD194E30000DF032FD27
:105DC000184D28000DF02EFD17480DF02BFD17483B
:105DD0000DF028FD16480DF025FD164C3800210069
:105DE0000DF044FD300021000DF040FD28002100A1
:105DF0000DF03CFD21000C480DF038FD21000B4852
:105E00000DF034FD21000A480DF030FD1EF0A1FD1B
:105E10000123019A08489377FEBDC046741E030013
:105E20007C1E03008C1E0300941E0300A41E0300AE
:105E30001C1E0300081603004CCA0200002313B501
:105E4000044A046A09050093890C8A58A16B1EF064
:105E50000BFE13BD2CDF0200F0B587B000931B785A
:105E600004000F0002927C2B05D18268525C002A4C
:105E700001D09A2A14D11A006B3A022A2DD8A568AB
:105E8000E8190378032B5ED104A966681EF0B8FEFA
:105E9000AB19984206D16760049920001EF014FEE9
:105EA00007B0F0BD0378032B4DD105A91EF0A8FE65
:105EB000009B1B786B2B04D1049B059A134304931E
:105EC000E6E76C2B03D1049B059A5340F7E76D2B53
:105ED000DED1059B049A1340F1E76E2B04D0022219
:105EE00019009143702966D1A368D81901930378EA
:105EF000032B28D1636804A903931EF081FE0600DA
:105F0000019B039A9B189E42C5D0B378B01C75784C
:105F1000032B18D105A91EF073FE0600372D15D1ED
:105F2000059A1F2A0FDC4149049B114199420ADB63
:105F3000C021090611418B4205DB93400493049A6A
:105F400053005340DCD5029D00224FE0392D08D18B
:105F5000059B1F2B01DD1F230593049B059A13410D
:105F6000ECE72F2D03D1049B059A9B18E6E7302D13
:105F700003D1049B059A9B1AE0E7312D09D10599BD
:105F80000498FAF741F90028DDD1059B049A5343A0
:105F9000D4E7332DD7D00599352D06D10029D2D09D
:105FA00004981CF019FF0490C9E70029CBD004988D
:105FB0001CF022FFF7E7752BC5D1A368D8198378A9
:105FC000032BC0D1457802301EF029FE2F2D01D1C0
:105FD000049060E7302D06D14042430004905840C1
:105FE00000D458E7AFE7C043F2E73200561CED0992
:105FF000FBD16368DB1B01930135DB09FCD1023265
:1060000052193900200021F0ADFF0400009B029AD4
:106010001B7831001A33037001301EF0A7FC701C8E
:106020002018019A29001EF0A1FC39E7FFFFFF3F6D
:10603000F0B597B00890C020002540230AAC80003E
:106040000F00160025706360A56022F067FF2561D0
:10605000E0606561A561E5612762E562A84218D14B
:10606000C349C4481EF0D4FB0023060013930D98C7
:1060700022F06EFF002E00D1E0E10023BA6B3968F8
:106080003000FFF75BFB38001CF069FF3000FAF7C7
:106090009EF8321E03D00422022E00D0033A0026BE
:1060A000B5490096920052582000B96B33001EF09B
:1060B000DBFC102022F025FF1021040021F0B2FEAD
:1060C0000AADAB68002B00D194E12A78002A00D0F9
:1060D00090E1013B0C32AB605343EA68A649D31808
:1060E000DA785D689200525802921A689B68120230
:1060F000120A0393029B05925B7806930F23069A7C
:1061000013400493002D01D1636803933023069A52
:106110001340102B27D0202B66D0002E00D042E158
:106120000123069A1A400992099A02992A405300BB
:10613000CB1880215B88490107931B0B1B038B4203
:1061400000D048E13B00079940331B780905090D51
:106150008B4200D026E1002A00D11EE138001CF05D
:106160006EFF0135E0E7002D0BD180213800029B46
:106170006A009A1849014030049BAB4205D80126B9
:106180009EE7002EF1D100269AE753881E0B3603B6
:106190008E4214D106781B0502321B0D9E4221D17E
:1061A00021000AA81EF09FFC0028ECD13B004033E0
:1061B0001B78062B00D035E17049714852E7049AEC
:1061C0006B1C9A4206D9039A059900920AA8029A72
:1061D0001EF04AFC029B6D005D1969880AA8FFF752
:1061E0002DFED0E70135C7E7002E0BD0029A6B00D9
:1061F0009B5A1B0B032B48D10121200021F07AFE72
:1062000000230370029B6E009E19049BAB4240D892
:10621000002380201E004001049A934269D3A368A2
:10622000039A981800230693A2686368D3189842CB
:106230006DD3029B1B781F2B01D02E2B00D1012682
:10624000029B597840230B4018004342434149B216
:106250005B421E40002900DA01260025039B0495BD
:10626000D0180795069B9D4258D1002E02D1079B5E
:10627000012B63D00499200021F0A8FE029B059A0F
:1062800003992000FFF7E8FD7DE7012D00D876E7B0
:106290008CE78021738849011A0B12038A4226D1A8
:1062A0003A0040321278DBB29A421CD1082A07D158
:1062B000B96CF86C06F004FA010020001EF0CAFB6D
:1062C000002D0AD1029B5B787F2B06D90E9B200004
:1062D000591C06930E911EF0F7FB38001CF0AFFE20
:1062E0000135023691E7002D00D148E75EE76B1CCF
:1062F00069E702995A008A185288110B09038142F2
:1063000003D1D2B2072A00D90126013384E7069BC4
:106310000121013306931EF04CFB85E7049A0378B4
:1063200001320492002B04D0079B01330793002312
:10633000049301211EF03DFB013593E7A268039B06
:10634000944663441D00069B9E4200D11BE72B78B8
:10635000002B07D1A3680122E91A200021F042FE98
:106360000136F0E7280001211EF023FB0500F7E7C6
:10637000103A030098DA02002CDF0200383A0300DA
:1063800060D90200012D00D1F9E601232A001A404C
:106390002ED0049A032A0DD008E721000AA81EF087
:1063A000A2FBDEE60135049B022BEBD10023012D7D
:1063B00000D1E4E6069A691ED20705D5029A9288B2
:1063C000120B012A00D16908012900D056E7002BE1
:1063D00000D1D8E652E7039A059900920AA86B1CEF
:1063E000029A1EF041FB07990AA8FFF727FD67E60E
:1063F0001300DFE72B78002B00D031E63B00403361
:106400001E78002E00D0D1E66368002B00D1CDE6C7
:106410002B692000591C1EF057FBA3686B62EB69C7
:10642000AB6224E6022B01D10949C6E60B3B0948C1
:106430000949012B00D815E6084913E638001CF07D
:106440008EFD089A13AB13CB13C2089817B0F0BD9A
:106450004A3A030048DC02007E3A0300E8320300B7
:10646000F7B5002806D13A4A3A493B481FF0A3F84D
:106470003A48FEBD0D68280007F0E2FD43680600BB
:10648000EF2B04D16D68280007F0DAFD0600002329
:10649000334AD9008858A84205D1521851682E486D
:1064A0001EF0BEFFE4E70133612BF2D12D4B2A4CE5
:1064B0009D4201D09E4202D12B492000F0E72B499A
:1064C00020001FF078F80021280007F0EBFD72682B
:1064D000274920001FF06FF8264B9E4228D1280044
:1064E00021F0CDFA1EF07FF90025061EC0D073689A
:1064F0009D42BDD2B268EB00D3181F68002F15D0A3
:106500005B681D49200001931FF055F800213800F9
:1065100007F0C8FD194920001FF04DF8002101982F
:1065200007F0C0FD164920001FF045F80135DEE7F1
:10653000144B9E4200D12E00B06B002898D08307E8
:1065400096D1114B02689A4200D091E7CAE7C04643
:10655000AE3A03002F380300B4EA02004CCA02002E
:10656000D0E10200B0000300253F0300413F0300DB
:10657000493F030020100300789B0300593F0300AC
:1065800007B00300C8CF020094D60200034B0448B2
:106590001B78002B00D103487047C04600BC0200A6
:1065A000AC090300A409030010B5DA2022F0A9FC0D
:1065B00000230370024B8C331860024810BDC046A4
:1065C000AC0900204CCA0200F0B507000E0015000F
:1065D000094C87B02000019320F018FD02AB1F701A
:1065E000019B102202A9200003960495059309F04F
:1065F00087FF07B0F0BDC04600BC0200F0B5784B85
:1066000099B08C331A680192002A02D1002019B087
:10661000F0BD00241C60019B1B78A342F6D001262C
:10662000019B704F02331093019B109DD233119345
:1066300002933B002341334211D01A2302991B1BC2
:10664000280003931EF096FBBB235B00984206DCF8
:106650003300A34032009F43039B9A409743029B21
:106660000134083B083502930D2CE2D10A2308932C
:1066700000230293029816F015FD089B12901391C7
:10668000013B089314AA39000198002B00D188E03F
:1066900000261EF03DFB109B0E93119B0D93524B59
:1066A0000F931A239B1B0B930E9B09960C930D9B28
:1066B0000A934D4B04930C9B4B4C07930B9B16ADCD
:1066C00005930A9B0693099B03933B00039A13418E
:1066D0000122134225D014AB0F9A1B882900D3182E
:1066E0002B8014AB5B88049A0798D3186B8014AB8B
:1066F0009B8814AAE318AB801EF06BFB011C029868
:1067000013F038FF002862D114AA290006981EF061
:1067100060FB8022029B1206991813F02BFF0028C1
:1067200055D1039B01330393069B083B0693059BBE
:10673000013B0593FA23DB00E418079BA4B208335E
:106740000793FA231B019C42BFD1FA22D200944640
:10675000099B033309930A9B183B0A930B9B033B4A
:106760000B930C9B18330C93049B63449BB20493D0
:10677000A342A0D10D9B0936483B0D930E9B483395
:106780000E930F9B63449BB20F931B2E89D11298DB
:106790001399164A164B14F035FF16F0D5FC0290EB
:1067A00068E71EF0B5FA040014AB04229B5E14AA3D
:1067B0000221525E14A90020095E1B011201090189
:1067C0000120FFF701FF200020F0ACFB1FE70122B2
:1067D000059B03999A4001238B4013439F43A0E7F5
:1067E000AC090020FFDFFF0730F800009A99999963
:1067F0009999B93FF0B5584C8BB00390A37F002B0B
:1068000005D1564956481EF003F8F9F7E0FC039805
:10681000FFF7CAFE0022534920001EF070F8FFF770
:10682000BFF800280BD050480BF03AFE002804D1E6
:106830004E480BF035FE0028F1D0FFF749FA202032
:1068400020F065FF00230700190007AA99540133BF
:106850000C2BFBD10224002325000293019306ABED
:1068600005AA04A9424820F080F80023220029004C
:10687000380020F074FC049B3E4A002593420CDB58
:1068800019000135C83108DBC821033589008B4266
:1068900003DC013DC82B00DC013D059B0024934235
:1068A0000CDB1A000134C83208DBC8220334920022
:1068B000934203DC013CC82B00DC013C0422029B18
:1068C000134205D1092322002900380020F047FC9B
:1068D0000023294E0093009A07ABD25C002A2AD0ED
:1068E000092372783178380020F039FC009B023699
:1068F000013300930C2BEED1174E390030001DF000
:10690000A1FF64200BF014FF029B01330293019B53
:106910000B2BA4DD194930001DF094FFFA208000F4
:106920000BF006FF0398FFF769FE0400FFF7D0F9AC
:1069300020000BB0F0BD3278AA42D7D17278A242C3
:10694000D4D10121009AD154019B2200013301933B
:1069500029000923C7E7C046180000201961030079
:10696000C4DB020045610300C0100300CC1003002B
:10697000A8000300E0FCFFFF01610300941703007F
:10698000002310B518001A001900FFF71DFE01487A
:1069900010BDC0464CCA020070B500210320FCF7B0
:1069A0005FF9084D0400686820F0BCFAA060A86890
:1069B00020F0B8FAE060E86820F0B4FA2061200026
:1069C00070BDC04600BC020070B548680C0007F0FE
:1069D0001FFC0500A06807F01BFC0600E06807F03C
:1069E00017FC3200030029000120FFF7EDFD0148EC
:1069F00070BDC0464CCA0200F8B50B4E3378002B70
:106A000010D10A4D2C78E4B2002C0BD1012700687C
:106A10002F7003685B689847054A2C7013683770BD
:106A2000DB191360F8BDC046190900201A090020BF
:106A3000F4020020F0B53E4B87B01B780400002B19
:106A400001D1FFF7D7FE201DFFF7D6FF394D2800F3
:106A500012F05CFA0021606822F073FF344E04905B
:106A6000736800216068059322F078FFB368002105
:106A700002906068039322F07EFFF368C01A14F05E
:106A80002BFD041C280023F064FF061C280023F0C3
:106A900057FF051C301C16F0F7FE071C301C16F0C3
:106AA0006FFD0190281C16F0EFFE061C281C16F046
:106AB00067FD029B039A051C981A14F00DFD291C12
:106AC00014F016FA311C051C201C14F011FA011CDC
:106AD000281C13F08BFE80231B06059AC518049B07
:106AE000981A14F0F9FC019914F002FA211C061C02
:106AF000381C14F0FDF9011C301C13F077FE8023C4
:106B00001B06C018291C17F02FF80B4914F0F0F9D8
:106B100016F0C8FA094A0A4B15F084F816F04CFA38
:106B2000002801DA6930FF3020F0FCF907B0F0BD31
:106B300000BC0200B40600200000B443EA2E445416
:106B4000FB21194010B504000430FFF755FF002168
:106B5000606822F010FF034BDB68C01A20F0E2F9F6
:106B600010BDC04600BC020010B504000430FFF7A1
:106B700043FF0021606822F0E4FE034B5B68C01A0B
:106B800020F0D0F910BDC04600BC020010B50400D2
:106B90000430FFF731FF0021606822F0DFFE034B75
:106BA0009B68C01A20F0BEF910BDC04600BC0200B0
:106BB00070B5002105000320FCF752F80400281DE1
:106BC000FFF71AFF0021686822F0BBFE0C4E7368C5
:106BD000C01A20F0A7F9A0600021686822F0BEFE6C
:106BE000B368C01A20F09EF9E0600021686822F0C6
:106BF000C2FEF368C01A20F095F92061200070BD34
:106C000000BC0200F0B54C4B89B08C331B6802937A
:106C1000002B4CD049480430FFF7EEFE484C0021D1
:106C2000200022F08EFE002103112000039322F0A9
:106C300095FE002103112000019322F09CFE031118
:106C40000493029B039A1B785242002B31D1019B83
:106C50000321D31A9C46494208006546093801249D
:106C6000032664420319029FDB00FB186A461F00DB
:106C700092896A373A806A46928870337A806A4687
:106C8000128A013EBA80049F67437F191F80013436
:106C9000002EE7D1019B0330ED188142DFD1039B29
:106CA00009319C441829D7D10123029A137009B0E5
:106CB000F0BD019BD71A03225242110005970939F2
:106CC000012003264042049C059B4443E31806939D
:106CD000029C0B18DB00E3181C007034079400259D
:106CE000645FA446069C644515DD6A24A4466D468F
:106CF0009C446446AD8925806C24A4466D469C4422
:106D00006446AD886E3325806C46248A1C806C46B0
:106D1000079B248B1C80013E0130002ED3D10598A7
:106D2000019B0331C31805938A42C9D1039B0932E1
:106D3000FF18182AC1D1BAE7AC09002034E60200D6
:106D4000F0060020F0B5050089B002AFB96016006A
:106D50003B6004F057FAAB687B611423F81821F00C
:106D600075F914237860F81821F070F9032358435B
:106D70007B68C0188300FB602C2B29D86B46F86811
:106D80002A30C008C0001B1A9D46002302ACFB60DD
:106D9000AA687B6929009B1A63607B682000A36155
:106DA0003B680093BA6833000CF0B4FB1A4E002124
:106DB0007368200063616B687360FDF7BBFA6369F9
:106DC000B860736000280AD0022819D0134D08E07B
:106DD000F8681C3022F0A2F8041ED9D1CEE7E3688F
:106DE0001D68FB68002B07D00023BB60200022F049
:106DF000AFF8BB68002B0BD12800BD4607B0F0BD33
:106E00007B6805339B00E3185D68FB68002BEDD1C0
:106E10002800F9F7DCF9C046AC0900204CCA020092
:106E20000122030030B5134085B004004510002B4B
:106E300014D128491D00884210D0274988420DD01E
:106E4000264B1500984209D00323034009D1244A58
:106E50000168914205D120F0A2F80500280005B094
:106E600030BD204A25002240062A05D0002B08D13B
:106E70001D4B22689A4204D101A9200001F0DCFADE
:106E8000EBE7200007F0DCF8184B984207D1FF230E
:106E9000DB05E0180323984314F0FEFADDE7144BFA
:106EA000984206D101AA694620001DF0A1F9019D72
:106EB000D4E7104B984205D101AA694620001EF084
:106EC00015FDF4E7022201A920001FF0FCFE0028B6
:106ED000C4D0ECE74CCA0200A4090300AC090300CB
:106EE000E81F0300070080FFDC140300381B0300C9
:106EF00000CE020060EC0200F7B506000F00009221
:106F00000193041E00D044683800431E98412018A5
:106F10000430800021F0F5FF0C4B050003600C4BA2
:106F20005B684360009B8360019BC360002E05D0BB
:106F30003100A2000831103024F0D3FA002F02D023
:106F40000434A40067512800FEBDC04678E6020064
:106F5000AC09002070B5060010200D00140021F0CF
:106F6000D0FF034B466085600360C46070BDC046BF
:106F70003CE602000022104B10491A600300123355
:106F8000FF3341185A701A7004338B42FAD1010052
:106F90000300002209310833FF311A709A705A70C9
:106FA000DA7004339942F8D1C3237F229B00C25484
:106FB000034A044B1A607047F802002011030000D6
:106FC0005361030050000020F0B500267E243300FA
:106FD00031009A008218FF32577C7F2F44D0927C78
:106FE000B618F6B25A1CEF2E2BD9C1267D25B60055
:106FF00086193700AC46D2B2944516DA9200821850
:10700000FF3251749174D17411757D220233DBB259
:107010009A4211DA00269A008218FF325474917451
:10702000D17411750133DBB2D3E73D68043FBD6015
:1070300001256D42AC44DFE73568013A7560043ED6
:10704000E6E77D2FEED8094DEF5D01252F42E9D00F
:10705000D3B2C1227D26920082189E42DADB1568E7
:10706000013E5560043AF8E7F0BDC04636620300C1
:1070700070B5012240240F49531EDBB29B00C31898
:10708000FF335D7C7F2D13D04D5D25420DD05D7D9E
:107090007F2D0AD04D5D7F2D07D9DD7D002D04D0D9
:1070A0006EB2002E01DB0135DD740132D2B2E3E7AE
:1070B00070BDC046E56103000300F7B500214B4AEF
:1070C0001333FF338218197004339342FBD1FC232E
:1070D00000249C462200844453B2002B04DA444A24
:1070E000444B00201A6008E063461F69BC4205D388
:1070F0007F234432920013540120FEBD6346DE68B4
:10710000355D602D01D9203DEDB2611CC9B28F42C1
:107110004FD0735C602B01D9203BDBB2232D4BD1C8
:10712000303B092B01D9344ADAE70234E1B28F420D
:1071300004D8FF2BF7D843700C00CDE7745C250012
:10714000303D092DF5D80A256B430131303BE3185A
:10715000C9B2ECE70136512E2FD10023274C1F5D19
:10716000DEB22A2F0CD1264FFF5CAF4208D193002C
:10717000C318FF335E74447801321C75D2B2DBE76A
:107180000133512BEBD11F4C493B08342678AE42DA
:1071900007D0013C002B01D11B4AA1E7013BDBB228
:1071A000F4E7002BF8D014004334A4000419A370B2
:1071B000C2E7232DB7D000230026F7B20197104F66
:1071C000F75DAF42C6D10D4FF75D2A2FC2D09F4267
:1071D000C0D1694693000979C318FF3359744178C7
:1071E000013202341975D2B2E1B2A5E712030000F0
:1071F00056610300500000206861030075630300BE
:1072000024630300C66303007661030010B51130E8
:10721000084A0949FF3003787F2B00D110BD0224B2
:107220000457002C03DCCB5C43700430F3E7D35CE1
:10723000FAE7C046D4620300846203008446002358
:10724000F0B585B09F0067443800FF30417C7F294E
:1072500001D105B0F0BD0224544A525C224202D151
:107260000133DBB2EEE70124224246D11A190C1990
:10727000E4B200944E4C7D2564186478D2B2019437
:10728000C47C007D02940390C1208000604404000F
:10729000954228DA6C46920024786244FF32547496
:1072A0006C4624798D1C94746C46247AEDB2D474A7
:1072B0006C46247B14753E4C9A1C61183C00FF34CC
:1072C0008E78217DE77C00917D21D2B291420FDA48
:1072D00092006244FF3255749674D77469460978F7
:1072E00003331175BDE72668013D6660043CCFE7B6
:1072F0000468013944600438E8E71A000132D2B268
:107300001000644644308000005D0028F6D05A1C0E
:107310007F2809D00825254C245C2C4201D0D3B20B
:1073200090E724380128FAD93C00481CC0B20090EC
:107330001F48FF34401840787D260190E07CD2B28F
:107340000290207D0390C120800060440500964299
:1073500022DA6D4692002D786244FF3255746D46F4
:107360002D79134E95746D462D7AD5746D462D7B0F
:1073700015758D1C71188F78217D9A1C00917D21C7
:10738000E67CD2B2EDB291420BDA92006244FF3257
:1073900055749774D674A1E72F68013E6F60043D61
:1073A000D5E70468013944600438ECE7E56103007F
:1073B00084620300F7B500218B00C3181A00FF3266
:1073C000547C9C46002C02D10131CBB24AE07F2C88
:1073D00000D129E11026954B1D5D4B1C35422BD069
:1073E000AD06ED0F2C00D67C177DC1227D2514340F
:1073F00092000194DBB282189D4218DA6A469B0023
:107400001279C318FF335A740022DE749A741F7500
:107410006246FF32547C4B1C352C00D0C6E0517BB9
:10742000834C615C490700D492E0102187E0146826
:10743000013D5460043ADFE74E2C1ED118210D2582
:10744000D47C5574167DC1229200DBB2821870354F
:107450009D420DDA9A008218FF3251740021D474D3
:10746000917416751900A7E71B21E8E71C21E6E7D0
:107470001768013D5760043AEAE74F2CF4D0502CCE
:10748000F4D06DB2002D2CDAD57C002D29D0DBB2E2
:107490001D004435AD002D5C002D22D18E1CF5B2AF
:1074A0000195AD004519FF356F7C7F2F19D05F4ED8
:1074B000F75D7F2F15D9EF7C002F12D0C1227D21DF
:1074C00092008218019C8C4206DD1F226A74002201
:1074D000AA74EA742A75C5E7146801395460043A3D
:1074E000F0E74B1C172C2CD1557B4C1EE4B2452DDC
:1074F0001CD12A235373230043339B001B5C4B4A4C
:10750000D55C4B1C7F2D23D90134E4B2A4000419AF
:10751000FF34617C00297FD0525C7F2A18D9E27C3D
:10752000002A15D162461E21FF3208E0392D01D113
:107530002C23DFE73D49495D7F2909D91221517488
:1075400006E0182C08D1517B384C615C7F2901D8AA
:10755000DBB287E71321F2E7202C04D1517B3C29D1
:10756000F6D12621EBE7482C15D1547D7F2C02D192
:107570004B24547403E02D4D2C5DA406F8D5547CA7
:107580002A4D2D5DED0700D442E7557B202D3CD1DF
:107590000C3C5474DCE73C2CF1D1517D7F29D7D0D1
:1075A000224C615C8906D3D43F21C8E72A2C17D12D
:1075B000D17C147DC1227D259200DBB282189D42D0
:1075C00009DA2B259A008218FF3255740025D174F0
:1075D0009574147546E71668013D5660043AEEE767
:1075E0002C2C12D1D17C147DC1227D259200DBB2DE
:1075F00082189D4204DA9A008218FF322D25E4E7B2
:107600001668013D5660043AF3E7452C02D0392C48
:1076100000D0D9E60C006EE7617D7F2998D0525CDE
:107620007F2A00D97EE793E7F7BDC046E5610300F6
:1076300036620300F7B505000022130044339B00B7
:107640005B5D7F2B41D05E4CE35CDB075FD51300B5
:10765000511EC9B2443189005A4F6918013BDBB24F
:10766000002B34D1022799006918FF314A7C7F2A08
:1076700000D1A4E053488446805C44B2002C5BDA1D
:1076800041265A1CD2B290002818FF30447C019049
:1076900000967F2C02D06646365D009666464020F6
:1076A000365D064236D1123C012C0CD860460233BE
:1076B000DBB244339B005B5DC35C4020034202D0DD
:1076C0008B7C013B8B741300CDE70023CAE708785D
:1076D0007F2803D0385C04397F28BFD99900691806
:1076E000FF31487C7F280ED02027265C3E4204D004
:1076F000344E305C0426304205D0887C4608B446BF
:107700000130604488740133DBB29342E6D1013228
:10771000D2B292E7009B5B0706D4009BDB07D2D571
:107720008B7CD8081B1ACDE7019B9B7B591C9B08BF
:10773000CB1801998B73C6E7214CA25C0824224226
:1077400010D00133DAB29300EB18FF33597C7F2954
:10775000B9D06046415C3942B5D006219974052103
:107760009973B0E738421DD018000130C0B2020052
:1077700044329200525D002AF7D001337F2A01D1B2
:10778000DAB2A0E70F4CA25C3A42F9D08000281888
:10779000FF30827C5208013282748A7C52080132A6
:1077A0008A74EDE71020024207D060464A7B825C73
:1077B0003A4202D08A7C023A8A740133E0E7F7BD8C
:1077C00036620300E561030070B50400FFF7D2FBE9
:1077D0002000FFF771FC23000022FC330100DA6077
:1077E0001A61904226D02500224E11353368FF35AC
:1077F000934203D0290020480AF088FC2000FFF7BC
:10780000D9FD2000FFF734FC2000FFF7FFFC20002B
:10781000FFF710FF2000FFF711FDC4222B0092009C
:10782000A1181A78502A07D97F2A08D00021134AB4
:10783000134B1A60080070BD04338B42F1D13368DA
:10784000002B02D00F481AF039FB2000FFF7BCFBD9
:107850003368002B03D029000B480AF057FC2000A6
:107860001DF09FFB064B0949186823F0B1FF414208
:107870004141DFE7E40200208D6103009C610300C9
:1078800050000020C2610300D26103005361030075
:1078900073B516000D4A0B0054681568012804D909
:1078A0004C682500022800D08D6801A9186800F0F6
:1078B000C3FD01009320019A0023400008F09EFDC3
:1078C0002B003100220008F03BF876BDAC09002007
:1078D000F7B5CC1CA400070020000E00019221F097
:1078E00010FB22000500054B4760866003600C3AE0
:1078F00001990C3023F0F5FD2800FEBD08E70200D9
:10790000032230B502400121002A04D1084C03684B
:107910000D00A3420AD00B0003401D1E06D1002A11
:1079200004D1036803481B1A5D425D41280030BD45
:10793000B4090300E81F030010B50400FFF7E0FFDF
:10794000012300280AD102332340022B05D1054828
:107950000440063C601E8441E0B203000120184050
:1079600010BDC046070080FF10B51FF096F903490F
:1079700002000348FDF772FEF8F729FCCF6303000D
:10798000CCDC020010B50400102021F0BAFA044B40
:1079900084600360034B43600023C36010BDC04696
:1079A00028010300C1530200F7B504000E00019343
:1079B00001208B180A0000210093009B934212D8EB
:1079C0002725002900D0053D224F2A00390020003C
:1079D0001DF0F1FD009B9E4214D32A0039002000C7
:1079E0001DF0E9FDF7BD1378272B08D0223B5D423F
:1079F0006B41DBB20132002BDFD02725E4E7002307
:107A00000100F7E73278954205D12A00124920009B
:107A10001DF0D1FD1AE011495C2A14D01F2A09D9A2
:107A20007F2A15D0019B002B02D053B2002B07DB1D
:107A30003900ECE70A490A2A05D00A490D2A02D082
:107A4000092A05D1084920001DF0EAFC0136C1E7EA
:107A50000649DCE799670300986703009C67030009
:107A60009F670300A2670300A5670300A8670300E0
:107A7000194B70B506000D0098420ED14968A868F0
:107A800004F0ECFD041E08D0280020F0F6F9E00018
:107A9000002306242B60204370BD102021F031FA12
:107AA0006968040081600660A86804F0B9FD6B682D
:107AB0006060591C2B68994209D1AB68E3600023D0
:107AC000E268A16820005354AB602B60E4E7A8682B
:107AD00021F02DFAE060F2E7DC14030070B5040039
:107AE0000D00002A05D004F0EBFDC300062018436A
:107AF00070BD04F0B3FD0028F7D12A002100024830
:107B00001DF02CFBF4E7C046DC14030010B50A009E
:107B1000010002481DF022FB10BDC04690E70200A4
:107B2000094B10B50340062B01D1C00810BD8307D7
:107B300008D1064B02689A4204D18168C06804F0FB
:107B4000BFFDF3E7FFF710FF070080FFDC14030021
:107B5000064B10B50340062B03D1C0081EF081FE72
:107B600010BD8368C0680B60FAE7C046070080FF5D
:107B7000F0B50F00002689B0110005001C00380088
:107B8000009603233200FBF773FE0E20B7420FD09E
:107B9000012F0FD102AA102104A80BF027FA2168A7
:107BA00002A8320006F064FA04A92800FFF760FF7B
:107BB00009B0F0BD206883071BD1134B02689A42BD
:107BC00017D104A9FFF7C4FF104B0600206803403B
:107BD000062B0CD1C0081EF035FE04001020049FB7
:107BE00021F08FF905608760C6604460E0E7446873
:107BF000F4E704A9012206F0C5FC002205990498C7
:107C0000FFF76CFFD4E7C04690E70200070080FF53
:107C1000F0B58BB0049008680D000692079306F04B
:107C20000FFA0600686806F00BFA864202D0686810
:107C3000FFF79AFE08A92868FFF78AFF040009A940
:107C40006868FFF785FF089A0590A3180393049BC3
:107C50002700022B19D9AB681E498B4206D001219F
:107C60003000009121000BF08DFB0700049B032BDB
:107C70000BD0EB68174A934207D0012221000092F3
:107C80003000089A0BF07EFB0390039B059AD91BEA
:107C9000069B38000093099B1DF041FA002809D18A
:107CA000079B0138002B0FD00B490C481CF0B0FD8E
:107CB000F8F78DFA0A4B9E4208D10100200020F00F
:107CC000A7FA4400012020430BB0F0BD041B640060
:107CD000F8E7C0464CCA0200C167030044DD020059
:107CE000DC140300F0B58DB00400039106F0A8F990
:107CF00004A906002000FFF72BFF019003988307DB
:107D00001ED10368314A934217D106AA05A91CF077
:107D10006FFA00242500059B9C4220D329000025F2
:107D200008A820F096F80A9C059B9D4236D308A926
:107D30003000FFF79DFE0DB0F0BD254A934208D0FC
:107D400023480022C36801210293029C03ABA04791
:107D5000039006AA05A903981DF0C8FDD9E7069B64
:107D6000A700D85906F06CF9864205D019491A487F
:107D70001CF04EFDF8F72BFA002C01D0049BED18F7
:107D8000069BD859154B0340062B05D1C0081EF0A1
:107D90005EFD2D180134BEE78068FAE7002D06D09D
:107DA0002000049A019923F09CFB049BE418069A96
:107DB000AB00985807A9FFF7CBFE079A01002000F7
:107DC00023F08FFB079B0135E418ADE700CE0200DE
:107DD00060EC0200D5670300CCDC0200070080FFE6
:107DE000F0B5070087B008680D0006F029F904A96E
:107DF00006002868FFF7ACFE05A904006868FFF7D5
:107E0000A7FE03902000022F07D901230093AB683F
:107E1000049A210030000BF0B5FA059A041B049B6C
:107E2000A418064D9C4205D8039923F04BFB00286B
:107E300000D1034D280007B0F0BDC046A4090300DF
:107E4000AC09030073B50D00060069462868FFF70A
:107E50007FFE01A904006868FFF77AFE0100022E88
:107E600002D9084807F0B6FD019A0098064D8242F3
:107E700006D8801A201823F025FB002800D1034DD6
:107E8000280076BDAF670300A4090300AC09030016
:107E9000F0B58FB0079010680C00160006F0D0F80F
:107EA0000690012C31D0706806F0CAF8069B834218
:107EB00002D07068FFF758FD0DA97068FFF748FE03
:107EC0000D9B089009930DA93068FFF741FE0D9BAB
:107ED0000B900493079B012B1CD1049B5D1E012377
:107EE0005B420A9300242700049B03940593059B9F
:107EF000002B13D1039B002B23D1214B069A0E207C
:107F00009A4200D01F480FB0F0BD072309931E4BC3
:107F10000893D8E7012300250A93E3E70B9B09990F
:107F20005A190123089800931DF0F9F8002816D17A
:107F3000039B002B19D1079B002B09D12F00049B19
:107F40005C1E049B0134E21B934212D13068DAE7D5
:107F5000079B2C00012B0AD001232F0003930A9BBF
:107F6000ED18059B013B0593C1E72C00F7E7039F44
:107F7000E7E70B9B0698D9191DF0F0F8C3E7C04658
:107F8000DC14030080E702003E680300F0B589B00E
:107F9000049008680D0006F053F80700686806F0C2
:107FA0004FF8874202D06868FFF7DEFC06A9286810
:107FB000FFF7CEFD060007A96868FFF7C9FD069A1E
:107FC0000590B3180393049B3400022B19D9AB68B6
:107FD0001D498B4206D001213800009131000BF081
:107FE000D1F90400049B032B0BD0EB68164A934293
:107FF00007D00122310000923800069A0BF0C2F936
:108000000390079B0025002B12D1039B2000191B16
:1080100020F00DF9013045000120284309B0F0BDE2
:108020000599200023F04EFA002808D101353400CC
:10803000079A039BA618B342F2D26D00ECE720002A
:1080400020F0DDF80600F2E74CCA0200F0B58BB074
:108050000E000700039205F0F3FF0500300005F065
:10806000EFFF854202D03000FFF77EFC05A9380003
:10807000FFF76EFD06A904003000FFF769FD069BBF
:108080000200002B05D11A491A481CF0C1FBF8F771
:108090009EF819498D4227D10E2107910891099127
:1080A0000399002922DD0797039920000091059983
:1080B0001DF035F8002811D0071B3A0021002800D8
:1080C0001DF04CF8059B0699DA1B521A7918079097
:1080D0006118280008961DF041F8099007A90320AF
:1080E000FAF7BEFD0BB0F0BD0449D6E70997DBE710
:1080F0001A68030044DD0200DC14030080E702007C
:1081000010B5010001481DF03AF910BD4F82020080
:1081100010B5010001481DF032F910BD6182020066
:10812000F7B50600080001A9FFF712FD019B050045
:10813000002B01D11348FEBD134B04009E4207D112
:108140000027019A631B9A4211D8002F07D1F1E74B
:108150000E4B9E42F4D0019A631B9A4201D80C4800
:10816000E9E72078B04701340028F4D1E2E720782D
:108170000CF010FA002803D02078B047071ED9D0A1
:108180000134DEE7A4090300FD45010015460100A6
:10819000AC09030010B501000148FFF7C1FF10BD95
:1081A0007D45010010B501000148FFF7B9FF10BD82
:1081B0009545010010B501000148FFF7B1FF10BD62
:1081C000AD45010010B501000148FFF7A9FF10BD42
:1081D000FD45010010B501000148FFF7A1FF10BDEA
:1081E00015460100F0B585B006000C00170005F03B
:1081F00027FF694605003000FFF7AAFC0600042FA0
:1082000023D1A30716D1124B22689A4212D101AA98
:10821000210000980CF020FB002802D10D4807F047
:10822000D9FB0199029A2800521A71181CF096FF86
:1082300005B0F0BD002322000099280006F0C0F828
:10824000335C01205B001843F2E70020F0E7C046F2
:10825000EC0003000535030070B51D008AB000294D
:1082600068D01868344C03002340062B05D08307E0
:108270001FD1324B02689A421BD10239012953D8CF
:1082800006A9FFF765FC060028680440062C0ED1FD
:10829000C0081EF0D7FA04001020069D20F031FE21
:1082A000274B85600360C66044600AB070BD4468B7
:1082B000F2E7012938D80122104210D044102100E1
:1082C00006A81FF0C6FD089B22000021180001939C
:1082D00023F022F906A91A48FFF7CAFBE5E703A92C
:1082E0001EF0F1FC002805D0049A039914481CF0F4
:1082F00035FFDAE7286806F0A5F81021002800D03D
:10830000411006A81FF08EFD286806F0B7FD040096
:10831000200006F0FFFD0028DCD005F079FFC1B297
:1083200006A81FF00AFEF3E7064907481CF070FA9A
:10833000F7F74DFF0548B8E7070080FFDC1403009E
:1083400090E70200FB630300CCDC020080E7020040
:1083500073B50400080001A91600FFF7F9FB05003A
:10836000042E06D10300019A074920001DF023F9CD
:1083700073BD064920001DF053F80123019A29001E
:108380002000FFF711FBF3E72A68030040790300A0
:10839000F7B502001C4B05000C001A401E00062A0F
:1083A00019D10B40062B04D1441A60426041C0B27F
:1083B00010E0C0081EF046FA07002640062E0CD139
:1083C000E0081EF03FFA002F09D0002807D08742AE
:1083D00005D00020FEBD4768EFE76068F3E7694617
:1083E0002800FFF7B5FB01A905002000FFF7B0FB4F
:1083F000009A019B01009A42EBD1280023F062F819
:1084000044426041D3E7C046070080FF084B07B5F0
:108410000340062B08D0830704D10268054B9269FC
:108420009A4201D0FFF7A0FA01A9FFF791FB0EBD18
:10843000070080FFF18900000A4B13B503400C00D0
:10844000062B08D0830704D10268074B92699A4231
:1084500001D0FFF789FA01A9FFF77AFB019B23609E
:1084600016BDC046070080FFF1890000F0B59BB043
:108470000B900C00079210210EAA12A809930AF083
:10848000B5FD079B9C4208D30B9A12AB13CB13C2CA
:108490001B6813600B981BB0F0BD21787D2914D1A7
:1084A000631C0593079B621C934208D961787D2960
:1084B00005D112A81FF041FD059C0134E1E7B54943
:1084C000B5481CF0A5F9F7F782FE7B2904D012A865
:1084D0001FF033FD0594EFE7079B651CAB4243D9C2
:1084E00061787B2904D112A81FF027FD0595E3E7E9
:1084F0002B007D2903D0212901D03A291FD1002545
:108500002E001A78212A23D00022049200211A7802
:1085100005913A2A31D15A1C5B7805927D2B30D0D7
:108520001300012207998B421ED219787B291FD193
:1085300001320133F6E7079A01339A4214D01A78D0
:108540007D2A03D0212A01D03A2AF4D11E00D8E78F
:1085500007995A1C914209D95A780492723A012A11
:1085600004D802339942D1D88C49A9E78C49A7E7AE
:108570007D29DED1013A002ADBD1059A05930692C6
:1085800005E0079B059A9342EED900230693059BCD
:108590001B787D2B01D0834992E7002D45D0002325
:1085A000287816930CF002F82C00002822D0099BA2
:1085B0001B680893002B01DD7B4981E716AA310077
:1085C00028001CF094FD209A169B013A04009A4260
:1085D00002D87649764874E7219A01339B009F5868
:1085E0000122099B52421A60B4422ED2714807F010
:1085F000F1F90134B44204D223782E2B01D05B2B45
:10860000F7D1611B01222800FFF768FA002205005C
:108610000100229803F098FA002804D12900664846
:108620001CF0EFF84FE74768DEE7099B1B68002B5B
:1086300001DA624944E7209A013A9342C9D20133F0
:1086400021999A005758099A1360069B002B16D15E
:10865000049B002B58D010AA102116A80AF0C6FCC3
:10866000049A3900733A531E9A4110A8D2B205F009
:10867000FFFC16A95248FFF7FBF9070002E0049B34
:10868000002BE8D101235B420D931093069B002B36
:1086900000D1B6E002F0B6FD229B059A0293219B21
:1086A00006990193209B16A80093099BFFF7DEFE15
:1086B00016A81FF031FC0026179B0400C3180A936C
:1086C00003780493B34213D03E4D1900280023F0E1
:1086D00071F8B04200D06FE16678002E17D03100FB
:1086E000280023F067F8002800D067E10600049016
:1086F000237808932B2B0CD02D2B48D00425202B2E
:1087000008D00025089506E073230493A3E7049698
:10871000EEE7022501342378232B02D1133B1D43BE
:1087200001342378302B07D1049B002B01D13D333A
:108730000493002E00D130360DAA0A9920001CF0B7
:10874000D6FC037806902C2B04D10C3B1D43030070
:1087500001330693069B1B782E2B06D1069810AA90
:1087600001300A991CF0C3FC0690069B1C78002C73
:1087700007D02100144823F01DF8002800D022E182
:108780000400069B1B78002B22D0104998E6002598
:10879000C0E7C046F864030044DD02003965030009
:1087A000206503005165030075650300BF65030084
:1087B0009CD90200D8650300D8D90200F5650300F2
:1087C000DC1403003F6603004466030054660300A4
:1087D00016A81FF052FB049B002B08D13800FFF7AE
:1087E000ABF83C230493002801D002330493002EFD
:1087F00000D12036089B002B0CD0732C06D1744975
:108800005EE6069D2C002E000895E7E7632C01D15B
:10881000704955E6049B3D2B1FD05E2B1FD03C2B8F
:1088200001D13B3B1D433800FFF76AF800282DD0EB
:10883000632C50D026D8472C13D8452C26D2002C98
:1088400040D0252C22D038001EF027FA2200030049
:1088500061496248FCF702FF35E64023E2E78023E6
:10886000E0E7582C53D0622CEDD1002303930D9BED
:108870000222029361230196009539000EA801F0AF
:1088800009F819E6672C17D8652C1BD33800FFF7B9
:1088900053F800286CD0002C56D06E2C54D0472CA6
:1088A0003FD8452C41D2252C50D038001EF0F5F988
:1088B000220003004A49CCE76F2C1AD0782C26D02E
:1088C0006E2CC0D1002303930D9B0196029300955B
:1088D00061230A22D1E7380005F09AFC0D9B16A906
:1088E0000870012201932B0000960EA800F076FF7D
:1088F000E2E5EB0602D580239B001D430023039392
:108900000D9B01960293009561230822B5E7002292
:10891000230003920D9A173B0292019600951022B4
:10892000ABE72300653B022BBFD8380005F0D4FC31
:10893000109B220002930D9B011C01932B000096BB
:108940000EA81CF0F0FDB7E56724EEE738008024A0
:1089500005F0C2FC234912F0CBFA109B640002938D
:108960000D9B2C430193011C009623006622E7E730
:10897000049B3D2B01D11C49A2E5002C01D0732C96
:1089800013D116A93800FFF757FD109B0100169A66
:10899000002B00DA1092109B9A4200D916930D9B7F
:1089A00000960193169A2B009FE738001EF075F988
:1089B000220003000D494CE7013499E633000234EC
:1089C000049E049394E6069B01330693D9E6C046C1
:1089D0006D66030099660300CC66030044DD020067
:1089E000FD6603000000C8423167030066670300AC
:1089F000F0B5A1B004000D000D920A2800D0E6E108
:108A0000073C0692144038D11368BD4A93422ED1D8
:108A10000FAA10A906981BF0EBFB0694109B11A956
:108A200008930F9B28000993FFF792F800230A9000
:108A30000C93AB0706D1B34A2B689B1A5942594194
:108A4000CBB20C9314AA102118A80AF0CFFA119AED
:108A5000002794460A9B0A9C63440593059BA34206
:108A600012D8089BBB4200D1A7E1A749B1E0A74AB1
:108A7000934202D10F941094D0E70DAB0F930123D2
:108A8000109300230693C9E72178252904D018A85C
:108A90001FF053FA0134E1E7059B661CB34205D889
:108AA0009B499C481BF0B4FEF7F791FB61782529A0
:108AB00004D118A81FF041FA3400EBE7002528295B
:108AC0000ED1A01C06003378292B1CD1311A0122AB
:108AD000FFF704F801000698FCF7B4FC0500013626
:108AE0000023340040220026302104200B93203341
:108AF0000793059BA34219D923782D2B0AD12C3B30
:108B00001E430134F5E7059BB34201D88249C8E70B
:108B10000136D8E72B2B01D1293BF1E7202B01D1DE
:108B20000643EEE7232B49D0302B44D00023129389
:108B3000059BA34245D801235B421393059BA342A7
:108B4000AED923782E2B15D1059B601C8342A7D963
:108B500063782A2B4FD1089A3B00BA4238D9099A38
:108B60009B00985805F054FB013713900234059B85
:108B7000A34295D9002D07D1089A3B00BA4227D9C4
:108B8000099A9B009D5801372278672A5DD8652A8B
:108B900000D3D1E0582A75D035D81300453B022BBD
:108BA00000D8C9E00A9B5D49E41A009413005948B3
:108BB000FCF754FD78E716430791A2E710230B93C7
:108BC0009FE723782A2B0FD1089A3B00BA4202D89C
:108BD0005349544866E7099A9B00985805F018FBDA
:108BE000013712900134A6E7200012AA05991CF063
:108BF0007EFA04009FE7002313AA059913931CF043
:108C000076FA0400B3E7632A49D0642ACAD1032262
:108C10002B001340022B0AD1434B2B40062B06D0CE
:108C2000FF23DB05E818904307F038FA0500139B93
:108C30000A220393129B00960293079B01936123E0
:108C4000290014A800F026FE24E7732A16D8722AF9
:108C500000D381E0692ADAD06F2AA3D10B9B002BC5
:108C600002D084239B001E43139B00960393129B08
:108C700008220293079B01936123E1E7752AC6D07E
:108C8000782A8FD11300139A173B0392129A0292FB
:108C9000079A01920B9A164300961022D0E7224BB6
:108CA0002B40062B05D0AB0716D1204B2A689A42E1
:108CB00012D11CA92800FFF7BFFB1C9A0100012A52
:108CC00001D01B4985E7129B0193202300933300B9
:108CD00014A800F083FDDDE62800FEF711FE002851
:108CE0000BD0280005F094FA129B1CA90870019380
:108CF0002023012200933300EAE70E4969E7C046CA
:108D000000CE020090E70200C364030094D6020084
:108D10001564030044DD0200276403008E64030031
:108D20003D640300CCDC0200070080FFDC1403007C
:108D3000646403007D640300280005F0CDFA139BF2
:108D400022780293129B011C0193079B14A80093A5
:108D500033001CF0E8FB9DE616AA10211CA80AF0BF
:108D600045F923781A00723A50425041C2B2722B30
:108D700009D00C9B002B06D0AB0704D1544B2968BB
:108D8000994200D10422290016A805F071F9139A1E
:108D90001D9B002A00DA1393139A9A4200D91A00F5
:108DA000129B1E990193202314A80093330000F016
:108DB00015FD1CA81FF061F86CE60C9B4448002BC5
:108DC00000D1444818A9FEF753FE050019E0080039
:108DD00005F036F916A906002800FEF7B9FE0700CF
:108DE000072C22D118A90D9805F050FA0025A842A9
:108DF00007D01899A94207DC364B0E359E4200D0A9
:108E0000354D280021B0F0BD169B1CA859431FF01A
:108E100020F81E9B169A059300930121189B380099
:108E20001FF02EFA1CA93000CDE70D9805F008F9C7
:108E300086420FD11CA90D98FEF78AFE1C9D059055
:108E40001D2C16D8192C3AD2052C21D0122C1FD04B
:108E50000025D6E71E4B00259E42D2D101221CA937
:108E60000D981DF030FFA842CBD01C9B1D9D059393
:108E7000E6E71F2CECD10123059A009316992B00ED
:108E800038001CF04CF9154D0028BAD1144DB8E744
:108E9000169B1CA8E9181EF0DCFF1E9B169A3900D1
:108EA0001800069322F01DFB169A1E9B944606930B
:108EB000634418002A00059922F013FBB2E70095DD
:108EC000059B169A390020001FF00EFADBE7C0461A
:108ED00090E70200DC14030080E70200AC09030005
:108EE000A409030070B50C008AB0050004A920682D
:108EF0001600FEF72DFE00230593049B0100C21807
:108F0000029605AB06A801940095FFF7AFFA06A9F3
:108F10000248FEF7ADFD0AB070BDC046DC14030088
:108F2000F0B5050087B008680C0005F089F80090DE
:108F3000012D2AD96668022D28D0A06805F068F9AD
:108F40000500002108001CF0BAFC04A9019020686B
:108F5000FEF7FEFD049B0400C7183F4B9E423FD125
:108F6000A7422CD920780BF009FB002811D1A74289
:108F700025D9002D0FD121003A1B00981CF0EEF8E6
:108F80000100019802F07EF919E0334E01256D428F
:108F9000D7E70134E4E7260030780BF0EFFA002839
:108FA00002D10136B742F7D12100321B00981CF0E4
:108FB000D5F80100019802F065F9B74202D801988E
:108FC00007B0F0BD340020780BF0D8FA002802D0AA
:108FD0000134A742F7D1EB175B1BDB0FED1AC6E795
:108FE000300005F02DF8009B834202D03000FEF7E0
:108FF000BBFC05A93000FFF71FFA059B0390002B6F
:1090000017D1164916481BF003FCF7F7E0F83E00AD
:109010002100321B00981CF0A1F80100019802F019
:1090200031F9B742CBD9059BF418EB175B1BDB0F6B
:10903000ED1A2600059B0293002DE8D0029BF31841
:109040009F42E4D3029A0399300022F03BFA0028B1
:10905000DED00136F0E7C0464CCA02001A680300B1
:1090600044DD0200F0B50D008BB0022803D8FFF7F5
:1090700057FF0BB0F0BD086804F0E2FF08A90490A8
:1090800028686C68FEF764FD0090A86805F0C0F8D9
:10909000431C07000021180005931CF010FC354B01
:1090A00005009C4202D1344806F094FC09A9200036
:1090B000FFF7C2F9099B0690002B05D12F493048D4
:1090C0001BF0A6FBF7F783F8089A3C009446009B38
:1090D00063440293BB000393099B0193019A029B93
:1090E0009E1A002C0BD0009BB34208D8019A069917
:1090F000300022F0E7F9002822D0013EF1E7EB68CA
:10910000BE009C19009A029B00999A1A04981CF0C0
:1091100025F82060002F11D0059BDC1BEB68A70011
:1091200099193A00180022F0E5F96B6800211A1B22
:10913000EB689200D81922F0EFF9AC60280098E7AC
:10914000039AEB68944663440793029B04989A1B26
:10915000019B013FD21AF1181CF000F8079B029600
:109160001860E3171B1BDB0FE41A039B043B0393FC
:10917000B2E7C0464CCA02002F6803001A68030019
:1091800044DD02002022074B07491A701D3A5A702D
:1091900004329A7000220548DA7059601A725A72C5
:1091A0007047C046FC020020746962754CCA020018
:1091B00002220A4B10B5DA6700220121084B5A61DE
:1091C000084A11615A69002AFCD0074C606F0028D8
:1091D00003D01FF0BDFE0023636710BD04E100E073
:1091E000FC10004000100040AC09002010B5FFF753
:1091F000DFFF014810BDC0464CCA0200F8B5FFF7BA
:10920000D7FF314C26786578013601357543280043
:109210001FF077FE00222D4B451958672C4B801903
:109220001D602C4B012118602B4B5A608022D20507
:1092300011605A68002AFCD00321284B6156284A45
:1092400000259950A178043A9950617A08329950D2
:109250006168244A08269950217A234A234F99505D
:109260000121234A9D5004329950224A9E50812266
:10927000247892042243A324E4001A5102221E4CB3
:109280001A511E4C1F511E4F043C1F5118271D4CD4
:109290001F511D4C1851C120C02480001E501B4876
:1092A000640002510260802080001C580E3222436C
:1092B0001A50174A5560596051680029FCD00021A6
:1092C000116101229A60F8BDFC020020AC09002067
:1092D0000C03002008030020FC00004000100040A8
:1092E0000C0500001C05000024050000FFFF000025
:1092F0002C05000014050000340500003C050000AA
:1093000021100100540500000405000000E100E008
:10931000FC10004010B5FFF771FF014810BDC046BA
:109320004CCA0200F0B505008DB01600002805D02B
:10933000734974481BF06CFAF6F749FF724B09AA9F
:10934000190091C991C21A789F7806925A780592AD
:1093500003229A5604925A6801921A7A5B7A029210
:10936000039373689D4239D2EB000793B368EA0018
:109370009B181A68002A02D0042A00D0A7E0013501
:10938000EFE7631EFA2B00D99FE0E3B20693F6E7FE
:10939000631EFD2B00D998E0E3B20593EFE7642C40
:1093A00000D992E0E7B2EAE7072C00D98DE0574BED
:1093B0001B570493E3E7022C00D986E0E3B2039342
:1093C000DDE70194DBE7FF2C00D97EE0E3B20293F6
:1093D000D5E74F494F48FCF741F9ADE74E4B09AC93
:1093E0005B6F002B17D16B461B7EA77023706B46FB
:1093F0001B7D63706B461B7CE370019B0A936B467D
:109400001B7A23726B461B7B63723F4B07CC07C3EF
:1094100042480DB0F0BD6B461B7E3B4D23706B4642
:109420001B7D637022882B889A4212D0FFF7C0FE02
:109430006B461B7CA770E370019B0A936B461B7AFB
:1094400023726B461B7B63720ECC0EC5FFF7D6FEF4
:10945000DEE70222324B3349DA670022324B4A619F
:1094600001321A614A69002AFCD06846007C09AAC8
:10947000D070019897700A906846007A107268461A
:10948000007B5072204870CA70C0284A04989850D7
:109490000398043A9F50083298500198244A9850F3
:1094A0000298244A985000224A6001325A604A6861
:1094B000002AFCD000220A61C02101329A601E4BB2
:1094C000013249005A501A60A2E71C4982E75868E5
:1094D00004F0CAFEB368EA0004009858FEF720FBC7
:1094E000174B0200C018062800D972E710F054FE8E
:1094F00049FF50FF57FF5CFF63FF69FF6BFFC046EA
:1095000066680300CCDC0200FC020020496803000E
:109510008A68030044DD0200AC0900204CCA020046
:1095200004E100E0FC100040001000400C050000C9
:109530001C0500002405000000E100E0A068030015
:1095400024FDFFFF10B5034903481BF061F9F6F74E
:109550003EFEC0465168030044DD0200F7B5314AC3
:109560000B00576F002F01D1FFF7ECFF02212E4CAB
:109570002E4DE167A324E4002C590195E4B2013497
:109580003C192B4F2B4A3D68AC4203D12A4E116047
:109590003000FEBD257800282BD1601C002B04D1A3
:1095A0002900FEF7B3FA06000AE05A68AA4200D979
:1095B0002A0001260100186821F09CFF6B001E4361
:1095C000691CED433B6861185A1A2000009321F092
:1095D00091FF009B019A5D19184B3D60D550002208
:1095E000174B1A610123019A9360124ADB1813602A
:1095F000CEE7022D0DD96378012B0AD1A278002A7B
:1096000007D1E378012B04D1E91E201DFEF766FA8D
:10961000C9E70223074A0B4913600B481BF0F8F80F
:10962000F6F7D5FDAC09002004E100E00010004091
:109630000803002000E100E04CCA0200040500001D
:10964000FC100040C568030044DD0200164B30B535
:109650005A681648002A03D000225A6001328260FC
:109660001A69002A1FD000221A61A323104CDB00C4
:109670002268C5581178EBB28B4201D219001570DF
:109680008025ED004559012D0BD10A4D02335B18A1
:109690002D68D3189D4204D30131074B5218226024
:1096A000C2500123836030BDFC1000400010004018
:1096B000080300200C03002004050000F7B5304F1C
:1096C0000D00796F01921E00002901D1FFF73AFFCA
:1096D000A3232C4CDB00E258AB19D2B29A4204D23D
:1096E000561BAA4201D215000026AB190B707B6FE6
:1096F000010001332A00180021F0F3FE002E06D0ED
:109700007B6F013558193200019921F0EAFE0222DF
:109710001D4BDA6700221D4B5A61013222615A69E2
:10972000002AFCD0796F1A4AA150002159600131FA
:10973000216059680029FCD00121A1600021196134
:1097400019690029FCD013490968A15000225A6107
:10975000013222615A69002AFCD000225A6001328B
:1097600062605A68002AFCD000221A610123C021DD
:10977000A360094B023249005A501A60F7BDC04637
:10978000AC0900200010004004E100E0FC100040A3
:10979000040500000803002000E100E007B501A96E
:1097A000FEF74AFE019B020003210248FFF786FFF5
:1097B00001480EBD456803004CCA02001FB50122D6
:1097C00001A904F0DFFE002301981A000299FFF7B7
:1097D00075FF014805B000BD4CCA0200F0B587B066
:1097E000039205910D9A03990500521A0CA9097864
:1097F00020200C00844339D030293BD00CA90291A1
:109800000121802401911C4036D0D40FA41864108B
:10981000171B002C37DD2600019B0493B34200DDAB
:1098200004966B68049A029928689847049BF61A74
:10983000002EF1DC039B002B06D01A0005996B6803
:1098400028689847039BE418002F0CDDE419019E5B
:10985000BE4200DD3E003200029928686B689847DE
:10986000BF1B002FF3DC200007B0F0BD07490291B9
:109870001021C6E70649FAE701271F4001D114006D
:10988000C7E71700D6E70024D4E7C046F76803000F
:1098900008690300F0B593B0069318AB20CB049091
:1098A0001B780F0016000793CB070BD48B0703D14F
:1098B000854B0A689A4205D0380004F0A9FC0127BC
:1098C0004000074381231D4209D1079B302B06D15D
:1098D0001A9B1B9A934200DA1A9200231B933800BA
:1098E0001DF0FCFA0AAA1300002806DDAB070FD50D
:1098F0002B231370123B04AA9B18EA0616D5022EDE
:109900000DD130221A70069A01325A7002330DE0DE
:1099100013006A07F1D520221A701923EBE7082EED
:109920003CD130221A70AA0535D4013300220AA98D
:109930001A705B1A0593AB0600D52C320EAB0B9355
:10994000102300210C931B9B0D91012B01DD402363
:109950001D4304ABD9756B4640241B7E2C400392FB
:10996000029322D03B00019100960DAA0CA90BA8EE
:109970000CF0FAFB037807002D2B2DD104AAD37528
:109980000D9B1B9A013B01370D93012A00DD95E0E9
:10999000002634004AE0069A0E32B6E7102EC5D1F2
:1099A00030221A70069A1732AFE70AAB019300967D
:1099B0003B000DAA0CA90BA80CF0D6FB1B9B0700C3
:1099C0002600012B32DD0D9B1B9C9C4215DA1C00EE
:1099D00013E00026340019E01B9B012BD8DD0D9B02
:1099E0001B9C9C4200DA1C00172304AA9B181B78BE
:1099F000002B00D00134059BE4181A9BA342E8DD3C
:109A000001261C1B2E4001D02600002401239D436B
:109A10002F330793002C09D0103B009300230194AF
:109A20001A002A490498FFF7D9FE04006B0621D5D5
:109A3000172104ABC9180B78002B0AD00023012290
:109A4000009301920498FFF7C9FE1A9B2418013B6A
:109A50001A93059B002B0DD0012301930023059A37
:109A600000930AA90498FFF7B9FE1A9B059A2418D7
:109A70009B1A1A931B9B012B00DD1A931A9B0D9ABC
:109A80000193079B3900009304982B00FFF7A6FE73
:109A90002418002E09D020230093002301961A00D9
:109AA0000A490498FFF79AFE24180B980EAB9842C7
:109AB00001D01FF04DFA200013B0F0BD1B9C9C425A
:109AC00098DA1C0096E7C046E81F0300C77603003B
:109AD000F0B50600140000278DB00D002B78002B88
:109AE0001ED1A94208D26B1A04931A003068736819
:109AF00098472900049BFF180B78002B00D13EE10A
:109B00004B1C0493202300253022082104200893B5
:109B1000049B1B78002B07D10693013B079355E06C
:109B2000252BDED00135D9E72D2B05D12C3B1D434C
:109B3000049B01330493EBE72B2B01D1293BF6E780
:109B4000202B01D10543F3E7212B01D10D43EFE792
:109B5000302B23D000230A210693049B1B781A0084
:109B6000303A092A1ED92E2B50D1049A049B5278E0
:109B700001332A2A1FD0049300230A210793049B50
:109B80001B781A00303A092A20D8079A4A43D3187A
:109B9000303B0793049B01330493F0E74023089282
:109BA0001D43C5E7069A4A43D318303B0693049BEE
:109BB00001330493D1E7049B0233049323680434F4
:109BC0000793DB43079ADB171A400792049B1B7825
:109BD0006C3B59425941049B5B1804931B780593D5
:109BE000002B00D1CBE0642B00D1A1E022D8502B78
:109BF00029D00ED8453B022B00D8A9E001220499B8
:109C00003068736898470137099452E001235B423A
:109C100084E7059B622B3CD057D8582BEED1231DEF
:109C20000993069B01950393089B0293412300939C
:109C3000313B7BE0059B712B53D00FD8672B00D8AD
:109C400086E0702BDAD1231D0993069B01950393BF
:109C5000089B029361230093513B67E0059B752BA2
:109C60005AD0782BEFD0732BC8D1231D24680993C9
:109C7000002C49D0079B013303D1200021F0B2FD15
:109C80000790069B079A0193089B210000932B00E5
:109C90000BE0231D09932368002B0ED0069B0422A2
:109CA0000193089B374900932B003000FFF796FD86
:109CB0003F180499099C01310FE7069B0522019387
:109CC000089B314900932B00EFE7231D099323687C
:109CD0000BA90B70069B01220193089B00932B009C
:109CE000E3E7231D0BA9206809931CF0BAFD079B2D
:109CF0000100013301D10B9B0793069B079A019347
:109D0000089B00932B00D0E7069B06220193089B3B
:109D10001E4900932B00C8E7231D0993069B01955C
:109D20000393089B029361230093573B00220AE0B0
:109D3000231D0993069B01220393089B019502931F
:109D400061230093573B216830001BF078FBAFE79D
:109D5000072307349C432300206861680833099374
:109D600013F0F2F9079B011C0293069B059A0193DD
:109D7000089B300000932B001BF0D5FB98E73800C0
:109D80000DB0F0BDE5680300EA680300F068030069
:109D9000F7B5314FB43701972F4A3049FC32536C35
:109DA0008B4200D8F7BD0325043B53641A682A4B45
:109DB000511CAC331E680C008B08F35C2C40640013
:109DC0002341881A2B400131022BF4D00326019B3A
:109DD00012011B6800019A181F4983080093009B19
:109DE000002BD9D00F23106818422BD11C4B1B68B5
:109DF000984227D30C00B8342468A04222D20F2402
:109E0000C01AC31723400C001B181B111D00AC34D3
:109E1000246898082418207835406D00844628412D
:109E2000304001280ED13700AF403D0067463D432A
:109E300025700D00FC356C6C0A4FBC4207D2201D0A
:109E400068642360009B0432013B0093C7E70B006A
:109E5000BC331860F6E7C046AC0900206C0A00204D
:109E6000600A0020EC0A00200F23994370B5060019
:109E70000D00081A412110F0A3F9104C0200230034
:109E8000B033186023002100AC331E608301EB1A4D
:109E9000B4310B6023003000B83300211D6021F085
:109EA0003BFB22000023FC32D364A2225200A352C7
:109EB000443A4733FF3AFF33E25270BDAC09002009
:109EC000A222034952008B5A01338B527047C0467D
:109ED000AC090020A222034952008B5A013B8B524D
:109EE0007047C046AC090020A223034A5B00D05A49
:109EF000431E9841C0B27047AC090020F7B500245A
:109F0000032500900191019B9C4200D1F7BD009A6E
:109F1000A300D3580F2213422DD11A4A1100B43195
:109F200009688B4227D31000B8300068834222D2E0
:109F30000F20591ACB17034010005B181B111F008C
:109F4000AC3000689908401801782F407F008C469B
:109F50003941294001290ED12E00BE403700664606
:109F6000374307701700FC37786C074EB04206D2B3
:109F7000021D7A640360FFF70BFF0134C3E7BC32B4
:109F80001160F8E7AC090020EC0A002010B5FFF7DB
:109F900097FF064800220300BC331A600300044AFE
:109FA000FC3328215A64FFF7A9FF10BDAC0900203B
:109FB0006C0A0020F8B503262C4C00252200BC3288
:109FC0001368AB420FD102221900032794462200E6
:109FD000B03212689200914226D30023FC34E3642D
:109FE000FFF778FFF8BD23001560214AFC335A645F
:109FF0002300B0331B689B009D42DDD22200AC32AF
:10A000001268AB08D35C2A0032405200134133403F
:10A01000032B07D12200FC32536C191D51641D60C3
:10A02000FFF7B6FE0135E3E72000AC3000688A0890
:10A03000801802780D0016003D406D002E413E4014
:10A04000022E09D0032E0BD0012E07D13B00AB40CE
:10A050009A430270012301E0002BF7D10131B6E7EA
:10A060006346AB409A4302700023F7E7AC09002037
:10A070006C0A0020274AF0B513001100B833B43140
:10A0800009681B6803265B1A110003600023B031C6
:10A090000C681900AC32156843608360C3600361CB
:10A0A0004361A400A14206D143681B014360836859
:10A0B0001B018360F0BD0F008A08AA5C37407F0057
:10A0C0003A413240012A0CD8012B0ED1C768013722
:10A0D000C7604769BB4200D94361012A10D0002AFA
:10A0E00009D0022A10D00131DCE7022BF1D1076937
:10A0F00001370761EDE78368013383601300F2E7FE
:10A10000436801334360F9E742680133013242603A
:10A11000E9E7C046AC090020A223F7B5424F5B0037
:10A12000FD5A0F300409002D02D000252800FEBD85
:10A13000002CFAD0A3235B00F95A4A424A4101920B
:10A140003A00B03212683B0094463A003026FC33A5
:10A15000AC32DB6C1068634507D3019B002BE4D164
:10A16000F9F7D2FE01230193EAE70321C25C0A4218
:10A170002AD10135AC4228D89B00591B4C1C012D1B
:10A1800004D13D005A1CFC359208EA64A2088018EC
:10A1900026000322012516407600B54006780231DC
:10A1A00035433E000570AC3601928B422CD23A000A
:10A1B000B4321568210101336D181A1B12010021F8
:10A1C000280021F0A9F9B1E700250C210A4205D1A8
:10A1D0000135AC4203D89B000133CEE70025324263
:10A1E00005D10135AC4203D89B000233C5E70025F9
:10A1F0003F218A4305D10135AC4203D89B0003338C
:10A20000BBE700250133A6E70D0032688808101867
:10A21000019A0131154002226D00AA401500027812
:10A2200015430570C1E7C046AC090020A22330B534
:10A23000214A5B00D35A002B3CD10F21084239D16F
:10A240001300B4331B68984234D31400B834246824
:10A25000A0422FD2C31AD8170840C018130000110B
:10A2600003250400AC331B6881085B5C2C40640050
:10A2700023412B40012B1DD11300FC33DC6CA14288
:10A2800000D2D9640321AC3214688308E3180400B7
:10A290000D000C406400A5401C780130AC431C70DC
:10A2A00014688308E35C04000C40640023410B4005
:10A2B000022BE9D030BDC046AC090020A223F0B586
:10A2C000002685B00700614802925B00C25A0D006B
:10A2D000B24206D1B74207D139002800FFF71CFF70
:10A2E0000600300005B0F0BD002904D13800FFF7AA
:10A2F0009DFF2E00F5E70F243B0016002340F0D110
:10A300000200B43212681E009742EAD30100B8314D
:10A3100009688F42E5D2B91ACA17224052181211A1
:10A3200000920200AC321268009C0192009A0199DE
:10A3300092088A5C0321214049000A4103210A4016
:10A34000012ACED129000F310909B0308C460168AD
:10A35000033689000391210014000131039A9142D0
:10A3600012D201988A08825C080030404000024105
:10A370003240022A02D101340131EFE7002A03D131
:10A380000133E2189445F7D8644501D13E00A8E7AF
:10A39000644521D9009B032663441900009B0800F3
:10A3A000E218AC239C46294B9C44634605001B687D
:10A3B00084081C19330035406D00AB40257801300E
:10A3C0009D4325709042F0D1204B8908FC33DA6C14
:10A3D0009142DBD2D964D9E71B199C4523D80325C8
:10A3E00002261A49009BAC31E3180191009A62449D
:10A3F000934209D36346191B090120010A0038184A
:10A40000002121F089F8C1E70199180009689A082C
:10A410008A1831002840400081400800117801333B
:10A4200008431070E2E7029E002E00D159E7002198
:10A430002800FFF771FE061E00D152E72201390005
:10A4400021F04FF83800FFF7F1FE4AE7AC09002091
:10A4500080235B051869034B1B7843438020C002AF
:10A46000C01A70471C09002080235B051869034B44
:10A470001B7843438020C002C01A70471D0900208A
:10A4800070B5084DC4012B68002118191CF0B2FDED
:10A490002868054B00197F3000781B788342F0D282
:10A4A00070BDC046100300201B09002010B5C37901
:10A4B0000400002B08D0064A037981791068DB017B
:10A4C000C01801301CF096FD0023237210BDC04659
:10A4D0001003002010B5034903481AF099F9F5F765
:10A4E00076FEC0461969030044DD020010B5124B28
:10A4F00001001A684379DB01D31818007F30047813
:10A50000FF2C08D10879C00112185278FF2A0FD009
:10A51000887990420CD08A799B180132D2B258784F
:10A520007E2A01D08A7110BD00234C718B71FAE72D
:10A5300001204042F7E7C04610030020F82270B522
:10A54000920213784D2B01D08022D20280268020E7
:10A5500076053469336964421440E41AC0023169F3
:10A56000001B0FF02DFE284B284918703369E218A4
:10A5700052185D421540264B264A27499A1A52180E
:10A580003169954230D38020C002401B0FF018FE85
:10A59000224B641B1870E411214BE4B21C70A12003
:10A5A000012300251F4A20491360C0004D604B68FD
:10A5B000002BFCD01358DBB2A342F7D21B49013366
:10A5C0000B7001235360FFF743FF03780500184C1D
:10A5D000FD2B0BD180235B051869164BC009C018F1
:10A5E000C0012818206070BD6D18C9E7FFF73CFF57
:10A5F0000378803DFD2B01D12560F4E7FFF734FFA0
:10A60000FD211CF0F7FCF7E71D090020FF87FFFF85
:10A61000980200200000002028BE03001C09002032
:10A620001B09002000D00040FCD000401E09002083
:10A6300010030020FFFFFF01F7B5254B254F1A78C7
:10A64000254B14001B7839680133E001405CFF287A
:10A6500039D00134E4B29C4200D101249442F4D1B7
:10A66000802300265B051B69DB090093E30101934E
:10A670003B68E2019D182A78280053425341F6189E
:10A680001CF0CEFC0023002815D1134B01341B789D
:10A69000E4B201339C4200D101240D4B1B78A3424C
:10A6A000E4D1072E11D91AF091FFC6E7DA01AA5CAE
:10A6B000002AEAD10133009A9342F7D13868019B0E
:10A6C000C0181CF0A3FC2000FEBDFF24FBE7C04621
:10A6D0001E090020100300201B090020F7B5070009
:10A6E0000D0001240E4B1B7801930E4B1E68019B3D
:10A6F0009C4202D9FF242000FEBDE10171180B78B5
:10A70000FE2B09D18B78AB4206D103312A003800E9
:10A7100020F0D8FE0028EED00134E4B2E7E7C046CE
:10A720001B0900201003002010B5054A03791068AA
:10A73000DB01C018817800220330FDF7CFF910BD8E
:10A7400010030020F0B585B002900D0016000393B1
:10A7500078294BD8FFF7C2FF0400002E3ED0FF2817
:10A7600001D0FFF78DFEFFF767FF0400FF2805D13A
:10A770001F4920481AF04CF8F5F729FD1E4FC0017B
:10A780003B680190FE2118181CF034FC3B68019ACC
:10A79000E9B2981802301CF02DFC3868019B2A00A1
:10A7A000C0180330029905F0ABFE0C201EF0A9FB87
:10A7B000039A0300002A17D0104A1A600E4A1C712F
:10A7C00012685C71E4011419A278DE7102329A7188
:10A7D00001221A726A46127B5A7202E03300FF2885
:10A7E000E3D1180005B0F0BD054AE6E70023F8E71D
:10A7F000366903004CDB020010030020F005030063
:10A80000A806030007B501A9FDF716FE0199FFF799
:10A8100065FFFF2805D10549054819F0F9FFF5F74F
:10A82000D6FCFFF72DFE03480EBDC0464C69030061
:10A830004CDB02004CCA0200F7B50192027A050017
:10A840000091002A01D1FFF745FEC479002C06D102
:10A85000214A17680279D201D25D002A04D1092267
:10A8600001201A604042FEBD69797E22C901791833
:10A8700008007F30AB790078D21AFF2809D12879F7
:10A88000C00138184078FF2819D0C01A824200D978
:10A8900002000198061B964200D91600002E19D01E
:10A8A000009A01331019C918320020F01AFEAB7952
:10A8B0009B19DBB27E2B04D0AB71A419D4E7002224
:10A8C000E7E70023AB716B79DB01FB187F331B7863
:10A8D0006B71F2E72000C6E710030020F0B585B0E9
:10A8E0000393037A04000192002B01D1FFF7F2FDDC
:10A8F000C379002B34D02D4A03791268DB019B5CAD
:10A90000002B2DD0019B02910093009B002B2CD09B
:10A910007E22A379D71A009A974200D9170060794E
:10A92000224E0133C001C01833683A00181802994A
:10A9300005F0E6FDA379DB19DBB27E2B33D10023D2
:10A94000A371FFF779FE0500FF2811D12079FFF7E9
:10A9500097FD002323721C23039A13601D3B03E021
:10A960000923039A13600A3B0193019805B0F0BDD7
:10A9700060793368C001181829007F301CF03AFB59
:10A980003368ED01581961791CF034FB6279336842
:10A99000D2019B187F331B786371029BDB190293F2
:10A9A000009BDB1BB0E7A371F7E7C0461003002054
:10A9B000002170B508001AF082FF012405000C4B3D
:10A9C0001B78A34201D2280070BD0A4AE301106837
:10A9D000C0180378FE2B08D1817800220330FDF7E0
:10A9E0007DF80100280000F04DFC0134E4B2E6E7F8
:10A9F0001B0900201003002073B501A9FDF71CFD01
:10AA00000199FFF76BFEFF2805D10F490F4819F098
:10AA1000FFFEF5F7DCFB00257E260D4B1C68C3010D
:10AA2000E31859789B780233DBB2C201A2187F3257
:10AA30001078FF2804D1C81A40191CF073FA76BDAB
:10AA4000F31AED180023F0E74C6903004CDB020019
:10AA50001003002010B5024B024A18F093FA10BD03
:10AA6000ADA40000EDA400000523020070B5094C60
:10AA7000094D2068434309489B189B0018582B68D0
:10AA80002260C0180F2319400901286001F028F83E
:10AA900070BDC04614030020F8020020BCEA02008A
:10AAA000A839030000B5080006292ED80FF06AFB6C
:10AAB000040A10161B2128009A18E223DB00D21882
:10AAC000107800BDC4329200D05C8006800EF8E79A
:10AAD000C4329200D05AC004400EF2E7C432920051
:10AAE000D0580003F8E7C43292009A189078000911
:10AAF000E7E7C43292009A18D0780007000FE0E729
:10AB0000C43292009A18D078F1E7024A024B002032
:10AB10001A60D6E75B69030050000020A83910B521
:10AB200004000800062949D80FF02CFB040A141F62
:10AB30002A343F00E221A218C9005218137010BD38
:10AB40003F210B401800C4329200135D8B43034336
:10AB50001355F4E77F21C432920019401948135B62
:10AB6000890103400B431353E9E77F21C43292006C
:10AB700019401059144B490303400B431351DEE7AE
:10AB80000F20C4329200A2181901937803400B439E
:10AB90009370D4E70F210B401800C4329200A21822
:10ABA000D3788B430343D370C9E70F20C43292009C
:10ABB000A218D1781B0101400B43F4E7034A044B70
:10ABC0001A60BCE73FE0FFFFFF1FF0FF7969030059
:10ABD00050000020F0B5D2B287B00F0005930721D6
:10ABE00013000B40013BDBB2042B02D92C4D2D4C42
:10ABF00025608A4319020291002A29D12A4BC55C9B
:10AC00002D09ED43EBB23D7801932C005B1BDBB2C9
:10AC100004930826254B029A1B199B5C5A00D2B25A
:10AC20005BB20392002B38DA1A210320013EF6B200
:10AC3000FFF71AFF039B002EF0D10134049BE4B20E
:10AC4000E318DBB2002BE4D1019BED1A3D701AE052
:10AC5000D4431749E4B2CF5C0825144B029A1B1960
:10AC60009B5C5E005BB2F6B2002B0FDA052102207E
:10AC7000FFF7FAFE013DEDB23300002DF1D10134B2
:10AC8000E4B2002CE8D1059807B0F0BD39000120EE
:10AC9000FFF7EAFE002FE9D0ECE706210420C5E724
:10ACA000666903005000002019070000F16E0300E0
:10ACB0004C7503000022F0B505000F00FF200F24A3
:10ACC0008BB008AB654EDA710100C4318900691898
:10ACD0008B781A09B25C234012011343CA788B7037
:10ACE00013071B0FF35CA243234013431A09B25C02
:10ACF000234012011343CB700138E5D2E223DB007D
:10AD0000EE5CB308F31ADBB20593554B1B68002BBE
:10AD10000BD0E222C4218120D200890000013B0037
:10AD2000AA186918281807F039FA00244823029451
:10AD300003930194009481222B1912019B181B7814
:10AD4000180004930723984320D008A92300049AED
:10AD500007312800FFF73EFF0230C4B2023FFFB2C6
:10AD6000002F78D02B780393013EF6B2002E47D106
:10AD7000E2222B19D2009B181E78B308F31ADBB21B
:10AD800005930023029301930093D4E7354B009A77
:10AD90009C469A5C2300C4339B00EB189978090900
:10ADA0000A4331498A5C019906926246DB78525C1B
:10ADB0001907090F0A432C491B098A5C2B49079282
:10ADC000029A8A5C07991343069A52182649C95C6D
:10ADD00001238918FF2A00DC031CC91888230906EF
:10ADE0001B06C918090F0020FFF73EFE039B013B1D
:10ADF000DBB20393002BB7D10134E4B2013FAEE7DD
:10AE0000059B013BDBB20593002B02D1049B002B79
:10AE100018D12200C4329200535D00999B069B0E0C
:10AE2000CB18DBB20093535B0199DB045B0ECB18AC
:10AE3000DBB201935359029A1B035B0ED318DBB2AA
:10AE4000029378E708A92300049A07312800FFF746
:10AE5000C1FE04008CE70BB0F0BDC046756A03006C
:10AE6000E4020020417403004D6C0300F16D030007
:10AE7000064B1B5C002B05D0054B185C4843C011EA
:10AE8000C0B27047034B185CFBE7C0469D6D0300E2
:10AE9000166C0300D66A0300064B1B5C002B05D022
:10AEA000054B185C4843C011C0B27047034B185C97
:10AEB000FBE7C0469D6D030051750300266B030040
:10AEC000F0B5037A8DB004007F2B00D145E103007B
:10AED000070000250933FF330837099301953E78B1
:10AEE0007F2E00D086E000230693019306998B0005
:10AEF000E31803931A7A481C1B7BC0B206907F2B81
:10AF000000D11DE19F49CE5C8D5C9F49AE4200D0CF
:10AF1000F3E08D5CCB5C0493039B597A019B591839
:10AF2000CBB20193049BEB18DBB20793023B1B06E9
:10AF3000DCD4A826019B5D1BEBB20593A82E00D0A4
:10AF4000E3E0039BA8215F7A5A7B7F085208BB1875
:10AF50000293019B20009A18D2B2DF1BFFF7A0FDDD
:10AF6000FFB205003A00A8212000FFF799FD2D1A35
:10AF7000EDB27F222B006DB293430893EB17E818D4
:10AF8000584002990FF08CFA2800CBB2029909932D
:10AF90000FF0A0F90025C3B20A93059F029BDB19AD
:10AFA000DBB20B933A0031002000FFF779FD0A9BDA
:10AFB00001370B9A1818FFB2C3B2974200D1B9E01B
:10AFC000099AAD18029AEDB2AA420DD8AD1A202105
:10AFD0006A4652181278EDB252B2002A00DAA7E09F
:10AFE000002B01D00133DBB23A0031002000FFF723
:10AFF00095FDD7E7012E7AD12B003100019A200070
:10B000001AF04BFBBA78614BA1789B185B78300043
:10B010000193FB780293FFF72BFF3F23E178034076
:10B0200030000393FFF738FF7F22594B9B5D1A4096
:10B03000584B04929A5D0F231A400592564A925D2E
:10B040001A400692554A925D1A4007923F22544B8D
:10B050009B5D08937B78EB18DBB20A93039B13404C
:10B0600003937F23184083019C462A003F21C4326A
:10B070009200135D0F268B4303990B431355135B0B
:10B0800048490B4061460B431353049B1059590325
:10B09000454B03400B430598190C314000011351F7
:10B0A0000843A21890701B0E0698B34307990343F8
:10B0B00009011E400E4320206946D67081220918DE
:10B0C0006319097812019A181170E222D2009B18B4
:10B0D0000299019A013552181A700A9BEDB29D42ED
:10B0E000C3D1099B0437BB4200D0F8E6FBE6022E31
:10B0F00088D12B00019AFF2181E72C48AE4201D96B
:10B10000C55C07E78D5C835C05E7049B019A310011
:10B110009A18D2B22000FFF7C3FC059A050031004F
:10B120002000FFF7BDFC079B2D1AEDB2029320E72C
:10B13000013B58E70136F6B2AF2E00D0FEE6D5E669
:10B14000023189006118019B497859186368C9B2B6
:10B15000002B04D02000FFF7ADFD0DB0F0BDE222C2
:10B160008025D200A0186D001A00C4329200125D32
:10B1700006789206D20EB21A013302700130AB4249
:10B18000F2D1E7E7866A03004D6D030041750300C5
:10B19000766B030085690300D5690300256A030007
:10B1A000F17303003FE0FFFFFF1FF0FFC66B0300DA
:10B1B00070B505000C200C001DF0A3FE024B45608D
:10B1C0000360846070BDC04620EB0200034B82B078
:10B1D00001AAA0331A6002B07047C046AC09002033
:10B1E000014BA43318607047AC09002010B5034927
:10B1F000034819F006FBF4F7EAFFC046FE0800001A
:10B20000C4DB0200064B07B51A00A033A4321B684A
:10B21000126801A95B1A9A4201D8FFF7E7FF07BD40
:10B22000AC090020002803D0012807D0002004E04A
:10B230008B680448002B00D1034870478B685B0083
:10B240001843FAE7AC090300A4090300002281684F
:10B25000F0B5CB0F094C5B185B100E199A4201DB5D
:10B260000748F0BDC568B11A940089002C196D58C3
:10B2700027682560C46801326750EFE7FFFFFF3F92
:10B280004CCA020070B583680D00416804008B420F
:10B2900012D3C900C0681DF04AFE63680A495A000B
:10B2A000A3686260D21A013352189B00E0609200DA
:10B2B000C018002120F030F9A368E268591C9B00F7
:10B2C000A16002489D5070BDFFFFFF3F4CCA0200C5
:10B2D000F8B5070016004C10836803D5E418E24364
:10B2E000D2171440A34200D21C000B493800FFF7CC
:10B2F000C9FFBB68094A591E9B189B00181FFA68B2
:10B300008C4203DBA40016510348F8BD15580139DF
:10B31000D5500300F2E7C0464CCA0200FFFFFF3FD2
:10B3200070B50025040085601021C0681DF0FFFD88
:10B3300004232900E0606360102220F0EDF801484A
:10B3400070BDC0464CCA020030B50C0085B0104B31
:10B3500002AD04310093013802230195F8F7BAFADF
:10B3600023680C4C996801290FD9D8680A4B029AB6
:10B37000C91889004118A24200D100222D79074B3B
:10B38000002D00D1064B1AF0F0F9200005B030BDB9
:10B390005CEB02004CCA0200FFFFFF3FA409030060
:10B3A000AC09030070B50C680B00A168020000290D
:10B3B00005D11A491A4819F02BFAF4F708FF20684A
:10B3C000012A27D05A68002302F0FAFFE168A26838
:10B3D00086008B19013A1D680436A260121A920089
:10B3E0008919180020F086F80021A368E0689A0007
:10B3F0001150616804290BD95B00994208D94908AA
:10B400008900E0681DF093FD6368E0605B0863609D
:10B41000280070BD01225242D5E7C046887503005E
:10B420009CD9020007B500900191022069461AF0EC
:10B4300002FA694601900220FFF7B4FF00480EBDF2
:10B440004CCA020070B50E000D490500002419F029
:10B45000E7FFB3689C4204D328000A4919F0E0FFD3
:10B4600070BD002C03D00849280019F0D9FFF168FD
:10B47000A30001225958280002F0FAFD0134E8E740
:10B48000C59803000ABD03000035030070B503260C
:10B4900004000D000E4029D1174B0A689A4225D1AD
:10B4A00083688A6899184368994210D904318900E1
:10B4B000C0681DF03CFDAA68A368E0609B181A1DD7
:10B4C0009B006260C0181022310020F025F8A368AC
:10B4D000E9689800E3681818AB689A0020F001F852
:10B4E000AB68A268D318A360044870BD290020008F
:10B4F0001AF0AAF9F8E7C04660EC02004CCA020054
:10B5000010B5040010201DF0FCFC044B84600360A7
:10B51000034B43600023C36010BDC04628010300F5
:10B520004F5702000B4B70B5050003600C0008007C
:10B53000042900D204206860AC6080001DF0E1FCAA
:10B540006A68E860121BA4009200001900211FF035
:10B55000E3FF70BD60EC02007FB50C0015001228FF
:10B560003CD005D8052819D007283CD0002432E06B
:10B570000300193B042BF9D893070DD1284B12680F
:10B580009A4209D1AB6800938A68EB68C96809F0F0
:10B590009DF9244C00281ED1234C1CE003231340AA
:10B5A000E4D11F4A2968914238D1A368AA68981843
:10B5B0001AF062F90600A368E1689A00C0681FF0FB
:10B5C00090FFA068F36880001818AB68E9689A00DB
:10B5D0001FF087FF3400200004B070BD1100200070
:10B5E000FFF754FFF7E703A9100002F04FFE002811
:10B5F000BCD0039B002B01DA00230393A3680398BC
:10B6000058431AF039F90500C36804210093A26871
:10B61000E068039B1CF034FE2C00DCE71C00DAE73A
:10B6200060EC0200AC090300A4090300F0B50400BB
:10B6300087B017000326002A29D10E401FD1544B92
:10B640000A689A421BD103AA806809F005F9049997
:10B65000039BA268E0685D1A521A890092004118A3
:10B660009B0018181FF046FFA368AA00E818E368BB
:10B6700080005242181831001FF04EFF6BE0049119
:10B68000022003A90394FFF78DFE424812E0042A2A
:10B690002DD1314221D13E4B0A689A421DD103AAD5
:10B6A000806809F0D9F8002806D103AAE168A068EB
:10B6B0001CF0F9FD07B0F0BD039B0498C01A1AF006
:10B6C000DBF805008368E1689A00039BC0689B0073
:10B6D000C9181FF006FF2800ECE700230A002068C5
:10B6E000A16802F06DFEE3688000C058E2E70E40FA
:10B6F00048D1274B0A689A4244D103AA806809F0CE
:10B70000ABF8049B0398BA68C51AAD180193002DD5
:10B7100025DDA368E9186368994207D98900E068C4
:10B720001DF005FCA368E0605B196360039BA268E1
:10B73000E068D21A9900EB189B0041189200C018DB
:10B740001FF0D8FE039BF9689800E3681818BB68DF
:10B750009A001FF0C6FEA3685D19A56095E7E3682F
:10B760008000F968181892001FF0BBFE0499B868B1
:10B77000A268039FE368521A38188900920059188A
:10B7800080006EE73A0020001AF0B7F87DE7C04667
:10B79000EC0003004CCA0200BFF34F8F024A034B78
:10B7A000DA60BFF34F8FFEE70400FA0500ED00E01A
:10B7B0000120024B1B685B0018437047C008002043
:10B7C0000120A922044BD2001B6898649B58034AAD
:10B7D0001360834018437047540000201803002072
:10B7E00001220F4B10B51A600E4A51680029FCD097
:10B7F00000215160A122D200985801225A6011F014
:10B800000FFC0022084B10F041FE11F09DFC0323B9
:10B81000020002209A43054B1043C01810BDC046D9
:10B8200000C00040FCC000400000D03F000080800D
:10B8300010B5C30708D483070ED10368094A9342A1
:10B8400002D0094A934207D102F0E2FC002801DD50
:10B8500006F06EFF054810BD02F03EFD0FF01CFE25
:10B86000F4E7C046E81F0300B40903004CCA020015
:10B87000F0B50F000A2485B001901C491C4818F04F
:10B88000E1FFFA200025800006F052FF019BAB4249
:10B8900003D0386802F0BCFC0500280021000EF03F
:10B8A000FFFD03AE3031B170280021000EF012FD13
:10B8B00021000EF0F5FD30317170280064210EF08A
:10B8C00009FD21000EF0ECFD002530313170705D76
:10B8D0001BF01DFF0100064818F0B4FFFA200135E7
:10B8E000800006F025FF032DF1D1C6E7F0ED020040
:10B8F0001800002073B501A9FCF79EFD019B06000E
:10B900001849502B16D8802040001DF0FAFA164C2A
:10B910000500231DD8670023019A93420FD15B22B3
:10B920002800EA5405F064FE2B0000280BD10434F3
:10B930000E49E0670E4818F06BFFF4F748FCF15C25
:10B94000E9540133E9E75A1B0133591E09789B2951
:10B95000F9D12900074819F001FC00230434E367FA
:10B9600076BDC046AB750300AC090020BA75030074
:10B9700044DD0200DC140300F0B58BB006000800C3
:10B9800011001A0010AB1F78334B05AD01950093E1
:10B990000523F7F79FFF912000011DF0B2FA2F4B0E
:10B9A00004A9D86702AB1B7B476043702B792C4FEF
:10B9B00003702B7A040083702B7BC3702B7C3000C8
:10B9C0003B60FCF739FD0025264B03900C201D60E1
:10B9D0001DF097FA244B0600036002F067F9B0608F
:10B9E00002F064F9214B224A1860224B11001D70AD
:10B9F000214B70601D70214B30001D602B0002F048
:10BA00002BF82000049A039919F0C7FA2000FBF7DD
:10BA1000DBFE0400A8420AD101F02CFF0F4B1848AE
:10BA2000DC67184B196818F0F3FEF4F7D0FB01221D
:10BA3000154B1A7002F034F90028FBD1134B043374
:10BA4000D8673B68002B04D00C4B1148196816F0DE
:10BA500085F907480BB0F0BD84EE0200B009002064
:10BA6000E402002020030020E4EE02001C0300207A
:10BA70004CCA0200210900201F09002024030020D5
:10BA800044DD02005000002020090020AC09002005
:10BA90009C75030000220D4910B50B78DBB2934270
:10BAA00010D10B4A1478002C02D001240C701370B2
:10BAB000084B1B78002B07D0074A1368203313600C
:10BAC000064B1A68100010BD8268FBE71F090020B2
:10BAD0002009002021090020200300201C03002051
:10BAE000D2235B005843134AF0B51368000C984208
:10BAF00006D2114C2368013323601368203B136086
:10BB00001F23050001270D4E9D431468A5420BD845
:10BB100003401A1D202A00D92022094C2468934290
:10BB200004D3084B1860F0BD3770EEE7E5182971B3
:10BB30000133F4E720030020240300202109002022
:10BB40001C03002028030020F0B587B00092027883
:10BB500004000E00930703D5009B002B00D0E0E00B
:10BB6000D307DB0F0ED0704B3340062B43D003239B
:10BB7000334003D16D493068884203D0009B012BCC
:10BB800000D0CEE00193530749D52368A568DF08AC
:10BB9000FF00EF19BD4230D3009B012B00D0C0E065
:10BBA0002368D9086368994210D104316160A068A4
:10BBB000C9001DF0BCF923686268DB08D21ADB00FB
:10BBC000A060D200C01800211FF0A6FC0721236846
:10BBD000DD086A1CD2000B4013432360A368ED000C
:10BBE0005D19514B2E601E40062E4ED00122237847
:10BBF0009343237049E00123C4E72868864204D1B7
:10BC0000009B022B41D104237CE0019B002B04D13B
:10BC1000310002F0ABFA0028F2D10835BAE76368C8
:10BC2000002B06D1009B012B00D07AE0200000F011
:10BC30007FF83D4B33400593062B29D1F0081AF0CD
:10BC400001FE0390616803980EF040FB0027049109
:10BC5000049B0293029BDD00A3685D1928680028FD
:10BC60001DD1009B012B5CD107212368DA0801322A
:10BC7000D2000B4013432360002F00D03D0000236F
:10BC80006B60059B2E60062BB0D1280007B0F0BD7D
:10BC90003100022002F090FF43100393D2E7042802
:10BCA0001DD1002F00D12F000298616801300EF0E5
:10BCB0000DFB049B02918B42CCD1009B012B30D118
:10BCC000002F2AD023683D000833236000237B60C7
:10BCD000059B3E60062BD8D02378009A88E78642E1
:10BCE00012D1009B022BD0D123680298083B23601D
:10BCF000013061680EF0EAFAA368C900CB58002B46
:10BD000000D080E72B60C0E7019B002BCCD1310035
:10BD100002F02CFA0028C7D0E3E7200000F008F872
:10BD200090E70025B1E7C046070080FFDC14030060
:10BD3000F7B54368040001935A1C002316495D5867
:10BD4000AA4204D904335C2BF9D101251543E8003C
:10BD5000A7681DF0E8F807232268656013400122F8
:10BD60003D000026236013432370A060019B9E4288
:10BD700003D138001DF0ECF8F7BD2968002907D081
:10BD8000042905D001222000FFF7DEFE6B68436026
:10BD900001360835EAE7C04638EF0200F8B505007D
:10BDA00000230768866811497A1C5858824204D9D2
:10BDB00004335C2BF9D101201043002428606C600F
:10BDC00080001DF0B0F8A860BC4203D130001DF027
:10BDD000BFF8F8BDA300F158002905D0042903D00D
:10BDE0000122280019F0F9FD0134EDE738EF0200D7
:10BDF000F0B50F00496887B005001600002901D092
:10BE0000002A05D13900280019F09AFF07B0F0BDCB
:10BE10000F321309C918019319F004FF0F22A86803
:10BE2000B9687C68324000D11032019B1E19254B45
:10BE3000F3185B00C3180393224B1020E3185B0038
:10BE4000CB189C46039B210002930023801A059087
:10BE5000002922D103986400041B1020821AD340C9
:10BE6000184823808446019B5B00E41A019B02343E
:10BE700063445A0020001FF04FFB002E04D07300D3
:10BE8000023BE35A002B1BD001216E603A782B78DD
:10BE90000A408B4313432B70B8E760460088013992
:10BEA000034318000493059BD840029B1880029816
:10BEB000049B02380290022040421B048444C7E7DE
:10BEC000013EDAE7FFFFFF7FF0B54B6815005268CF
:10BED00089B006000C00934201D22C000D0001270E
:10BEE000227861683A4000D12A783A4051183000EF
:10BEF00019F098FEB36838000193636829780293BB
:10BF000023781A0098430300A8684A400490A06868
:10BF10003A40039001988F43BC460590029F6868A1
:10BF20000299C01B01390690481C17D1029B590089
:10BF3000019B5918002A02D001230B80023101987D
:10BF400019F05CFE012170602B7822785A4033781A
:10BF50000A408B431343337009B0F0BD0398078840
:10BF600012483F18FF18069B5B1899421CD3049B8C
:10BF70001B881B1804980230049038006344584012
:10BF800000936B46D883D88B009B84460598624407
:10BF900002800230059003981B0C02309C46120C64
:10BFA0003B0C03900139BFE7004BE6E7FFFF0000C1
:10BFB000F0B591B007935B6804000E000692002B69
:10BFC00003D143604B6011B0F0BD069B5B68591C08
:10BFD000019319F027FE069B00215B68A0685A1C9C
:10BFE000520001931FF098FA00236360069B300013
:10BFF0005B68591C019319F015FE0699300019F081
:10C000009FFEB36875680293079B9B680393079B29
:10C010005B680593A3680893059BAB421AD81BD3B2
:10C02000039A2900029819F042FE002810D101233A
:10C03000089A706013806360069B1A78079B1B78D0
:10C040005A4001231A42BED0227813432370BAE724
:10C05000002801DA0023EEE78A4A059B9B185B0063
:10C060009C460022039B634404931B8801921AB2EE
:10C07000002A6CDA634610200027991C039B019A62
:10C080005B180993821A039B0A92099A934264D31C
:10C0900000201027029A6B00D0526A1C029D099260
:10C0A00072609A1CAA180A922A00019D791B0B91B2
:10C0B0000A998A425CD3049A12880D92029AD51882
:10C0C000059B099AD11A6F4B6160C918089B4900FA
:10C0D0005B180A93022362465B429B1A0F937368B4
:10C0E0000B930B9A059B93424DD310220020019B8A
:10C0F000D21A039B04998B4200D8A8E0614A102110
:10C10000944600250B9B029A63445B00D318019A66
:10C11000891A029A9A4200D8A7E06368002B07D0D8
:10C12000584A08999A185200525A002A00D1A6E09B
:10C130007368002B00D17FE7524A02999A18520087
:10C14000525A002A00D077E7013B7360F0E7019A6A
:10C150005B0001329BB292B288E71A880198110005
:10C1600081400F430A991F800A41023397B28CE73E
:10C17000158801992F008F400B9938430D4110808D
:10C18000A8B2023294E7AB1E28880E931B880004E5
:10C1900018430D990EF014F8002284460F9BEB18FB
:10C1A0000C93039B0C9909938D4212D82B889A42C9
:10C1B0002BD3D31A5A42190C9BB22A805A1E934190
:10C1C000CB180993099B002B21D0039F0C990020C9
:10C1D00030E06046099B0F881B884343BB4202D274
:10C1E000F81A90420DD8DB1B9B189FB2781E87412E
:10C1F0005A420A801A0CD219099B02310233099360
:10C20000D2E7821A0A800022F6E79A1A2A8062464A
:10C210000A9B0E9D1A80023B0A930B9B013B7360A5
:10C220005DE70B881A003B880237D318181808807E
:10C23000000C02318D42F4D82B881818099B2880F5
:10C24000000C1B1A099301235B429C44BAE7049B30
:10C25000019D1B88190029419340014304980180E6
:10C2600098B2049B023B049343E71A88019F100095
:10C2700038418A402843188095B2023B49E7013B88
:10C2800063604AE7FFFFFF7F436870B55A000023F1
:10C2900084680A4DA218944206D30278D20700D5CA
:10C2A0005B4201200B6070BD023AAB4203D8168896
:10C2B0001B043343EFE70020F5E7C046FF7F000093
:10C2C000F8B51F008B1E160000241E2B14D80B4B34
:10C2D0004068595C00010DF073FF0500A74204D0CF
:10C2E000013003210DF06CFF0400301E01D01FF05F
:10C2F00079FA03352C1924182000F8BDD1750300F4
:10C30000F0B593B0060006A80F001400F3F744FF41
:10C31000051E2BD13368310001263A0003A8019392
:10C32000F9F786FEA3082A003340019903A8F6F71F
:10C330008BFA0500032006F06FF928001AF0E9FCDB
:10C340000120404206F068F9F3F73CFF344203D085
:10C350003100134806F094F9012501210C4202D066
:10C360000F4806F08DF9280013B0F0BD01204042BF
:10C3700006F052F901210C4202D0094806F080F97A
:10C38000079801F05DFE0749F7F712F9051E04D181
:10C390000799054801F090FEDFE780256D00DCE796
:10C3A000C676030090DC0200B4EA02001FB520212B
:10C3B000684680241BF036FD640025481BF09FFB77
:10C3C00068461BF065FD23481BF099FB06F040F919
:10C3D0000128F2D002280BD11F481BF090FB6846C1
:10C3E0001BF04BFD012200201C4B1A7004B010BD45
:10C3F000032803D168461BF04BFDE7E7042804D06F
:10C40000C1B268461BF099FDE0E715481BF077FBC9
:10C41000019A002A08D110481BF071FB68461BF0F6
:10C420002CFD80204000E1E7282000230299FF3006
:10C4300003F0E4FF002803D10A4815F08FFCBFE7A2
:10C4400001221100FFF75CFF2042B9D0CEE7C046C1
:10C450009E7603007AB0030006B003004402002079
:10C4600053610300B976030070B586B0202102A89D
:10C4700080241BF0D7FC640044481BF040FB444878
:10C480001BF03DFB02A81BF003FD424902A816F079
:10C49000F2FC01280AD140481BF031FB02A81BF036
:10C4A000ECFC00203D4B187006B070BD022803D193
:10C4B00039481BF024FBDFE7032801D13648DFE7CA
:10C4C000042808D134481BF01AFB02A81BF0D5FC45
:10C4D00080204000E8E7052836D131481BF00FFBEB
:10C4E00002A81BF0D5FC06F0B3F86B46C1B2DD1D07
:10C4F00029700329E2D0042917D127481BF0FFFA3D
:10C50000012502A81BF0CFFC060002A81BF0D2FCFC
:10C510000200282000233100FF3003F06FFF0028C5
:10C520002CD1204815F0CAFCACE702A81BF005FD91
:10C530002B780D2B03D11C481BF0E1FAD3E7012126
:10C54000280006F09DF8CEE702A81BF0B3FC0028F7
:10C5500098D002A81BF0E0FCF7F720FA00280BD0D7
:10C560000A2102A81BF0E9FC104902A816F083FC7E
:10C570000328A3D00428ECD10025C2E70622290015
:10C58000FFF7BEFE204200D17CE78DE7F275030085
:10C59000377603005D76030006B0030044020020F6
:10C5A00062760300ED7A0300927603009976030029
:10C5B000074BDB68002B01D1180006E05A68824265
:10C5C00004D8801A04308000C05870471B68F1E717
:10C5D000AC09002070B5114D0400EB689868DB6869
:10C5E00083420FD30230C0001CF08BFCEB685A680A
:10C5F000D96803609B6852185B0083600023426027
:10C60000C360E860EA68D3685068591C04339B0033
:10C610000138D16040189C5070BDC046AC09002064
:10C62000074B4118884204D3D8B2002800D101300A
:10C6300070475A01D318027801305340F2E7C046E0
:10C6400005150000034B044ADA60002294331A6097
:10C650007047C046AC09002094EF0200F0B585B0E9
:10C6600001900E00FFF7DCFF144B0290DC68002CF9
:10C6700001D120001EE0270010373D00E3689B0039
:10C68000FB180393039B9D4201D32468EFE72868BE
:10C69000029A03789A420FD143789E420CD102301D
:10C6A000320001991EF00EFF002805D1ED1B6068D5
:10C6B000AD10281805B0F0BD0435E3E7AC09002043
:10C6C000F0B585B002900191FFF7C8FF002858D15E
:10C6D0002F4C019B27009437DD1C3B68002B17D0A3
:10C6E00026002C4A9836126831680392AA188A42AA
:10C6F0000ED90200691818001CF026FC03900028CF
:10C7000041D1244B386819681CF011FC039B3B6035
:10C71000230094331B68002B17D12E00802D00D2EC
:10C720008026300027001CF0F9FB94373860002881
:10C7300004D128001CF0E5FB2E003860230098335C
:10C740001E60230000229C331A6023009C331A6869
:10C7500094342468AD1801990298A4181D60FFF75D
:10C760005FFF6B461B7920706370019AA01C0299D1
:10C770001EF0B7FE0022019B2000E3189A70FFF71D
:10C7800029FF05B0F0BD33685B193360C0E7C046D0
:10C79000AC090020480A0020036810B5186B002877
:10C7A0000ED0CB0702D50368002B09D08B0702D52A
:10C7B0004368002B04D04B0708D58368002B05D1B4
:10C7C0000349044818F024F8F3F701FD10BDC046F2
:10C7D0008E9203004CDB0200F0B5012189B001907C
:10C7E000FFF7DAFF80210600490004A81BF01AFBBE
:10C7F00080240023069D6400009303AB22002900DF
:10C8000001983768B847431C1AD103990B290FD1F7
:10C81000009B1848002B09D0009B17480593337BD9
:10C82000DB0700D4154804A9FBF722F909B0F0BDD5
:10C83000012349001943124817F0E3FFF3F7C7FC3F
:10C840000028E9D0009B1B180093844202D9241AC7
:10C850002D18D2E7802104A849001BF032FB051EE9
:10C8600004D108490648F8F7F9FEE7E78024640098
:10C87000C3E7C0464CCA0200DC14030090E7020084
:10C880004CDB0200BB920300F0B50E008BB004003D
:10C8900001213068FFF780FF0700012C04D13068C8
:10C8A000FFF79AFF0BB0F0BD706801F0B1FC030018
:10C8B00000900133F3D001253B7B2B4275D0010062
:10C8C000040006A81BF0AEFA002303950193002C88
:10C8D0005FD0210006A81BF00DFB011E05D14249C7
:10C8E0004248F8F7BBFEF3F772FC3D6805AB220047
:10C8F0003068A8470500431C16D1210006A81BF08C
:10C9000065FB05990B2908D1079B0093002B40D1AB
:10C9100006A81BF0B2FA3648C4E7012349001943C0
:10C92000344817F06EFFDEE784422CD8089B079C42
:10C93000029302239C460198019A029B9B5C039AF6
:10C9400059B2002912DA19001F256246A943C029ED
:10C950000CD01900103D0322A943E02906D004326F
:10C960009343F03B1A00511E8A410432019BD318B5
:10C970000193A34212D8009B0198013B0093A0426F
:10C98000DAD3009CA3E7211A06A81BF01FFB002D99
:10C99000CCD1194806A9FBF76BF883E7E443009B69
:10C9A000E418019B0190E41891E7009906A81BF098
:10C9B00050FA05AB009A089930683C68A047431CC0
:10C9C0000AD106A81BF059FA059909480B2900D18C
:10C9D00068E749002943A3E73B7B079006482B42C1
:10C9E00000D1064806A9D6E7AD92030098DA020006
:10C9F0004CCA02004CDB0200DC14030090E702008A
:10CA00007FB50C00060001212068FFF7C5FE022259
:10CA1000050001A9606801F0B5FD029A022E06D951
:10CA2000A06801F0F5FB029A824200D902006B4631
:10CA30002D6801992068A847431C0BD1009908482C
:10CA40000B290AD0012349001943064817F0D9FEE3
:10CA5000F3F7BDFB43000120184304B070BDC0468E
:10CA60004CCA02004CDB0200F0B589B00191019B79
:10CA7000040001211868FFF78FFE0600012C1AD967
:10CA8000019B5B685C10631C15D0210004A81BF09F
:10CA9000C9F9631C03D0631E002C36D01C00012191
:10CAA00004A81BF027FA071E0CD11E491E48F8F7F0
:10CAB000D5FDF3F78CFB0124102104A81BF0B2F97B
:10CAC0006442E6E70100019803AB01220068356883
:10CAD000A847431C13D103990B2909D1059B019346
:10CAE000012B0ED104A81BF0C8F9104809B0F0BD05
:10CAF0000123490019430E4817F083FED9E70028A7
:10CB00000CD1012104A81BF061FA337B0948DB0733
:10CB100000D4094804A9FAF7ABFFE7E73B780A2BF2
:10CB2000B7D1F2E7AD92030098DA02004CCA0200D6
:10CB30004CDB0200DC14030090E70200F7B50E00A6
:10CB4000022104001700FFF727FE01AB45683A00F9
:10CB500031002000A847431C0BD1019907480B293D
:10CB60000AD0012349001943054817F04AFEF3F79C
:10CB70002EFB430001201843FEBDC0464CCA0200F4
:10CB80004CDB0200014B58687047C046AC090020DE
:10CB9000014B18687047C046AC090020F0B5194E2B
:10CBA00087B03368050000200C00019317F0D0FD1A
:10CBB0003060009020681AF0ACF8019B07003360E9
:10CBC000114E022D03D0A06801F03AFA06002100B0
:10CBD00063680831A81E0393F6F742F8009B04909F
:10CBE0000593002203AB0321300002F04DF8074B00
:10CBF00004009F4203D0010038001BF0CEFC20004F
:10CC000007B0F0BDAC090020C8CF02004CCA02003A
:10CC1000F8B50326050007003540022D16D10E4B4E
:10CC20000340062B12D0FF23DB05C418B443201C9D
:10CC300000210DF08BFC002806D080231B06E41891
:10CC4000B443064B2C43E7183800F8BD380003F016
:10CC5000FDF90700F8E7C046070080FF000080806C
:10CC600010B502F00BF90400200002F053F900287F
:10CC700001D1044810BD01F009FC0028F4D102489C
:10CC8000F8E7C046AC090300A409030010B502F0A0
:10CC9000F5F80400200002F03DF9002801D1044815
:10CCA00010BD01F0F3FB0028F4D00248F8E7C046BD
:10CCB000A4090300AC09030007B5044B019000224E
:10CCC000694602200093FCF70DF90EBD0604000032
:10CCD00010B501F039FA034B002800D1024B1800BF
:10CCE00010BDC046AC090300A409030037B501F02C
:10CCF0008FFA01AB7F2806D8012118700122180095
:10CD0000FAF7ECFE3EBD1F49820988420BD840214C
:10CD100049420A431A703F22024080204042104399
:10CD200058704231EAE7184C010BA0420ED820247B
:10CD300064422143197080215F34494222402040DF
:10CD40000A43014399705A700321D7E70F4CA04260
:10CD500012D81024850C64422C431C703F2580247B
:10CD6000294064422A4028402143224320435970ED
:10CD70009A70D8700421C1E70549064817F048FDAC
:10CD8000F3F725FAFF070000FFFF0000FFFF100088
:10CD9000C992030044DD020010B5020002490A20D6
:10CDA00002F0F8F810BDC046BE04000010B5020045
:10CDB00002490A2002F0EEF810BDC0463E05000010
:10CDC000F0B585B0019202900D0000223149019822
:10CDD0000393FEF7B9FE0090002801D0436800934A
:10CDE000029B012B10D0002634000196029B9E422C
:10CDF0001FD0009B002B3DD12F68002C40D12C6808
:10CE0000019701360435F1E70024286802F036F86E
:10CE100027000290029802F07DF8051E0CD1002C2C
:10CE200007D122001C490198FEF78EFE00281BD076
:10CE30004468200005B0F0BD009B2E00002B04D0FC
:10CE40002900180019F06CFF0600002C09D03A00E8
:10CE50003100039802F09EF8104B984201D0250053
:10CE60003E002C003700D5E70D490E4817F0D0FCE6
:10CE7000F3F7ADF92968009819F052FF0700BCE7F5
:10CE8000019A3900039802F085F8044B9842B8D112
:10CE9000B5E7C046D60600001E050000AC09030039
:10CEA000EA92030044DD020037B501A90500FBF753
:10CEB000C3FA1E4B04002B40062B05D0AB072AD12A
:10CEC0001B4B2A689A4226D1019920001BF0AFF92A
:10CED0000190012822D1207843B2002B04DB0120ED
:10CEE00023785B0018433EBD7F23013418403F3B4D
:10CEF000034208D13F22237819009143802905D0AD
:10CF00001AF010F8EFE798435B10F1E78001134047
:10CF100001341843EFE7019B012BE0D0019A05494A
:10CF20000548F8F79BFBF3F752F9C046070080FF6E
:10CF3000DC14030003930300CCDC0200F0B5140002
:10CF400087B002900391002223492000FEF7FCFDE8
:10CF50000022050021492000FEF7F6FD0123040010
:10CF6000049305931E4F002D07D068681D4B98420F
:10CF700003D004A9FBF760FA07001B4E002C07D072
:10CF80006068184B984203D005A9FBF755FA0600D4
:10CF90000024029B154D9C420AD10023059A01935F
:10CFA000009331002800FCF719FC0E4807B0F0BDD3
:10CFB000002C07D00023049A019300933900280025
:10CFC000FCF70CFC0399A3000022C958280001F0CB
:10CFD0004FF80134DDE7C046EE050000F60500001D
:10CFE000799B03004CCA020007B00300B4EA0200B8
:10CFF0007FB50D4D0400A84213D00C4E0122010054
:10D00000300001F035F80A49300018F009FA04231D
:10D010000293084B0394DB6902AA0321064801939B
:10D020009847280004B070BD4CCA0200B4EA020060
:10D0300007B0030020100300ECFC020010B5040050
:10D0400086B06A4602A8102105F0D0FF0122210017
:10D05000684601F00DF802A90248FAF709FD06B08A
:10D0600010BDC046DC14030070B50C68E30726D47D
:10D07000A30703D1254B22689A4220D0012820D94A
:10D08000486801F0C5F80600200001F025F9051CEC
:10D0900030000EF021FA011C1D4810F0C1FE011CE9
:10D0A000041C281C0DF024FF10F066FB211C0DF061
:10D0B0002FFD032302249843164B0443E418200059
:10D0C00070BD200001F008F9051C10F055FB061C8E
:10D0D0000EF0E2F9311C0400281C0EF029F8FC21A6
:10D0E0008905051C0DF02CFA002803D0013401231A
:10D0F0009C4306E0BF21281C09060DF021FA0028F8
:10D10000F5D1200019F00EFF0400D8E7E81F030056
:10D11000000020410000808013B504000800FAF7E9
:10D12000FFFC6A460100200001F02CFE009B024833
:10D13000002B00D1014816BDAC090300A40903006F
:10D1400037B50024022800D98C6848680D68FAF7C2
:10D15000E7FC0A4B0100002C00D0094B28006A466E
:10D1600098470098002806D001990400002902D0B1
:10D17000FEF71EF8040020003EBDC046E5ED0000AD
:10D1800085ED000070B5040008001500FAF7C8FC32
:10D190002A000100200001F04DFE014870BDC0468C
:10D1A0004CCA020010B501F08FFE002804D10348DC
:10D1B00017F021FBF3F70BF810BDC0460CDC0200A2
:10D1C00030B50B0085B01400012805D90A490B4879
:10D1D00017F01EFBF2F7FBFF09480121C26801921C
:10D1E000019D0022A8472200039003A90120FEF719
:10D1F000ABF8039805B030BD3D930300CCDC0200D2
:10D2000060EC0200F8B50E0000280FD10400294B95
:10D210001D680021080018F052FB00270600002DB1
:10D2200034D10025002C40D13000F8BD08688307B8
:10D2300015D10268204B9A420DD11AF020FC05004E
:10D24000306800F0FDFE1D4BC26800249A42E0D118
:10D2500034680434DDE71A4903008A4202D000F042
:10D26000EFFE03009D6B002DEAD0164B2A689A4210
:10D27000E6D00025E4E7EA68FB009958002904D0CD
:10D28000042902D03000FDF7FDFF0137AB689F4253
:10D29000F1D3C6E7A268EB009958002904D004290D
:10D2A00002D03000FDF7EEFF013563689D42F1D3F7
:10D2B000BAE7C046AC09002020100300213200006C
:10D2C000C8CF020094D6020073B50090000C431E34
:10D2D00001910A2B1AD80126330083400C4A118889
:10D2E0000B439BB213800B4B1A780F2A0EDC1A7873
:10D2F00019783240F14092009040074C655C284319
:10D30000C0B260541A789219D2B21A7073BDC04676
:10D31000080900202C09002024090020094A70B5C2
:10D320001378002B0CD1084D2C78E4B2002C07D1D7
:10D330000068013313702B7003685B6898472C708A
:10D3400070BDC046220900202309002010B504004A
:10D350000430FFF7E3FF60681DF004FB034B80001F
:10D36000C3580620DB00184310BDC046C8FF0200AA
:10D3700010B5FAF7D5FB0023074A9900895888426F
:10D3800008D001330C2BF8D10449054817F040FAB6
:10D39000F2F71DFFD8B210BDC8FF0200689303006A
:10D3A00044DD020070B504000800FFF7E1FF05004E
:10D3B000201DFFF7B3FF60681DF0D4FA024B8542D1
:10D3C00000D0024B180070BDAC090300A409030093
:10D3D00070B504000800FFF7CBFF0500201DFFF724
:10D3E0009DFF0123AB40064A064811880B4200D13D
:10D3F00005481188994311800022044B1A7070BDB2
:10D4000008090020AC090300A40903002C0900202E
:10D41000F8B50430FFF782FF124C13482378002B35
:10D420001FD020780021C0B2F5F71AFC0126002297
:10D430000E4F2378934212D915005308FB5C3540F8
:10D44000AD002B410F252B40094D9B005B59062554
:10D450009100DB0041182B438B600132E9E7002388
:10D460002370F8BD2C090020F8CD0200240900200B
:10D47000C8FF0200C02307B5002200931B21024B06
:10D4800002480AF031FF07BDC9D20000C4050020E0
:10D4900070B504000D00104917F0C2FF6968012241
:10D4A000200000F0E5FD0D4E2000310017F0B8FF20
:10D4B000A9680122200000F0DBFD3100200017F0F8
:10D4C000AFFFE9680122200000F0D2FD04492000EE
:10D4D00017F0A6FF70BDC046789303000035030027
:10D4E0004A95030070B5060010200D0014001BF0D3
:10D4F00008FD034B466085600360C46070BDC04694
:10D50000EC00030001220020074B08495A60086024
:10D51000A821DA60064AC9005A5006495A50043117
:10D520005A5005495A507047009000400C9C0040EA
:10D53000FCFF0000440500004C050000034B0448BC
:10D540001B78002B00D103487047C0462E090020ED
:10D55000AC090300A4090300F8B5A826324A334BEE
:10D56000F600196813680420CB18C9181160304AF6
:10D570008C4612781B11170009112E4A2E4C2F4D84
:10D58000002F47D0002B39DA9051C31AA920C000D0
:10D59000135081239B00002936DA591A1351515137
:10D5A0000123274CD3602378002B21D03F2225482C
:10D5B000254B01689B6F01310A409D5C1C4B1B7819
:10D5C000002B01D0803D6D001C23026062466B433E
:10D5D00008339B1A154A9B1013601F23194007D16B
:10D5E0001A4B1A78002A03D019481970F2F764FF11
:10D5F00001232278042053402370F8BDA927043367
:10D60000FF00D0519351C4E7535181239B00C918A7
:10D610001151C5E7043390515351A9208123C00013
:10D620009B001350F3E7C0462C0300203C0300206E
:10D6300045020020009000404C0500004405000019
:10D640002D09002030030020AC09002046020020F4
:10D65000436A020030B585B001220400080001A928
:10D6600000F090FF029A202A00D920220023019D79
:10D67000934204D0E85CE11808710133F8E70148EF
:10D6800005B030BD4CCA020070B50400080015009A
:10D6900000F0BEFD0E491F2815D8002D05D10D49FB
:10D6A0000D4817F0B5F8F2F792FD2418042D04D1B7
:10D6B000012023795B00184370BD280000F0A8FD0D
:10D6C000FF2802D905490648EBE720710548F3E732
:10D6D00091930300A5930300CCDC0200CA930300DE
:10D6E00044DD02004CCA02000123A022834010B591
:10D6F000134CD20513510300C133124CFF339B006E
:10D700009C50114B8900C918A223DB00CA580F4C4A
:10D7100000022240CA50F82252011040C022CC58C8
:10D720009202224310430322C850CC580848224397
:10D730002043C850C046C046C046CA5010BDC0466F
:10D740000C0500000303000000600040FFE0ECFF58
:10D75000031F0000A0221E21114BD20070B59C585F
:10D76000104D8C439C50A324E4001D510E4C0F4DD2
:10D770000F4E5C5104355E510E4D80005C51A52466
:10D780000D4DE4001D51084C0C4D00190C4C185166
:10D7900004341D510B4C185198580143995070BDD9
:10D7A00000F0014040910040006000401C05000076
:10D7B0004491004024050000489100404C910040F5
:10D7C0002C0500003405000070B50D00040006F0C3
:10D7D00029F8134E2800310006F048F831002000E7
:10D7E00006F044F80F4BA0221C600F4BD2051D60C1
:10D7F000607901242100814026000C4BD1506979C9
:10D800008E400021D650FFF76FFF68792100FFF7A7
:10D810006BFF2000FFF79EFF054B1C7070BDC046DC
:10D820002016030034030020380300200C050000FC
:10D830004502002010B504000A4906F017F80A4B0B
:10D84000A0211C6001236079084A8340C9058B50E0
:10D850000021FFF749FF0020FFF77CFF0022044B67
:10D860001A7010BD20160300340300200C050000C0
:10D8700045020020F8B50025FFF744FE214B2800A3
:10D88000DD67F2F7E7FDA0221E201F4B1F491D7028
:10D890001F4BD2001D601F4B1F4C1D608B581F4F2C
:10D8A00083438B50A223DB00E2581D4E3A40E250E6
:10D8B000E2581C493243E2500122E5501A4B1868E5
:10D8C00043799A401300A022D205535005F0B8FFC7
:10D8D000164B1B78AB4213D0154B1249E258174038
:10D8E000E750E25816430122E650E550114B186804
:10D8F00043799A401300A022D205535005F0A0FFAF
:10D90000F8BDC046AC0900202E09002000F00140FF
:10D910002C0300203C03002000600040FFE0ECFFEF
:10D92000001F03000C050000340300204502002006
:10D930001405000038030020F0B53A4E8DB0F36FA7
:10D940000500002B03D1FFF795FF0DB0F0BD0028B7
:10D9500001D0FCF7B5FA6846F2F71EFC00281DD18D
:10D96000F06F01F0B1FA0400F2F72CFC002D01D0A9
:10D97000FCF7B0FA20222C4B1D68B36F6D110135F6
:10D980006D0115405D19002C2CD121002800F46791
:10D990001DF0C2FD0122254B1A70D6E7002D01D0E3
:10D9A000FCF798FA019B22491868F5F701FE00245C
:10D9B0000500A042DED1019F380000F041FB1D4B65
:10D9C00098420BD129000120F5F74AF92A000400FA
:10D9D000F8601F211848FAF781F8A060019B002425
:10D9E0003363C7E7200000F02BFB144B984207D0AD
:10D9F000002313491348F36716F00AFF3063A4E7C6
:10DA000063682B60A3686B60E368AB602369EB60BD
:10DA100063692B61A3696B61E369AB61236AEB61A5
:10DA2000B8E7C046AC0900203003002046020020C1
:10DA30000CDC020098DA0200F03903002C0203002B
:10DA40007F930300CCDC020010B5FFF713FF014801
:10DA500010BDC0464CCA0200F0B589B00493704BAB
:10DA600003901B780E001500002B01D0FFF702FF7A
:10DA70006C4B1A78002A07D16B4C4020E2670132C8
:10DA80001A701BF03EFAA06780270122674BBF0087
:10DA9000674CDF67674BE250FFF734FD0023664AAF
:10DAA000F021A3500432A3500832A350C22209032C
:10DAB0009200A150E351614F0594BE4200D09FE017
:10DAC000B54200D096E05E4D07AC280005F0C2FEDE
:10DAD000002805D001235B492800237005F0C6FE0D
:10DAE000594D280005F0B6FE002805D00123554900
:10DAF0002800637005F0BAFE544D280005F0AAFE18
:10DB0000002805D001234F492800A37005F0AEFE80
:10DB1000A0270024FF0507ABE35C002B33D10134C1
:10DB2000022CF8D1464808F0E5F8FFF783FE0026FE
:10DB30000124039801F0A2F93F22454B3A4D1E7093
:10DB4000444B80211C70444BE8671A60A86F12197F
:10DB50001DF0E2FC3000FFF7EFFE404B304F1C6041
:10DB6000059B50221C603E4930003C70F2F73EFCA1
:10DB7000049BB34252D03B78002B4FD02B6B002B31
:10DB80004CD120BFF7E7374BA200D6580322737958
:10DB9000651CC133FF339B00DA5107ABEB5C002BF4
:10DBA00024D0304BAA00D3580193042300930122C0
:10DBB00073799A40A123DB00FA50019B05331800CA
:10DBC000029318F01EFF012810D173799840264B5C
:10DBD000F850029818F015FF002807D1009B013B70
:10DBE0000093002BE3D10199300014E00135032D9F
:10DBF000D3D194E71D491E4816F00AFEF2F7E7FA62
:10DC0000300008F077F80400BD428ED0280008F0FC
:10DC100071F801002000FFF7D7FD88E709B0F0BDDB
:10DC20002E0900202F090020AC09002004E100E0AB
:10DC300000900040FC0F0000040500004CCA0200E8
:10DC4000141E0300F01503005C1E03006C1E03008D
:10DC50002D09002046020020300300200C9C0040CB
:10DC600059D50000E40103000C050000DD9303001A
:10DC7000CCDC020010B5084B86B002AC00930194D6
:10DC80000423F5F727FE02982379E268A168FFF7DD
:10DC9000E3FE024806B010BDF00103004CCA0200CA
:10DCA000014B1878C0B270472E09002010B524200F
:10DCB0001BF027F90400044B202208C080211DF02E
:10DCC0002BFC200010BDC0462C020300F8B5050057
:10DCD00008000E00170000F0B3F9324B984201D053
:10DCE0000020F8BD681F0F28FAD80CF041FA080888
:10DCF00035F9F9F9F9F9F9F9F9F9F9333358FFF781
:10DD0000D5FF04230400F25CE2540133242BFAD142
:10DD1000380000F095F9234B9842E1D10121052DFF
:10DD200005D0123D691E8D4101216D422943042217
:10DD3000FF20BB5CA55C803B4B435B19FF2B03D9E9
:10DD40000500DB179D432B00A3540132242AF0D198
:10DD50002000C6E73400DBE7FFF7A8FF0423040038
:10DD6000F25CE2540133242BFAD1380000F0B4FA0B
:10DD70000F2118F06BFE2100FF25221D243113789E
:10DD8000803B4343DB138033FF2B03D92E00DB178B
:10DD90009E433300137001329142F0D1D8E7340032
:10DDA000E3E7C0462C02030070B50D0000F094FAC2
:10DDB000041C280000F090FA211C0DF0B9F9051C94
:10DDC00018F012FF011C281C0DF092F8211C0CF019
:10DDD0000DFD0323020002209A43024B1043C0189A
:10DDE00070BDC0460000808010B518F0FDFE032312
:10DDF000020002209A43024B1043C01810BDC046D7
:10DE000000008080F8B5070008680D0000F000FAF7
:10DE10000600012F06D1002826DD04F02FF919F0A5
:10DE200081F8F8BD686800F0F3F9841B022F06D171
:10DE3000864219DA200004F021F98019EFE7A8687A
:10DE400000F0E6F9051E0ADD2018013829000CF063
:10DE500041FA002808DD04F011F96843EDE70028D5
:10DE600002D020180130F1E7024816F0C4FCF2F7A6
:10DE7000AEF9C04644DD020010B5074C002802D0C0
:10DE80000868A04203D104F019F9200010BD00F089
:10DE9000EBF904F035F9F8E74CCA020010B50400BC
:10DEA00000F028FB00F0B4F9002804DC074816F065
:10DEB000A2FCF2F78CF904F0E1F819F033F804222F
:10DEC0000100200000F02CFB10BDC0469CD90200D0
:10DED00010B5024816F08FFCF2F779F944DD020024
:10DEE000F0B5114B87B003AD40C9013800930195DF
:10DEF0000323F5F7EFFC68680C4C1E27A04202D004
:10DF00001AF043FB0700A8680022A04202D01AF0D2
:10DF10003CFB0200706803990771427108F070FAC7
:10DF2000200007B0F0BDC0467C0303004CCA0200CD
:10DF300030B5124B8BB003AC20C90138009301946B
:10DF40000323F5F7C7FC616806A819F082FF039B5D
:10DF5000089A5900237A00936868079B09F0D2FB5E
:10DF6000021E05D006490748F7F778FBF2F72FF9AC
:10DF700006A90548F9F77CFD0BB030BDA0030300EE
:10DF8000FF9303004CDB020090E7020030B5114B19
:10DF900089B002AC20C90138009301940323F5F73E
:10DFA00099FC012205A9606800F0ECFA029B059A31
:10DFB0005900237A00936868069B09F0EDFB021E66
:10DFC00005D005490548F7F749FBF2F700F9044881
:10DFD00009B030BDC4030300229403004CDB0200EF
:10DFE0004CCA0200F7B50191114904001700002541
:10DFF00017F016FA7B689D4204D30E49200017F0F3
:10E000000FFAF7BD002D03D00B49200017F008FAD6
:10E01000019BAE009A5909492000BE1917F0CBFAAE
:10E020000122B168200000F023F80135E2E7C04684
:10E030007D9303004A9503000035030046940300D6
:10E04000074BC2070AD4074A074B0240062A05D0ED
:10E050000322064B0240022A00D0036818007047D2
:10E06000E81F0300070080FFDC140300381B0300D7
:10E0700070B50D0004001600FDF7C4F82800FFF786
:10E08000DFFF8368002B04D032002900200098476E
:10E0900070BD42680249200017F08DFAF8E7C046CB
:10E0A0008E95030010B50A0001000248FFF7E0FF5B
:10E0B00010BDC046B4EA0200F7B5050008000E0026
:10E0C00016F0AAFB002812D001AA69463000F7F723
:10E0D0006DFB009B002B0AD01649280017F0A0F911
:10E0E000009C154BE71EE418A400002F09DA31004C
:10E0F00028000222FFF7BCFF2800104917F090F912
:10E10000F7BD019A0E4913195B681259280017F0E0
:10E1100052FA019B1B199A68002A06D10749280068
:10E1200017F07EF9033F0C3CDFE70649280017F0A3
:10E1300042FAF7E74C950300FDFFFF3F07B00300ED
:10E14000709503008595030010B50400FFF778FF74
:10E15000054B0069984203D0431E9841C0B210BDE0
:10E16000200016F036F9FAE7AD33000070B505006F
:10E170000C0001208D4203D0214B9D4201D1002093
:10E1800070BD9942FBD001231D4204D01942F6D143
:10E190002B000D001C002A001A4B1A40062A05D03D
:10E1A000AA0711D1184A296891420DD12340062BA4
:10E1B00005D0A307E3D1144B22689A42DFD1210096
:10E1C0002800FAF7E5F8DBE72340062BD7D0A307B2
:10E1D00003D10D4B22689A42D1D02800FFF730FFBF
:10E1E0008369002BCBD0220029001B2098470028F0
:10E1F000C5D0064BC01A42424241D0B2C0E7C04629
:10E200004CCA0200070080FFDC140300AC090300C5
:10E21000104B10B5984219D00F4A0123904217D0E5
:10E22000184201D0184110BD830706D10B4B02687C
:10E230009A4202D101F06AFFF5E718F02EFD084975
:10E2400002000848F7F70AFAF1F7C1FF0020EAE7F1
:10E250001800E8E7A4090300AC090300E81F030065
:10E2600013950300CCDC020010B5C30705D4830767
:10E2700006D1054B02689A4202D118F090FE10BDFB
:10E28000FFF7C6FFFBE7C046E81F03000F4B70B562
:10E290000D000124984204D100230B6023001800D4
:10E2A00070BD0B4B984201D10C60F7E7030023408F
:10E2B00002D040102860F1E78207F0D1054A0168DA
:10E2C0009142ECD101F022FFF4E7C046A40903001B
:10E2D000AC090300E81F0300184B10B5984228D082
:10E2E000174B984227D0C30703D540100DF0F4F820
:10E2F00010BD0323184206D1124A0168914202D18F
:10E3000018F056FEF4E70340022B09D10E4B0340F0
:10E31000062B05D0FF23DB05C01803239843E7E74E
:10E3200018F0BBFC094902000948F7F797F9F1F723
:10E330004EFF0020DCE7FE208005D9E7A40903009A
:10E34000AC090300E81F0300070080FFF9940300F5
:10E35000CCDC020010B583070CD103680A4CA34241
:10E3600002D115F045FF10BD084CA34202D117F0B1
:10E37000BDFAF8E718F091FC054902000548F7F7E7
:10E380006DF9F1F724FFC04600CE020060EC0200F8
:10E39000A9940300CCDC020013B50C0001A9FFF71F
:10E3A000D9FF019BA34206D0220003490348F7F797
:10E3B00055F9F1F70CFF13BDCC94030044DD0200C6
:10E3C000F7B505000C0017001E00D3070ED5571037
:10E3D0000197019B002B1FDA1B190193002E1DD002
:10E3E000002B15DA002301930198FEBD01A910004E
:10E3F000FFF74CFF0028ECD138006C6818F04DFC9A
:10E40000220003000B490C48F7F728F9F1F7DFFE6B
:10E410009C42E9D20194E7E7002EF9D1019B002B41
:10E4200001DB9C42E0D86A6804490548F7F716F911
:10E43000ECE7C0466F940300CCDC02009394030029
:10E440009CD9020010B50400830710D10D4B02685F
:10E450009A420CD10C4B0340062B06D1C00818F091
:10E46000F6F943000120184310BD8068F9E7200049
:10E47000FFF7E6FD4369181EF6D0210001209847FA
:10E48000F2E7C04690E70200070080FF164B70B528
:10E49000040000209C4203D0144DAC4201D1012065
:10E4A00070BD134B00209C42FAD0012626408642C4
:10E4B00003D06010431E98410DE02000FFF7C0FD1F
:10E4C0004369002B09D0210030009847002804D070
:10E4D000401B43425841C0B2E2E72000FFF7B2FFC1
:10E4E0000028DCD00138E5E7A4090300AC090300EB
:10E4F0004CCA020010B50400FFF7A4FF002809D1A0
:10E50000200018F0CAFB044902000448F7F7A6F8F7
:10E51000F1F75DFE10BDC0462B950300CCDC020078
:10E5200070B504000D001600FFF78AFD036A002B8A
:10E5300005D03200290020009847002818D10D4D41
:10E540002000002E08D118F0A8FB02000A4928007C
:10E55000F7F784F8F1F73BFE042E04D118F09DFB89
:10E5600006490200F3E718F098FB05490200EEE7C0
:10E5700070BDC046CCDC020093950300BE9503003D
:10E58000DF95030010B518F09EFB002805D1034964
:10E59000034816F03DF9F1F71AFE10BD4A94030046
:10E5A000CCDC0200F0B5456887B00393AB6805A8E2
:10E5B00017000291059319F049FD060005A819F00E
:10E5C00045FD03000320584333000933C018800081
:10E5D0001AF097FC04000A4BAA6803606B682900D4
:10E5E0004360059B06629B1AC360039B083000933F
:10E5F000029A3B0004F08EFF200007B0F0BDC04639
:10E60000A804030070B5050088680C0016F0BCFC77
:10E61000230002000249280016F0CDFF70BDC0465D
:10E620000C96030010B5024816F0E5F8F1F7CFFD9F
:10E630000CDC020010B5040008201AF062FC024B4A
:10E640004460036010BDC046E4040300F8B5040054
:10E65000C0681D00002801D11860F8BD2000636962
:10E660002030834208D1154B994206D014491548F1
:10E6700016F0CEF8F1F7ABFD19602000124E63687A
:10E680001100083077687360F5F754FE7760012851
:10E6900007D00023E36002280AD063691B682B605F
:10E6A000DBE763691B682B60002BD6D1E360D4E7FE
:10E6B000236A07339B00E4186368F0E74CCA020042
:10E6C0004A960300CCDC0200AC09002013B501AB74
:10E6D0001400FFF7BBFF01280ED0184C02281CD0F5
:10E6E000019BA34228D0002B26D001AA0121144867
:10E6F00016F07BF8F1F76BFD002C0CD02000FFF733
:10E700009FFC1049F4F754FF002804D00E490F482D
:10E7100016F07EF8EEE7019816BD0198FFF790FC21
:10E720000749F4F745FF002801D10198E2E7019875
:10E73000F6F774FFA042F8D10020EDE74CCA0200C2
:10E740000CDC0200E8D802002A960300C4DB0200B9
:10E7500010B50C0002280BD1486801F053F80649A7
:10E7600002002068FFF7B2FF002803D1FFF75AFF2D
:10E770008868F2E710BDC0464CCA020010B50022FE
:10E780000149FFF7A3FF10BD4CCA020013B5124C9C
:10E7900001AB124A2100FFF759FF012803D00228DC
:10E7A00007D0200016BD0E490E4816F031F8F1F7DB
:10E7B0000EFD0198FFF744FC0B49F4F7F9FE002821
:10E7C000EFD10198FFF73CFC0849F4F7F1FE00286F
:10E7D000E7D10198EBE7C0464CCA02003CD70200E3
:10E7E0002A960300C4DB0200E8D802000CDC020019
:10E7F000F7B50125284B070001911D70FFF708FDB3
:10E80000102805D02549264816F002F8F1F7DFFC5C
:10E81000A1220021234BD200A22699500922F60002
:10E820009A51802080228000D2021A501E481F4C2C
:10E830001950A9211F20C9005850C12189005A50E0
:10E840008023C022C220DB005200A3508000225847
:10E8500017491140C02212040A432250C02252001C
:10E86000A35038002360FFF7D3FC0300A0220C2143
:10E87000C133FF339B00D20599504023C12223604E
:10E880000C4B000218430C4B920098519D500B4BBF
:10E89000019A0B481A60FEBD220B002080960300EF
:10E8A000CCDC020000A000400405000000E100E014
:10E8B000FFFF00FF0100020000600040F80A002096
:10E8C0004CCA02000B4B0C481A68C16C013210B5DF
:10E8D0001A600A4B012907D1C124A4001C59640302
:10E8E00002D50024C464D960C82A02DD01225A601E
:10E8F000DA6010BD48030020FCA0004000A00040EA
:10E90000F7B5474B5A680193012A22D1C1234549E3
:10E910009B00CB5813421CD0434C444D23683C2BE6
:10E9200009DD002342490B8042494A60CA60424ADD
:10E9300023602B7013702B78002B0BD101223D49E3
:10E940002A702360CA600A603C4A13600023019A5F
:10E950005360F7BD3A4E226833783A4F0133337033
:10E9600000230D2A35D1337023603349314B0C3AE3
:10E970000A70DA603B78012B06D132783249013ACD
:10E9800093400A6813430B603378202BDED10023B9
:10E9900001212E4A1370274A5160D1602A4A236010
:10E9A0001068234C010C218029492B70088080B20B
:10E9B000136018F0B7FA274D2860208818F0B2FAD3
:10E9C000254B02001860254B2968186818F0B0F92B
:10E9D000BCE7012A04D117492360CA603B70C9E72C
:10E9E000022A04D123600123124AD360F6E70B2ADE
:10E9F000C0D101210F4A23605160D160134A2B70AE
:10EA000013785B18DBB21370052BB3D9124B1A685D
:10EA1000104B1968114B186818F08AF9AAE7C0461C
:10EA2000FC600040006000404803002033090020E3
:10EA30000C09002000A00040310900204403002000
:10EA40003009002034090020400300203209002052
:10EA50000A090020FC0A0020000B0020F80A002010
:10EA600070B5FDF7EFFD0B4C00262300A8331E60A8
:10EA7000266303F039FC084D01212800F6F7F6FC67
:10EA800028005E226E2115F09BFE6560256066649D
:10EA900070BDC046AC090020E009002070B5062416
:10EAA000134EC3001C437368002205002100181D8B
:10EAB000FDF74AF8021E18D1706C002807D0043008
:10EAC0002100FDF741F8002801D0406870BD002208
:10EAD00021000848FDF738F8021E06D12A00064931
:10EAE0000648F6F7BBFDF1F772FB5068EEE7C0464B
:10EAF000AC090020FCFC02009D970300D4DA020060
:10EB00000A4B10B5040018685B6898420AD00621C9
:10EB1000E300194304300022FDF716F8002801D065
:10EB2000406810BD2000FFF7B9FFFAE7AC090020EC
:10EB3000074B10B5586C002801D1064810BD0430B1
:10EB400000222621FDF700F80028F6D04068F5E7FE
:10EB5000AC09002078FB02000A00C100062010B5B5
:10EB6000024B0143186815F02BFE10BDAC090020C4
:10EB7000062110B5034BC0000143186815F02AFEAA
:10EB800010BDC046AC0900200A00C100062010B527
:10EB9000024B0143586815F013FE10BDAC0900206C
:10EBA000062110B5034BC0000143586815F012FE52
:10EBB00010BDC046AC09002070B505000C00062849
:10EBC00006D10800FFF762FC00280ED0274870BD70
:10EBD000012001421AD04B10042D08D0052D13D06E
:10EBE0000800002DF3D1002BF0D02148EFE7C02220
:10EBF0001206934204D18020C00518F093F9E6E78D
:10EC00005B425B001843E2E7DB43FAE7022D12D1D7
:10EC1000184B0B40062B08D08B070CD10A68164BFB
:10EC200092699A4207D1486802E0C80817F00AFEC4
:10EC300043000120E6E72000FFF702FA4369002BBA
:10EC40000DD10E4BAD002000ED5818F026F82A002B
:10EC500003000B490B48F6F701FDF1F7B8FA210064
:10EC6000280098470028B2D1EBE7C046A40903006A
:10EC7000AC090300070080FFF189000004D0020006
:10EC800029980300CCDC0200F7B5040001911600BE
:10EC90001F00FFF7D5F90569002D09D1200017F0F5
:10ECA000FCFF064902000648F6F7D8FCF1F78FFA98
:10ECB0003B00320001992000A847FEBD6B350300E0
:10ECC000CCDC0200F8B504000D0017001E0000297E
:10ECD0000BD01868FFF7B4F96368984205D006496D
:10ECE000064815F095FDF1F772FA33003A00290055
:10ECF000A068FFF7C9FFF8BD92960300CCDC0200C4
:10ED0000F8B506000F0014001D00930714D1136816
:10ED1000174A934202D163682B60F8BD154A9342AB
:10ED200007D1002802D0FFF78BF90700636888C578
:10ED3000F3E7114A934201D12C60EEE75B681A00B9
:10ED4000F23A012A01D9F02BF6D1002E0ED1200083
:10ED5000FFF776F9094B984208D10C201AF0D1F848
:10ED6000074B4760036084602860D6E750C5D4E74E
:10ED700050CF020014CF0200C8CF0200B4E6020058
:10ED800064050300F8B500231360536006000D000E
:10ED90001400FFF755F90700102D05D1836A002BE9
:10EDA00002D00F4B48C4F8BDFB69002B04D02200F1
:10EDB000290030009847F6E7B86B0028F3D0062109
:10EDC000ED00294304301A00FCF7BEFE0028EAD00B
:10EDD0004268230039003000FFF792FFE3E7C046A6
:10EDE00074FC020070B5160004000D00FFF7CAFFA6
:10EDF0003368002B15D10B4EA3070BD10A4B2268A9
:10EE00009A4207D12B00626808493000F6F726FCC9
:10EE1000F1F7DDF9200017F040FF2B000200044954
:10EE2000F3E770BDE0D70200C8CF0200B697030039
:10EE3000DD97030073B504000D001600FFF700F91D
:10EE4000C369002B09D004220196009229006A466A
:10EE500020009847009B002B0AD0200017F01DFFD0
:10EE60002B00020003490448F6F7F8FBF1F7AFF96D
:10EE700073BDC046DD970300E0D7020013B5040060
:10EE8000FFF7DEF8436A002B11D16A461A212000F1
:10EE9000FFF778FF009B002B0ED1200017F0FDFE3E
:10EEA000074902000748F6F7D9FBF1F790F920006F
:10EEB00098470028E9D016BD684607F079FAFAE7C6
:10EEC0004C970300CCDC020037B50400FFF7B8F81C
:10EED000856A002D02D02000A8473EBD6A46102159
:10EEE0002000FFF74FFF009B002B05D06A4629004A
:10EEF000280017F026FFF0E7200017F0CEFE0349A8
:10EF000002000348F6F7AAFBF1F761F97E970300C8
:10EF1000CCDC020030B505008FB0FCF773F9280097
:10EF2000FFF78EF8846A002C05D02800A047040063
:10EF300020000FB030BD6A4610212800FFF722FFE5
:10EF4000009B002B16D002A8F1F726F9002807D164
:10EF50006A46010017F0F5FE0400F1F733F9E7E720
:10EF6000039B09491868F4F723FB0028E0D10398B4
:10EF7000F1F72DF9280017F090FE0449020004482B
:10EF8000F6F76CFBF4E7C0460CDC02007E9703004A
:10EF9000CCDC0200F0B585B003900F0016002028ED
:10EFA00004D1914210D0B14805B0F0BD039B1B2B9A
:10EFB00001D01E2B0DD131003800FFF7D7F8039B8D
:10EFC000002803D01B2BEED1A948EDE71B2BFBD16A
:10EFD000E9E7039B212B28D11000F6F787FB0028D7
:10EFE00006D03100380015F01DFC0028ECD1DAE71E
:10EFF0000324344000D05EE19E4B32689A4200D038
:10F0000059E173689C42CED2A300F3189D68280092
:10F01000F6F76CFB002800D14CE12900380015F010
:10F0200001FC0028D0D10134EBE70123194200D1C3
:10F03000FCE013404D100293002B00D1EEE0039B47
:10F0400054101D2B00D936E118000BF0AFF81E004C
:10F0500028002A002D0047004E00510053005E009A
:10F0600067007D008500BA001E0028002A002D00E0
:10F0700047004E00510053005E0067007D00850090
:10F08000D300D7003401DB00DF0025430295029B4B
:10F090005C00634000D5BDE00120204384E765406B
:10F0A000F4E72C400294F2E7002C04DA724973482A
:10F0B00015F0AEFBCFE01F2C08DC714B23419D42C5
:10F0C00004DCC0231B0623419D4205DAE917280012
:10F0D00017F019FF07004BE0A540D7E7002CE5DB50
:10F0E0001F2C00DD1F242541D0E72B190293CEE70A
:10F0F0002B1BFBE721002800F1F786F80028E5D15B
:10F10000012065436D0028434EE7002C00D1E5E067
:10F110002100280013F070FE0290B8E7002C00D107
:10F12000DCE028000CF0D8F9051C20000CF0D4F924
:10F13000011C281C0BF0ECFC0323050002209D435E
:10F14000504B2843C0182FE7002C00D1C6E0210007
:10F15000280013F041FEDFE72F00002C2EDA2800F4
:10F160000CF0BAF9032302279843464B0743FF18D4
:10F170003800FEF765FF8369002B00D19BE0320069
:10F18000390003989847002800D00DE793E0012349
:10F190001C4208D039000298F1F736F8002895D1C2
:10F1A000029B7B430293012C00D170E739003800A9
:10F1B0006410F1F729F8002888D17F43002CE6D1AC
:10F1C00065E7002C00D189E000210220F3F748FD1B
:10F1D00021000600280013F00FFE012740003843ED
:10F1E000B0602100280013F0F7FDB8400743F76036
:10F1F0003000D9E6A54200DAE6E6D4E6A54200DD15
:10F20000E2E6D0E6A54200DCDEE6CCE6A54200DB85
:10F21000DAE6C8E6029817F085FEC5E60323134038
:10F22000022B03D1184B1340062B5AD1039B1F2BE3
:10F230009ED13000FEF704FF83690400002B0CD13F
:10F24000636A002B26D1300017F027FD0F4902001A
:10F250000F48F6F703FAF0F7BAFF3A0031000398C7
:10F260009847002800D09FE6EAE7C046A4090300BB
:10F27000AC09030000CE02000197030044DD020048
:10F28000FFFFFF3F00008080070080FF4C970300D6
:10F29000CCDC02003000FFF7F1FD04002000FFF796
:10F2A00039FE002800D17EE63900FEF75FFF002816
:10F2B000F4D089E62E00039B38009A000D4BD458F9
:10F2C00017F0EBFC0500300017F0E7FC2B00009076
:10F2D000220009490948F6F7C1F9BCE7084909487D
:10F2E000E6E628000CF0F8F83200011C039805F05F
:10F2F00007FC48E774CE020016970300CCDC02003E
:10F300003B9703008CDD0200F0B513688DB00693C7
:10F31000002800D06CE00400131D0393FF220B00B3
:10F32000090A1340114001934B000593059A019B74
:10F3300004919B18039A9B00D558D3185F68381E18
:10F3400009D00020BB0706D1844B3A689A4202D10B
:10F35000380015F032FA049B1E18002D4DD1019B88
:10F3600076000133F3189800009319F0CAFD2500C8
:10F370000600002C01D001250460019BA8009A0022
:10F38000301803991CF0ADF8019B5B190293029BA6
:10F390009800049B3018DA00019B9900039B5918D0
:10F3A0001CF09FF8029A059B944663441C00002FB2
:10F3B0000FD003253D4000D09CE0684B3A689A424C
:10F3C00000D097E0380015F00EFA41688D4200D069
:10F3D0007FE0029B0299E21A520833000698FFF779
:10F3E00053FC0400300019F0B3FD20000DB0F0BD57
:10F3F000130008330393546890E7AB072FD12B68B1
:10F40000574A934202D0574A934228D128000AAA69
:10F4100009A9FEF79FFF099B019A01339B1876000B
:10F420009B199800009319F06CFD25000600002C34
:10F4300001D001250460019BA8009A0003993018AF
:10F440001CF04FF8019B0A995819099B80009A00FB
:10F4500030181CF046F8019B099A9B1895E7019B10
:10F460007600181D33189800009319F04AFD029495
:10F470000600002C02D0012304600293029B039932
:10F480009800019B30189A001CF02BF8019A029BFF
:10F490009446280063440293FFF7F0FC029B079018
:10F4A0009C000798FFF736FD051E00D16FE7009B13
:10F4B000029A934207D8D900300019F038FD0600AF
:10F4C000009B5B000093029B35510133029304348F
:10F4D000E7E78368EF00DA59002A09D0042A07D049
:10F4E000A300F2508268F318D219526802345A60AD
:10F4F00001356BE70AAAC5213800FFF773FC00212C
:10F500000AAA080017F01DFCFFF7B8FCA50001903F
:10F510000198FFF7FFFC071E00D15AE7009A631C11
:10F520009A420BD853000093042B01D2042300937A
:10F53000009B3000990019F0FAFC060009AA02218C
:10F540003800FEF729FF099B02341B687351099BA1
:10F550005A6873195A600835DAE7C04694D6020033
:10F5600000CE020060EC020073B50C0015008307AA
:10F570001ED10368204A934207D0204A934217D1F4
:10F5800001AA694616F0B2F903E001AA694614F02F
:10F590002FFE009B9C4228D817D3019BA4001C1966
:10F5A000043B043C9C4200D173BD226804C5F8E7CB
:10F5B000FFF764FC002306000093009B3000A34289
:10F5C00006D3FFF7A7FC0028EED022000C490EE07E
:10F5D000FFF7A0FC002808D0009A0A49A31A5B187C
:10F5E0009B00013258510092E7E7009A064907480C
:10F5F000F6F734F8F0F7EBFD00CE020060EC020005
:10F600006A980300FFFFFF3F4798030044DD0200B4
:10F61000F7B514000A0AFF230E0015001E401D4016
:10F6200083073BD107683D4B9F4208D03C4B9F422C
:10F6300034D1FF231143194224D12060F7BD01AA20
:10F64000694614F0D5FD009B72199A425ED89A0063
:10F650009446002001998200A84218D19B1BB50056
:10F660004919181AA41816F02AF9019B20605D198F
:10F670000023013601339E42E0D09A00514269587E
:10F68000A150F7E701AA694616F030F9DBE76746B3
:10F69000BF1A043FCF590130A750DCE7FFF7EEFB5C
:10F6A000002307000093009B9E4217D8002108000A
:10F6B00016F005F906003800FFF72CFC011E1AD1E0
:10F6C000B1688D4222D8AB00E3181E6088009C42CE
:10F6D00015D1491B300016F00EF9AFE73800FFF7DF
:10F6E00019FC002812D0009AB31A5B199B00013252
:10F6F00018510092D7E73000FBF7C4FDDBE7F26852
:10F70000C71AA218D259043B1A60E0E7009A0549CB
:10F710000548F5F7A3FFF0F75AFDC04600CE0200FA
:10F7200060EC02004798030044DD0200F0B587B0AA
:10F730001D0006000C000192FEF782FC2E4B984241
:10F7400007D12B00019A21003000FEF77FFF07B0A0
:10F75000F0BD876A294B002F08D09C4221D1300090
:10F76000B84728600028F2D00120F0E79C4218D169
:10F7700003AA10213000FFF705FB039B002B0CD1DF
:10F7800003AACD213000FFF72DFB059403AA002129
:10F79000012017F0D6FA2860E6E703AA39003800FE
:10F7A000F7E7002CECD1019B2000002BCFD01800F4
:10F7B000FEF746FC1249F3F7FBFE00280FD003AA20
:10F7C000CC213000FFF7DEFA039B002B07D003AA01
:10F7D0002100200017F0B5FA28602000B7E703AA3F
:10F7E000CE213000FFF7CEFA039B01AA002BCED129
:10F7F000019B02202B60AAE7A80403004CCA020068
:10F80000E8D8020010B50400F5F770FF002808D012
:10F81000002320001A001900FFF736FA0400200028
:10F8200010BD200014F0F8FF0028F8D10249034869
:10F8300014F0EEFFF2E7C046FF970300CCDC0200B5
:10F840007FB5C30006201843054B019004910520A5
:10F8500001A902930393059204F066FB07B000BD73
:10F860004CCA02001423F0B58DB000AFFA180500A1
:10F870000C00FFF787FABB69002B06D022002C4949
:10F880002C48F5F7EBFEF0F7A2FC786900284BD185
:10F89000280018F08FFC0028F0D014232800FA1854
:10F8A0000D21FFF76FFA10237869F918F8F7C4FDF6
:10F8B000B860200016F0CBFF6A463E69B968731C39
:10F8C0007B60C318FB600E33DB08DB00D31A9D4658
:10F8D000320068461BF005FE6D462E23AB557B6853
:10F8E0002000EB18BB6016F0B7FF0600200016F0F2
:10F8F000AEFF31000200B8681BF0F3FDF9686846FE
:10F90000FCF7DEFEC300062018430B4B10223B62BF
:10F910007B620A4BBA18BB620123FB620B33F861AE
:10F92000D118052004F000FBBD460DB0F0BDC04667
:10F930006897030024D902004CCA0200AC090300F6
:10F94000F0B5174C0F00616895B00391216806006F
:10F9500008A8049162602360F0F71EFC051E06D023
:10F96000039B09986360049B2360F0F730FC3368C5
:10F970003A00310005A80193F6F75AFB2B002A0044
:10F98000019905A8F2F760FF17F0C3F90500F0F739
:10F9900019FC2800039B6360049B236015B0F0BD35
:10F9A000AC09002010B50400FAF79EFA031E0648C1
:10F9B00004D0064914F02CFFF0F709FC220004499A
:10F9C000F5F74CFEF8E7C04698DA0200AA96030065
:10F9D000D3960300010010B5024814F019FFF0F7A8
:10F9E000F6FBC04610DB0200C3790248002B00D1B1
:10F9F00001487047AC090300A409030010B5FAF7E9
:10FA000055FD014810BDC0464CCA020010B508683B
:10FA1000FAF74CFD004810BD4CCA020073B50D004A
:10FA2000022838D1012601A96868F8F705FD764259
:10FA30003400019BC318834211D101A92868F8F74B
:10FA4000FBFC7342734162426241DBB2D2B2019964
:10FA5000FAF778FE002822D11149124817E00278FF
:10FA6000722A01D0772A06D1611C0ED1723A544213
:10FA700054410130DFE7622A01D0742A05D1711C9C
:10FA800003D1743A56425641F3E70749074814F048
:10FA9000BFFEF0F79CFB012676423400CDE776BD31
:10FAA0004C6903004CDB02009298030044DD020025
:10FAB00037B50400A068FFF72DFA019000280ED09A
:10FAC0006568074B9D4205D001AB0022012128004B
:10FAD000FFF7DAF8FEF7DAFC0028EBD001983EBD1C
:10FAE0004CCA0200002803D0012807D0002004E0FF
:10FAF0008B680448002B00D1034870478B685B007B
:10FB00001843FAE7AC090300A40903007FB5040019
:10FB10000122080001A9FEF735FD002221794020CD
:10FB200001F092FB0100050002980AF049FB6368AE
:10FB300006001A0A904217D9A368C1186943E06801
:10FB400019F0F5F92379E0602A00A0686360684342
:10FB5000E3687243181801991BF0C3FCA3680548B9
:10FB60009E19A66004B070BD121A1202DBB21343D4
:10FB7000EAE7C0464CCA0200F7B5FF274568040013
:10FB80000191BD431DD101792A00402001F05CFBA9
:10FB9000636806003B408027A1683F011F4308318E
:10FBA00041436760E06819F0C2F96368E0601A0ACF
:10FBB000A368013A013372435E43290080191BF0A8
:10FBC000ABFC2079019BA268E16801F091FCA3687D
:10FBD00003480133A3606368013BFF3B6360FEBDE4
:10FBE0004CCA020010B50400102019F09CF9024B19
:10FBF0004460036010BDC0469007030070B50A79E9
:10FC000004000D00002A0DD1194915F009FC01234B
:10FC1000AA68E9682000F7F7C7FE1649200015F02A
:10FC2000FFFB70BD144915F0C6FCAB68002BF4D087
:10FC30001249200015F0F4FB0026AB689E4204D365
:10FC40000F49200015F0ECFBE7E7002E03D00D492B
:10FC5000200015F0E5FB3200E968287901F016FB79
:10FC6000012201002000FEF703FA0136E5E7C04655
:10FC7000AC9803004A950300B8980300C3980300AA
:10FC80000ABD030000350300F8B5002207000D008F
:10FC90000100402001F0D8FA061E05D10C490D489C
:10FCA00014F0B6FDF0F793FA102019F02AF90A4B78
:10FCB0000400002F00D0094B28002360FBB2A56090
:10FCC0007043636019F01DF9E0602000F8BDC04684
:10FCD0009F98030044DD020028080300EC0703009E
:10FCE00070B506008AB00C00150012285CD003D84D
:10FCF000052826D0002454E01B2800D16CE01F28E2
:10FD0000F8D1012207A9280016F0DDFF03230028FF
:10FD10004FD01C4213D13B4B22689A420FD1012293
:10FD200004A9200017F06FF80123079A00930599A2
:10FD3000089B049815F0F3F9334C002831D1334C6B
:10FD40002FE0012204A9200017F05DF8280001220D
:10FD500007A9FEF717FC069B002203936B46402081
:10FD6000197B01F071FA0100060008980AF028FAE0
:10FD7000069BA16803936B4641180500187BFFF7AB
:10FD800083FF059B04001A000499C06803931BF0CD
:10FD9000A8FB2A000598E3687243181807991BF01E
:10FDA000A0FB20000AB070BD11002000FFF7AEFEDE
:10FDB000F7E7EA070DD41D4203D1154B2A689A4292
:10FDC00007D003232B40022BB9D1124B1D40062D27
:10FDD000B5D01148FFF7FEFD012204A9200017F05D
:10FDE00012F8012207A9280016F06DFF0028A6D0FE
:10FDF000089B059A00930499079B300018F074FA49
:10FE00009AE7C04628080300AC090300A4090300D0
:10FE1000E81F0300070080FFC7760300F0B5050068
:10FE200087B00E00002808D08B0726D10B68254A22
:10FE3000934202D0244A93421FD1012203A93000E9
:10FE400016F041FF002818D000222900402001F0C0
:10FE5000FBF90100070004980AF0B2F9060001005E
:10FE60002800FFF711FF320004007A430399C068AD
:10FE70001BF037FB200007B0F0BD3000FEF7E2FAC0
:10FE8000071E00D0471039002800FFF7FDFE0400D0
:10FE90003000FEF7F3FF002600900098FFF73AF8D5
:10FEA000031EE7D0002F04D119002000FFF764FEE5
:10FEB000F3E7721C0192E1683200280001F018FBA0
:10FEC000019EEAE790E702002808030070B50500EC
:10FED00086B0161E44D003240C402DD1214B0A6855
:10FEE0009A4229D103AA806804F0B6FC002802D106
:10FEF0001D48FFF76FFD2000042E1BD12200297939
:10FF0000402001F0A1F9049B06000093039B28798F
:10FF10000193019A009B991AFFF7B6FE040003991A
:10FF2000049AC068521A71437243EE6871181BF04C
:10FF3000D8FA200006B070BD0A000023A96828681E
:10FF4000FEF73EFA02002879042E03D1E96801F099
:10FF50009DF9EFE73300E96801F0CAFA0348E9E7E1
:10FF60001000E7E7EC000300053503004CCA02006F
:10FF700037B50C00110000221D0000920123200063
:10FF8000F3F776FC002C04D121002000FFF77CFE63
:10FF90003EBD2968CB0705D48B0713D10B4B0A68EC
:10FFA0009A420FD10800FEF733F901000500002046
:10FFB000FFF76AFE04002A000021C0681BF0ACFABB
:10FFC0002000E5E70020FFF729FFE1E7E81F030035
:10FFD00010B5102018F095FF0400034B08C015F071
:10FFE00099FE200010BDC046E81F030070B50C004C
:10FFF000052804D80AF0C6F806030E04151E0024CE
:020000040001F9
:10000000200070BD081D15F0B6FF0E4C0028F7D07B
:100010000D4CF5E7081D16F0D4FA01244000044306
:10002000EEE7FFF7D5FF211D0500043015F0D6FFE0
:100030002C00E5E7FFF7CCFF211D0500043015F08B
:10004000DDFFF5E7AC090300A409030070B5050066
:1000500083070CD1104B02689A4208D1FFF7B8FF12
:100060000400291D043015F0AEFF200070BD2800EB
:10007000FEF7CEF8C0231B06984205D18020002150
:10008000C00516F040FFF1E7C21783180120534066
:100090005B001843EAE7C046E81F030070B5440060
:1000A0006408051C211C201C0BF0DEF9002820D15F
:1000B0001149201C0AF05EFA002814D1281C18F0FF
:1000C000F4FE002808D0FFF783FF0400291C043049
:1000D00015F09FFE200005E0281C0BF0DDF901243F
:1000E0004000204370BD05490548F5F7B7FAF0F721
:1000F0006EF804490448F8E7FFFF7F7FF498030097
:1001000088DB02000D99030044DD020007B5C30738
:1001100001D540100EBD043001A9FCF7B5F8002848
:1001200001D00198F6E70349034814F071FBF0F79A
:100130004EF8C046C798030088DB02000123F0B5E3
:100140008DB006000C0000920B402ED04B10022206
:1001500002A903A815F01CFE03AD009BDB072ED5FA
:10016000009B02225B1002A903A815F011FE03AC4C
:10017000092E01D0162E3ED1200015F0FCFE0028DD
:1001800067D1280016F073FA051C200016F06FFAEC
:10019000011C281C0AF0BCFC0323020002209A4325
:1001A0008D4B1043C0180DB0F0BD0320084000D0A7
:1001B00007E18A4B0A689A42F5D10D1DCDE703236A
:1001C000009A1A4208D10099844A09680191914223
:1001D00002D1009B1C1DCBE7009A1340022B04D1D7
:1001E0007F4B1340062B00D0EDE0009A2100300039
:1001F00006F07CF8D7E7182E00D9BAE0FFF7E8FE42
:100200000700300009F0BEFF6E74687A7A0D131A89
:1002100020DD4D8E946E74687A7A0D131A20DD4DB0
:100220008E0022002900381D15F07FFF04E0381DE4
:100230002200290015F0B3FF3800B4E7381D220072
:10024000290016F0F9F8F7E7200015F094FE0028D1
:1002500005D06449644814F0DBFAEFF7B8FF06A84C
:100260003E1D15F057FD23002A0006A93000FBF7BC
:100270009FFE2B7822785340DB070ED506A815F099
:100280007AFE002809D1012109A8494215F076FD1E
:1002900009AA3100300015F048FF06A815F046FD08
:1002A000CAE7200015F067FE0028D2D109A83E1D3C
:1002B00015F030FD23002A00310009A8FBF778FE75
:1002C00009A815F033FD2B7822785340DB07B3D50E
:1002D000220031003000A7E7381D2200290015F068
:1002E000A6FFA9E7381D2200290016F022F8A3E78F
:1002F000381D22002900FBF7E7FD9DE70098FFF776
:1003000005FF021E02DA39493948A4E7381D2900E1
:10031000032E01D0102E02D1FBF76AFD8CE715F0F9
:10032000A4FE89E7381D2200290016F008F983E7AA
:10033000200015F020FE00288BD1FFF749FE3E1D5E
:10034000009023002A0004303100FBF731FE2B78A7
:1003500022785340DB0704D522003100300015F02D
:10036000E4FE009B09A9022009930A97F2F778FCA2
:1003700019E72100280015F003FE193E03000020B4
:10038000042E00D90FE7300009F0FCFE0309160D1A
:1003900012001848002B00DB05E7174803E7154853
:1003A000002BFADCFFE61348002B00DDFBE6F4E748
:1003B0001048002BF1DAF6E60E48002B00D0F2E6EA
:1003C000EBE70020EFE6280016F051F9009A011C37
:1003D000300004F095FBE6E600008080E81F030093
:1003E000070080FF3B9703008CDD020001970300AC
:1003F00044DD0200A4090300AC090300F8B50500C0
:1004000010200C0016001F0018F088FD011E09D0F6
:1004100044608460A4190760C460034B034A280049
:1004200012F0B0FDF8BDC046DD6F0200C76F0200DC
:10043000F0B5802787B02C4D02907F422C78002C9D
:100440001CD063B2002B10DA6E1C6D787C40E4B2D5
:10045000002D13D0013CE4B2FF2C0DD004AB981D4D
:100460000121057002F01AF9F4E704ABD81D01214F
:1004700004702E0002F012F9751CDFE70627013F19
:10048000002F2ED0029802F053F90124BC42F6DA74
:100490000025052D22D0154E220029003000F5F749
:1004A0006FFC6B4601901B79002B15D0631E1A0060
:1004B000290030000393F5F763FC031E0CD12200E2
:1004C00029003000F5F724FCFF22019B290013408E
:1004D0003000621EF5F71CFC0135DAE70134E4B2A6
:1004E000D4E707B0F0BDC0462699030018000020ED
:1004F00010B5C820FFF79CFF004810BD4CCA020091
:10050000F8B50D0004001600EFF7C2FE2B0003271C
:1005100023433B4219D1BE4217D9B208290020001B
:1005200009F0CAFD3100B94360183E406918002E39
:1005300002D032001AF01CFF80220549D2008B58ED
:10054000002BFCD0EFF794FEF8BD29002000EEE769
:1005500000E00140F8B5040005200D0009F0D8FCCA
:100560002000FDF755FE554C20702800FDF750FE89
:10057000534BC0B218702378012B1DD0022B1DD015
:10058000102B1DD00F2B1DD0052B1DD00E2B1DD0D9
:100590000D2B1DD04B4C4C490B2B08D1012819D0E9
:1005A000022800D17BE0494A102814D04849494824
:1005B00014F02EF9EFF70BFE474CEFE7474CEDE751
:1005C000424CEBE7464CE9E7464CE7E7464CE5E7AB
:1005D000464CE3E7404AA02504216379ED05C13389
:1005E000FF339B005951517903200B00C133FF3376
:1005F0009B005851012318008840A121C900685070
:100600000A200138C046C046C046C046C046C04663
:10061000C046C046C046C046C046C046F1D1527929
:10062000A2279340324AFF00AB5006F005FE314E40
:100630003060EB596279D340DB0708D406F0FCFD4B
:100640002D4B18603368C01A2C4B9842F1D906F034
:10065000F3FDA027A2262A4DFF052860F600BB590E
:100660006279D340DB0708D506F0E6FD254B18601C
:100670002B68C01A214B9842F1D906F0DDFD1E4BC4
:10068000214C18602B68C01A204B421E1860204B6A
:100690009A4206D9012023685B001843F8BD0F4A2F
:1006A00099E70AF069FF1B490AF022FC1A490AF08F
:1006B0002FFA0AF0F1FE2060ECE7C0463509002071
:1006C00036090020241E0300C49903004C1E0300B9
:1006D000039A0300CCDC02005C1E03006C1E0300C6
:1006E000441E0300841E03003C1E0300341E03004E
:1006F0000C05000018030020080B0020C8AF000004
:10070000040B00200C0B00204C030020100B0020D9
:10071000C6AF0000000008420000FA4410B50348CC
:100720000968FDF7C9FC024810BDC046B4EA0200E2
:100730004CCA0200F7B5244900250B000833DA6FD4
:10074000224B94461B785488981C80001618805AB7
:10075000883144430968A4120195F078002823D019
:10076000B07801268640A1273000A026FF00F605BC
:100770000133F051DBB2981C80001618805A070034
:10078000508878438012001BE7D0104A1370019BF9
:10079000002B02D00C4B88331960002D03D0624629
:1007A000094B0833DA67FEBDA024094B5668E405FF
:1007B000E650002902D10B000C00DCE701258C4635
:1007C0000A0001950100F6E7AC0900203709002076
:1007D0000C050000044B05491A000832D1670022BD
:1007E00088331A607047C046AC090020980903009E
:1007F00010B5782202490220EFF7F8FD10BDC0467F
:1008000035070100421E104BFF3A70B59A4218D8C6
:10081000061172B60D4C00212300220088331D689A
:100820000832196062B68D4200D1D56F2978280050
:1008300016F000FC6B68883443604680206000201E
:1008400070BD01204042FBE740410F00AC09002091
:10085000054B1A0088331B680832002B00D1D36F78
:10086000588800017047C046AC090020F7B5414ADE
:1008700007000B00914200D913008022D200D21A47
:10088000019272B63C4A0020110088321468083187
:10089000106062B6844200D1CC6F0126BE4062680F
:1008A000324207D13A00A0210320C132FF32920028
:1008B000C9055050002521788D421CDB002B19D032
:1008C0000131200016F0B6FB6A46636892881E4329
:1008D000466023789B00C3181A8101229F72DA7246
:1008E00001216388021D4380037899421CDB224B5F
:1008F00088331860F7BDAA00A218927A97422CD0CC
:100900000135D9E70139200016F094FB6368B34341
:10091000436023785A1EAA42E2DD01339B00023570
:100920001B59AD002B50DBE71700D37A1489967A58
:1009300001934B1EBD88A54204D97D68043FFD602C
:10094000013BF7D203339B00C3181C806C4624790B
:100950009E70DC7001310432C6E7002BD2D020003B
:1009600016F068FB6368023543606B469B88AD00F8
:100970002B52B5E7FF030000AC09002010B50021A1
:100980000400FFF773FF0D4B0833DA6F0023107874
:10099000834200DB10BD99005118897A8C4201D046
:1009A0000133F5E702339B00D3181F229A7001230D
:1009B000A021A340024AC9058B50EBE7AC090020F7
:1009C0000C05000010B50B790349002B00D1034939
:1009D00014F026FD10BDC046C07B0300B87B0300A9
:1009E00037B50C00110000221D00009201232000E9
:1009F000F2F73EFF054B002C06D02868FDF746FDB8
:100A0000034B002800D1014B18003EBDA409030090
:100A1000AC0903000300203B5E2B00D93F200523D7
:100A200020384343014A1068C01870477000002006
:100A300070B50500080068430130401008300C0014
:100A400018F05FFA0122044B857103600379447149
:100A50009343037170BDC046800D030010B50400C0
:100A6000102018F04EFA044B036063684360A368DB
:100A7000C3600023836010BD540A030070B50500F5
:100A8000202018F03EFA05210B4B040003600800FB
:100A9000FFF7CEFF6B68EA68A060236162602A7C82
:100AA0002000A276AA689B1863616B7CE37616F03F
:100AB0001BFB200070BDC046C80D0300037910B5B4
:100AC000DB0705D50349044813F0A2FEEFF77FFBCF
:100AD00010BDC046289A0300CCDC020070B50D00A2
:100AE0000400FFF7EBFF2800FDF792FB0100092847
:100AF00005D90549054813F08BFEEFF768FB200088
:100B000016F054FB024870BDD639030044DD0200E4
:100B10004CCA0200F0B50C000B6889B00700180041
:100B20000493FFF7CBFF65682800FDF789FA1F4B98
:100B30001F49984202D1072F05D11E491E4813F0C4
:100B400067FEEFF744FBA068FDF762FB0690E068E4
:100B5000FDF75EFB07902069FDF75AFB0590606981
:100B6000FDF756FB059B0600002B01DB002802DA8F
:100B700012491348E3E7062F14D0A069FDF748FB9C
:100B80000700E069FDF744FB059B039000932800F4
:100B900002970196079B069A049916F0B8FB09483C
:100BA00009B0F0BD00200700EEE7C046800D03004D
:100BB000559A0300689A0300CCDC0200829A030075
:100BC00044DD02004CCA020070B5040008001600A3
:100BD000FDF71EFB05003000FDF71AFB0600002D97
:100BE00001DB002805DA0D490D4813F011FEEFF77F
:100BF000EEFA200016F076FB854204DA200016F0AB
:100C00007FFB864201DB0749EEE732002900200026
:100C100016F05AFB43000120184370BDC69A03002A
:100C200044DD0200DF9A0300F8B50D000C682000D7
:100C3000FFF744FF6868FDF7EBFA0600A868FDF7C8
:100C4000E7FA0700002E01DB002805DA10491148F9
:100C500013F0DEFDEFF7BBFAE868FDF7D9FA0500FF
:100C6000092801D90C49F2E7200016F03BFB864227
:100C700004DA200016F044FB874201DB0749E6E76F
:100C80002B003A003100200016F069FA0448F8BD44
:100C9000C69A030044DD0200D6390300DF9A030040
:100CA0004CCA0200F7B50E0026490400019214F068
:100CB00082FC019B002B03D12349200014F07BFC14
:100CC0002249200014F077FC0025300016F018FBB4
:100CD000854221DA0027300016F004FB87420CDA47
:100CE00039002A00300016F0EFFA194B19491A5C46
:100CF000200014F060FC0137EDE71749200014F0E4
:100D00005AFC019B002B05D1300016F0F9FA01388E
:100D1000854211DB0135D8E70C49200014F04BFC6B
:100D2000019B002B03D10D49200014F044FC0C4919
:100D3000200014F040FCF7BD0A49200014F03BFCF1
:100D4000E8E7C0466E9B0300759B0300839B03008E
:100D5000859B0300996703007B9B030007B003009A
:100D60004A9503007D9B0300F0B50F00110000229F
:100D70008BB01E00009203233800F2F779FD032F99
:100D800000D9D5E0380009F0FDF9020C9494052152
:100D90000800FFF74DFE040016F016FA20000BB015
:100DA000F0BD3068654B0340062B07D0830700D0A9
:100DB000C1E0634B02689A4200D0BCE007A9F7F794
:100DC0003BFB079B03900593012B04D1039B1878F1
:100DD00016F09DFCE3E700231E00039A029303999B
:100DE0000598511A814218DA11780A2901D03A2956
:100DF00008D19E4200DA1E00029B013302930023B9
:100E00000132ECE701332029FAD03929F8DD4D49C8
:100E10004D4813F0FDFCEFF7DAF9002B05D0029AEC
:100E2000013202929E4200DA1E0002993000FFF762
:100E3000FFFD002507002C00039B0493039A049BED
:100E40009B1A059A9A4223DD049B1B780A2B01D03A
:100E50003A2B0FD1A64207DD210000232A003800DB
:100E600016F07DF90134F5E700240135049B0133C8
:100E70000493E3E7202B07D1002321002A00380048
:100E800016F06DF90134F1E7392BEFDC303BF4E774
:100E9000029B3800AB4200DC81E7A64207DD21005F
:100EA00000232A00380016F05AF90134F5E738001B
:100EB00075E73068FDF7ACF905007068FDF7A8F933
:100EC000029001002800FFF7B3FD0390022F03D129
:100ED00016F07AF9039862E7012207A9B068FDF7D6
:100EE00051FB002D1FDB029B002B1CDB6B43089A80
:100EF000934218D100242700029B9C42EAD03E0076
:100F0000EB190493049BF11B9E420ED0079B9A5D44
:100F1000131C092A00D90923DBB22200039816F01A
:100F20001EF90136EEE7094972E77F190134E3E75C
:100F3000074908486DE70849FBE7C046070080FFFE
:100F4000DC140300EF9A030044DD0200199B030048
:100F5000369B0300CCDC0200559B0300F0B585B046
:100F6000019105000021019809F0F0FA041E05D056
:100F70002349244813F04CFCEFF729F9280016F018
:100F8000B1F90600280016F0BBF901003000FFF7A8
:100F90004FFD0700280016F0A5F984422CDA002640
:100FA000280016F09FF9864224DA3200210028003A
:100FB00016F08AF90AF090FA019909F099FF0CF0FD
:100FC00071F80022104B0AF01DFB104B002202901A
:100FD000039109F081FA0923002804D002980399AB
:100FE0000BF0EAFF030032002100380016F0B7F8DA
:100FF0000136D5E70134CDE7380005B0F0BDC04675
:101000009A9A030044DD02000000E03F0000224005
:10101000F0B587B007000391059216F071F904004E
:10102000380016F05FF90190039816F069F98442D0
:101030002DD121000198FFF7FBFC0025029006E06E
:10104000049B1B1ADA43D217134019E00135019BA8
:101050009D4222DA0026A642F8DA32002900380042
:1010600016F032F9320004902900039816F02CF99A
:10107000059B002BE4D0049B1B18092B00DD0923E2
:1010800032002900029816F06AF80136E3E70449B5
:10109000044813F0BDFBEFF79AF8029807B0F0BDD3
:1010A000909B030044DD0200F8B5040008000D0029
:1010B0001600FCF7C5FF164FB84201D000200FE024
:1010C000053C042CFAD8200009F052F8141403F857
:1010D0000B003000FDF700F9011C2800FFF73EFF70
:1010E000F8BD3000FDF7F8F8011CFE20800509F07E
:1010F0000FFDF1E73000FCF7A3FFB842DED16242FA
:1011000062413100D2B22800FFF782FFE8E7C04613
:10111000800D0300F7B507000193142008AB0E0003
:1011200015001C7817F0EDFE044B476003606B461A
:101130001B798660C56003744474FEBD040E030011
:1011400070B505000C2017F0DCFE0521044B0400EF
:10115000456003600800FFF76BFCA060200070BDD5
:10116000080A030010B54A68014914F024FA10BDBA
:101170007B97030070B5050000291CDB032905D807
:101180000800002408F0FEFF1818060601230239A3
:1011900099430C00FE26B52109023143280016F0C0
:1011A0001FFB002C04D005492800214316F018FB32
:1011B000EE612C6270BD0024F226ECE780B00000E6
:1011C000F0B5060000248BB0184B1948E158FFF722
:1011D000C5FE03AFE05104341C2CF5D114230024C8
:1011E0007343019300257959124813F02BFB043502
:1011F000300001F09DFA1C2DF5D1163DAB000D48D5
:10120000F95813F01FFB300001F092FA013DF5D2BE
:101210000134082C03D1F4F75BFD0BB0F0BD0123C2
:101220001C42DFD1019801F083FADBE7B80E03001E
:101230009C1703001800002010B51920FFF7C0FF0D
:10124000004810BD4CCA02003E2803D040280CD0F4
:101250003C2811D14239C9B22F290DD8084B585C0E
:101260000123002A00D013607047712904D8054B70
:10127000585C054B5B56F4E701230020F1E7C046BC
:10128000AE9B0300DE9B0300509C030010B5512869
:101290003DD011D849282ED007D8422803D048285D
:1012A00026D0002806D18B5C10E04F284BD017D8F1
:1012B0004C2820D0002309E0682816D00AD86428DA
:1012C00036D066282AD06228F4D18B5601205B00E4
:1012D000184314E06C2803D0712811D06928E9D193
:1012E0009200505815F01EFE09E05200535EEDE7E3
:1012F0005200535AEAE79200505815F02EFE10BDE6
:10130000D2008A181068516815F0FDFDF7E7D20089
:101310008A181068516815F011FEF0E70323920057
:1013200050589843030002201843084BC018E6E7C2
:10133000D2008A18106851680BF006FF03230200E0
:101340009A431300EFE792005058D8E700008080DE
:10135000F7B51700156801AA04000E00FFF774FF27
:10136000402C05D1019B043C5A1EAA185D42154031
:101370005A213E3C62426241B14289412B183B6096
:10138000D2B22B00494216F0FAFA04000D004F2E9B
:1013900008D0532E07D11AF025FA002201002000B0
:1013A000F6F79CFBFEBD662E06D10323022498436C
:1013B000154B2043C018F5E7642E06D10BF0C4FE90
:1013C0000323040002209C43F2E75A2E0FD9802207
:1013D0000023D20512196B41002B04D1002A02DB35
:1013E00015F0A0FDDEE7290015F08DFDDAE70029F4
:1013F00005D1064B984202D815F0AFFDD2E729007F
:1014000015F09CFDCEE7C04600008080FFFFFF3F47
:10141000F0B587B0140003AA07000E0001931D6801
:10142000FFF712FF0090402F05D1039B043F5A1E87
:10143000AA185D421540009B019AEB1813603E3FCD
:10144000642E14D0662E0DD04F2E2ED179424F41EE
:101450000098F9B2042800D9042023002A0016F0CD
:10146000B7FA30E02000FCF737FF0400EEE7200079
:10147000FCF732FF0BF016FE0490059139004B4249
:101480005941C9B28B0006AAD318083B2A001B6831
:10149000042016F09DFA3B005A1E934106AA9B00B9
:1014A000D318083B04351C68D0E7A3070DD10F4BB8
:1014B00022689A4209D179424F412B00F9B2009A31
:1014C000200015F006FD07B0F0BD2000FCF7A0FEDF
:1014D000009B0400042BB9D95A2EB7D90028B5DADD
:1014E0001A1F281DFF211AF017F8AFE7E81F0300A5
:1014F00070B505000E0014001800642D0CD0662D88
:1015000004D04F2D11D19400A35104E094000E1982
:10151000FCF7E2FE306070BDD4000E19FCF7DCFE73
:101520000BF0C0FD30607160F5E720232B43712B79
:101530000CD10321014009D1094B02689A4205D11F
:10154000E300F318082215F0C4FCE4E7FCF760FEA2
:10155000220003003100280016F04DFADBE7C046F8
:10156000E81F03000139C9B2054B401880301970DB
:10157000044A03781370044AD25C044B1A70704713
:10158000390900203A09002081AE03003809002003
:101590000131C9B2054B401880301970044A0378F4
:1015A0001370044AD25C044B1A707047390900204A
:1015B0003A09002081AE030038090020074B984209
:1015C00006D9074B1818074B4118C91808787047F7
:1015D000054B18184118054BF7E7C046A4920000C8
:1015E000C2AC03005B6DFFFFD69C03000083FFFFCE
:1015F000030020228033F0B504001A707F200022FF
:101600004F255F2689B0A15C531C0A00DBB2024063
:101610006F2A28D90A003240E11880310A701A0076
:101620007F2BF0D1BB4A137023001B22FF331A70AB
:10163000E4320192531CDBB203936B46B6481B7B2A
:10164000B6490370039BE31880331B780B705B2B48
:101650000ED19B22019B0A700133DBB20370E2546E
:10166000012009B0F0BD5F2AD6D90A002A40D3E78D
:101670002E2B13D10232D2B20270A218803212780D
:10168000A4480270A648825C0120024206D1019A59
:101690000B701218D2B20192A3546FE202209D4A3D
:1016A00013709F4AD25C104000D0ADE0002A19D1DF
:1016B0009948203203780A70E31880331A70019B2E
:1016C0000133DBB201936B461B790370019B782BCE
:1016D00001D8E25452E29B23019AA3546B461B7B30
:1016E0000B70BDE716007F2552B2AE430E70002A84
:1016F00003DB8C4A8C4B1A60B3E7413B8B4ADBB26D
:101700008B49D25CCB5C120213430293029B0021F3
:1017100001339BB218000293FFF750FF0306F5D583
:101720000123012700267B4D2B7039000298FFF71B
:1017300045FF7B1CDBB2282868D1002E00D02F701B
:101740002B780133DBB2059305990298FFF736FF3A
:10175000059B0133DBB22928F5D17F250493049939
:101760000298FFF72BFF049B28400133DBB23D2892
:101770004FD16A46694B127B1870674B00261A706E
:101780006A467B1CDBB200931278624B039D1A7091
:101790000695631980331B78009902980793FFF729
:1017A0000DFF079B8342B1D1009B05990133DBB24A
:1017B0000093009A6B1CDBB28A422CD1002E01D020
:1017C000554B1D70039D013FFFB2524B39000298EB
:1017D0001F70FFF7F3FE514E030600D504E14E4B98
:1017E0007F2118704E4B1B5C1A005BB28A4332702B
:1017F000002B14DA484B013DEDB21D7063198033A4
:101800001B789842DFD081E74A4B7EE71F00012614
:101810008BE70493A3E71D0001260693B9E7307018
:1018200020281BD0232825D02E282CD0262832D0A3
:1018300040284ED05E2856D02B285CD03A2800D0C5
:101840000EE1202629002000FFF78CFE334A137892
:1018500033401370B7D0304B1D78F3E729002000D8
:10186000FFF780FE0023F356002B00DA4EE72A4BE9
:101870001D78A8E729002000FFF774FE4022337886
:101880001342F4D142E729002000FFF76BFE3378C2
:101890001B07ECD43AE729002000FFF763FE102273
:1018A000337813403370E2D11B4B1B78E118803141
:1018B00009783170482900D028E7013B1649DBB28E
:1018C0000B70E31880331B789343432B00D01DE744
:1018D000CDE729002000FFF745FE042233781340AE
:1018E0003370C4D112E729002000FFF73BFE3378A4
:1018F0009B06BCD40AE7084B013DEDB21D7065198B
:1019000080352B78452BB2D010229343492B00D041
:10191000FCE6ACE73A09002039090020380900202C
:1019200081AE0300C29C03005000002007AF0300FB
:10193000EDAE0300A59200006B1C934ADBB213705E
:10194000E31880331B7891490B70452B36D1A81CC6
:10195000C0B2231880331B788D4E33708D4EF656EF
:10196000002E02DB884B1D783FE010700B70522B6D
:10197000F8D0532BF6D0442BF4D04C2B08D10335A0
:10198000EDB21570651980352B78592BEAD0BDE67C
:10199000462B00D0BAE6EB1CDBB21370E3188033A1
:1019A0001B780B70552B00D0B0E60435EDB21570E6
:1019B000651980352B784C2BD4D0A7E6492B00D065
:1019C000A4E6AB1CDBB21370E31880331B780B70FA
:1019D0004E2B00D09AE60335EDB2157065198035AF
:1019E0002B78472BBED091E6069D6A46009B0133BB
:1019F000DBB200931278664B1A70009B049A9342F4
:101A000000D19CE019000298FFF7D8FD614B7F21BF
:101A10001B5C5D4F1A005D4E8A435BB238703270BA
:101A2000002B08DA0135EDB2631980331B783D7065
:101A30009842DAD06AE63070202816D023281ED0CB
:101A40002E2826D026282DD0402848D05E2851D0D8
:101A50002B2858D020263A2864D0252800D16BE7BF
:101A60004D4A4E4B00201A60FBE529002000FFF78D
:101A70008FFD0023F356002B00DB73E746E62900B9
:101A80002000FFF785FD40223378134200D069E73C
:101A90003CE629002000FFF77BFD33781B0700D5CB
:101AA00060E733E629002000FFF772FD102233784B
:101AB0001340337000D055E73B78E1188031097846
:101AC0003170482900D021E60133DBB23B70E318C6
:101AD00080331B789343432B00D017E642E729005D
:101AE0002000FFF755FD042233781340337000D0F7
:101AF00038E70BE629002000FFF74AFD33789B0604
:101B000000D52FE702E60135EDB23D70651980354D
:101B10002B78452B00D125E710229343492B00D089
:101B2000F4E51FE729002000FFF732FD174A13787C
:101B30003340137000D158E7134B1D78F2E70025AE
:101B40007F272E0000990298FFF738FD03003B40E5
:101B50003D2B04D0019A0132D2B20192A354009AD3
:101B60000132D2B201060BD5002E03D06946084AD5
:101B700009781170054A1370069B0393039A59E57F
:101B800000920126DEE7C04639090020380900200E
:101B90003A09002081AE0300CC9C030050000020D5
:101BA000F0B58BB0079310AB10CB009001911B7870
:101BB000062A12D8012A08D93F230B700B000133E3
:101BC0000193002301990B7001E0002AF9D1012053
:101BD0009042804140420BB0F0BD009900292ADAC2
:101BE000019B01995F1C2D230B70802109068C46F7
:101BF000009B63440093019BFF210993009BC9054F
